:020000022000DC
:1060000000000420CD910200098402006189020091
:1060100009840200098402000984020000000000D3
:1060200000000000000000000000000009840200E1
:1060300009840200000000000984020009840200B3
:106040007990020009840200D19502001D9202009D
:106050002D9202000984020089870200098402004F
:1060600009840200B1950200C19502009D910200D1
:1060700009840200098402000984020009840200E4
:10608000F9950200AD910200098402000984020022
:10609000098402000984020095920200098402002A
:1060A00009840200098402000984020009840200B4
:1060B00009840200098402000000000000000000C2
:1060C0000984020009840200098402003D92020052
:1060D000BD9102000984020009840200F1950200CA
:1060E000E1950200799102000984020069920200A0
:0860F000000000000984020019
:1070000040F8044B40F8045B40F8046B40F8047B04
:1070100040F8048B40F8049B40F804AB40F804BBF4
:1070200040F804CB40F804DB6846704781F000412B
:1070300002E000BF83F0004330B54FEA41044FEA5D
:10704000430594EA050F08BF90EA020F1FBF54EAF8
:10705000000C55EA020C7FEA645C7FEA655C00F094
:10706000E2804FEA5454D4EB5555B8BF6D420CDD65
:107070002C4480EA020281EA030382EA000083EAE8
:10708000010180EA020281EA0303362D88BF30BD88
:1070900011F0004F4FEA01314FF4801C4CEA1131DE
:1070A00002D0404261EB410113F0004F4FEA03333D
:1070B0004CEA133302D0524263EB430394EA050FC8
:1070C00000F0A780A4F10104D5F1200E0DDB02FA37
:1070D0000EFC22FA05F2801841F1000103FA0EF2CB
:1070E000801843FA05F359410EE0A5F120050EF191
:1070F000200E012A03FA0EFC28BF4CF0020C43FAC2
:1071000005F3C01851EBE37101F0004507D54FF0CE
:10711000000EDCF1000C7EEB00006EEB0101B1F51E
:10712000801F1BD3B1F5001F0CD349085FEA300064
:107130004FEA3C0C04F101044FEA445212F5800F6F
:1071400080F09A80BCF1004F08BF5FEA500C50F10C
:10715000000041EB045141EA050130BD5FEA4C0CEF
:10716000404141EB0101013C28BFB1F5801FE9D24C
:1071700091F0000F04BF01460020B1FA81F308BF6F
:107180002033A3F10B03B3F120020CDA0C3208DD3B
:1071900002F1140CC2F10C0201FA0CF021FA02F116
:1071A0000CE002F11402D8BFC2F1200C01FA02F186
:1071B00020FA0CFCDCBF41EA0C019040E41AA2BFAB
:1071C00001EB0451294330BD6FEA04041F3C1CDA73
:1071D0000C340EDC04F11404C4F1200220FA04F093
:1071E00001FA02F340EA030021FA04F345EA03013D
:1071F00030BDC4F10C04C4F1200220FA02F001FAFF
:1072000004F340EA0300294630BD21FA04F0294680
:1072100030BD94F0000F83F4801306BF81F4801119
:107220000134013D4EE77FEA645C18BF7FEA655C8C
:1072300029D094EA050F08BF90EA020F05D054EA5E
:10724000000C04BF1946104630BD91EA030F1EBF63
:107250000021002030BD5FEA545C05D14000494167
:1072600028BF41F0004130BD14F580043CBF01F55A
:10727000801130BD01F0004545F0FE4141F4700140
:107280004FF0000030BD7FEA645C1ABF194610461B
:107290007FEA655C1CBF0B46024650EA013406BF1C
:1072A00052EA033591EA030F41F4002130BD00BFDB
:1072B00090F0000F04BF0021704730B54FF4806498
:1072C00004F132044FF000054FF0000150E700BF19
:1072D00090F0000F04BF0021704730B54FF4806478
:1072E00004F1320410F0004548BF40424FF0000165
:1072F0003EE700BF42004FEAE2014FEA31014FEAA8
:1073000002701FBF12F07F4393F07F4F81F06051F6
:10731000704732F07F4208BF704793F07F4F04BF41
:1073200041F40021704730B54FF4607401F000451E
:1073300021F000411CE700BF50EA010208BF70477E
:1073400030B54FF000050AE050EA010208BF70476F
:1073500030B511F0004502D5404261EB41014FF4D8
:10736000806404F132045FEA915C3FF4D8AE4FF0E0
:1073700003025FEADC0C18BF03325FEADC0C18BFC3
:10738000033202EBDC02C2F1200300FA03FC20FA14
:1073900002F001FA03FE40EA0E0021FA02F1144461
:1073A000BDE600BF4FEA4102B2F1E04324BFB3F5AE
:1073B000001CDCF1FE5C0DD901F0004C4FEAC0026C
:1073C0004CEA5070B2F1004F40EB830008BF20F050
:1073D0000100704711F0804F21D113F13872BCBF0A
:1073E00001F00040704741F480114FEA5252C2F15F
:1073F0001802C2F1200C10FA0CF320FA02F018BFA8
:1074000040F001004FEAC1234FEAD32303FA0CFCFA
:1074100040EA0C0023FA02F34FEA4303CCE77FEA89
:10742000625307D150EA01331EBF4FF0FE4040F4D3
:107430004000704701F0004040F0FE4040F4000082
:10744000704700BF80F0004002E000BF81F00041C3
:1074500042001FBF5FEA410392EA030F7FEA226CFA
:107460007FEA236C6AD04FEA1262D2EB1363C1BF8A
:10747000D218414048404140B8BF5B42192B88BFF9
:10748000704710F0004F40F4000020F07F4018BF1C
:10749000404211F0004F41F4000121F07F4118BF3C
:1074A000494292EA030F3FD0A2F1010241FA03FCE4
:1074B00010EB0C00C3F1200301FA03F100F00043CC
:1074C00002D5494260EB4000B0F5000F13D3B0F194
:1074D000807F06D340084FEA310102F10102FE2A03
:1074E00051D2B1F1004F40EBC25008BF20F0010073
:1074F00040EA03007047490040EB0000013A28BF12
:10750000B0F5000FEDD2B0FA80FCACF1080CB2EB94
:107510000C0200FA0CF0AABF00EBC2505242184312
:10752000BCBFD0401843704792F0000F81F40001B7
:1075300006BF80F400000132013BB5E74FEA41038A
:107540007FEA226C18BF7FEA236C21D092EA030FF6
:1075500004D092F0000F08BF0846704790EA010F70
:107560001CBF0020704712F07F4F04D1400028BF9D
:1075700040F00040704712F100723CBF00F500007F
:10758000704700F0004343F0FE4040F400007047B5
:107590007FEA226216BF08467FEA23630146420261
:1075A00006BF5FEA412390EA010F40F48000704774
:1075B0004FF0000304E000BF10F0004348BF40421A
:1075C0005FEA000C08BF704743F0964301464FF056
:1075D00000001CE050EA010208BF70474FF00003B2
:1075E0000AE000BF50EA010208BF704711F00043F3
:1075F00002D5404261EB41015FEA010C02BF8446C3
:107600000146002043F0B64308BFA3F18053A3F521
:107610000003BCFA8CF2083AA3EBC25310DB01FA68
:1076200002FC634400FA02FCC2F12002BCF1004FEC
:1076300020FA02F243EB020008BF20F0010070477D
:1076400002F1200201FA02FCC2F1200250EA4C00D1
:1076500021FA02F243EB020008BF20EADC70704717
:107660007BB972B90029BEBF00204FF0004106E08F
:1076700008BF00281CBF6FF000414FF0FF3000F042
:107680001DBBADF1080C6DE904CE002909DB002B10
:107690001ADB00F081F8DDF804E0DDE9022304B034
:1076A0007047404261EB4101002B1BDB00F074F896
:1076B000DDF804E0DDE9022304B0404261EB410162
:1076C000524263EB43037047524263EB430300F0C3
:1076D00063F8DDF804E0DDE9022304B0404261EB29
:1076E00041017047524263EB430300F055F8DDF867
:1076F00004E0DDE9022304B0524263EB4303704728
:1077000053B94AB9002908BF00281CBF4FF0FF3108
:107710004FF0FF3000F0D2BAADF1080C6DE904CEA5
:1077200000F03AF8DDF804E0DDE9022304B0704728
:1077300007EE900AF5EEC07AF1EE10FA01D400F0EF
:107740000BB8F1EE677A08B517EE900A00F004F86E
:10775000404261EB410108BDD0B5FFF7CBFD0C4BBA
:10776000002206460F4600F07FF900F0A9FA044611
:10777000FFF79EFD074B002200F076F902460B460C
:1077800030463946FFF756FC00F09AFA2146D0BD44
:107790000000F03D0000F0412DE9F047089D04464F
:1077A0008E46002B4DD18A42944669D9B2FA82F2B4
:1077B00052B101FA02F3C2F1200120FA01F10CFAF0
:1077C00002FC41EA030E94404FEA1C48210CBEFB28
:1077D000F8F61FFA8CF708FB16E341EA034306FBB1
:1077E00007F199420AD91CEB030306F1FF3080F040
:1077F0001F81994240F21C81023E63445B1AA4B28D
:10780000B3FBF8F008FB103344EA034400FB07F72E
:10781000A7420AD91CEB040400F1FF3380F00A816F
:10782000A74240F207816444023840EA0640E41B64
:1078300000261DB1D4400023C5E900433146BDE810
:10784000F0878B4209D9002D00F0EF800026C5E9B2
:10785000000130463146BDE8F087B3FA83F6002ECA
:107860004AD18B4202D3824200F2F980841A61EB42
:10787000030301209E46002DE0D0C5E9004EDDE760
:1078800002B9FFDEB2FA82F2002A40F09280A1EB48
:107890000C014FEA1C471FFA8CFE0126200CB1FB9D
:1078A000F7F307FB131140EA01410EFB03F0884296
:1078B00008D91CEB010103F1FF3802D2884200F223
:1078C000CB804346091AA4B2B1FBF7F007FB1011B5
:1078D00044EA01440EFB00FEA64508D91CEB040453
:1078E00000F1FF3102D2A64500F2BB800846A4EBAE
:1078F0000E0440EA03409CE7C6F12007B34022FA99
:1079000007FC4CEA030C20FA07F401FA06F31C43C7
:10791000F9404FEA1C4900FA06F3B1FBF9F8200CD4
:107920001FFA8CFE09FB181140EA014108FB0EF01A
:10793000884202FA06F20BD91CEB010108F1FF3A6A
:1079400080F08880884240F28580A8F10208614476
:10795000091AA4B2B1FBF9F009FB101144EA014184
:1079600000FB0EFE8E4508D91CEB010100F1FF342F
:107970006CD28E456AD90238614440EA0840A0FBC7
:107980000294A1EB0E01A142C846A64656D353D09D
:107990005DB1B3EB080261EB0E0101FA07F722FAC1
:1079A00006F3F1401F43C5E9007100263146BDE8EA
:1079B000F087C2F12003D8400CFA02FC21FA03F34D
:1079C000914001434FEA1C471FFA8CFEB3FBF7F0CE
:1079D00007FB10360B0C43EA064300FB0EF69E42F3
:1079E00004FA02F408D91CEB030300F1FF382FD28C
:1079F0009E422DD9023863449B1B89B2B3FBF7F634
:107A000007FB163341EA034106FB0EF38B4208D90C
:107A10001CEB010106F1FF3816D28B4214D9023E4D
:107A20006144C91A46EA004638E72E46284605E76B
:107A30000646E3E61846F8E64B45A9D2B9EB02083C
:107A400064EB0C0E0138A3E74646EAE7204694E7CC
:107A50004046D1E7D0467BE7023B614432E73046FF
:107A600009E76444023842E770B54FF0FF0C4CF46C
:107A7000E06C1CEA11541DBF1CEA135594EA0C0F6C
:107A800095EA0C0F00F0DEF82C4481EA030621EAA7
:107A90004C5123EA4C5350EA013518BF52EA0335E2
:107AA00041F4801143F4801338D0A0FB02CE4FF094
:107AB0000005E1FB02E506F00042E0FB03E54FF0C4
:107AC0000006E1FB03569CF0000F18BF4EF0010EBC
:107AD000A4F1FF04B6F5007F64F5407404D25FEAB8
:107AE0004E0E6D4146EB060642EAC62141EA55516B
:107AF0004FEAC52040EA5E504FEACE2EB4F1FD0CAD
:107B000088BFBCF5E06F1ED8BEF1004F08BF5FEA2A
:107B1000500E50F1000041EB045170BD06F00046DC
:107B200046EA010140EA020081EA0301B4EB5C0489
:107B3000C2BFD4EB0C0541EA045170BD41F4801181
:107B40004FF0000E013C00F3AB8014F1360FDEBFA6
:107B5000002001F0004170BDC4F10004203C35DA82
:107B60000C341BDC04F11404C4F1200500FA05F305
:107B700020FA04F001FA05F240EA020001F00042A6
:107B800021F0004110EBD37021FA04F642EB06011C
:107B90005EEA430E08BF20EAD37070BDC4F10C0446
:107BA000C4F1200500FA04F320FA05F001FA04F20A
:107BB00040EA020001F0004110EBD37041F10001F6
:107BC0005EEA430E08BF20EAD37070BDC4F1200501
:107BD00000FA05F24EEA020E20FA04F301FA05F269
:107BE00043EA020321FA04F001F0004121FA04F211
:107BF00020EA020000EBD3705EEA430E08BF20EAE1
:107C0000D37070BD94F0000F0FD101F0004640001A
:107C100041EB010111F4801F08BF013CF7D041EA9C
:107C2000060195F0000F18BF704703F000465200A0
:107C300043EB030313F4801F08BF013DF7D043EA71
:107C40000603704794EA0C0F0CEA135518BF95EA27
:107C50000C0F0CD050EA410618BF52EA4306D1D1AE
:107C600081EA030101F000414FF0000070BD50EACD
:107C7000410606BF1046194652EA430619D094EA57
:107C80000C0F02D150EA013613D195EA0C0F05D141
:107C900052EA03361CBF104619460AD181EA030195
:107CA00001F0004141F0FE4141F470014FF000004D
:107CB00070BD41F0FE4141F4780170BD704700BFD6
:107CC0004A0011D212F5001211D20DD56FF478735B
:107CD000B3EB62520ED44FEAC12343F0004343EAB0
:107CE000505323FA02F070474FF00000704750EAFB
:107CF000013002D14FF0FF3070474FF00000704765
:107D00009FED177BF8B5184C84ED007B19B3002369
:107D1000164E101F9C461D4602E0013399420DD0BD
:107D200050F8042F9707F8D11768B742F5D19DB9DD
:107D30000133994294464FF00105F1D15DB19CEDBC
:107D4000017ADFED0B7A67EE277A17EE900AFFF7DC
:107D5000EFFCC4E90001F8BD064839F0EDFF00BFB3
:107D60000000000000000000480B012084C509004D
:107D700000007A44AC7009002DE9F8439DF834C046
:107D800080F84AC00446CCF1080C80F84EC00020B0
:107D900084F854006060BDF92800A4F85600BDF9CD
:107DA0002C00A4F858009DF8380084F84F009DF886
:107DB0003C0084F851009FED307B9DF8400084F832
:107DC0004B009DF8440084F852009DF84800BDF82F
:107DD0002050BDF82470BDF8306084F8530084ED65
:107DE000027B91469846A9B18B0740D10868244B85
:107DF000984226D0234B98422ED0234B984236D11E
:107E000022482061224860612248A0612248E06146
:107E100022482062216022498C420DD0A4F8409073
:107E2000A4F84280A4F84650A4F848703146204691
:107E3000BDE8F84322F01EB94146484657F08AF99A
:107E4000ECE718482061184860611848A06118489C
:107E5000E06118482062DDE717482061174860613B
:107E60001748A0611748E06117482062D2E7174819
:107E700039F062FFAFF30080000000000000000056
:107E800090FC09008CE6090064E8090091D3030026
:107E9000CDD20300C5D20300C1D3030089D30300B0
:107EA000880A01207DF4030081F2030071F20300CF
:107EB000ADF4030075F40300C9CE0300B5CD030093
:107EC00081CD030005CF0300B1CE0300AC760900DD
:107ED00030B5144685B019A3D3E90023FFF710FC91
:107EE0000546A0F16150A0F5351001A9A0F560701C
:107EF00058F0C0FB9DF807309DF806109DF808204B
:107F00001B0443EA41539DF8091043EAC2239DF83C
:107F10000A2043EA411343EA5203BDF8042006490C
:107F2000A2F2BC7225F0010543EA4263A5FB010100
:107F3000236005B030BD00BF00CA9A3B00CA9A3B1F
:107F400000000000D2B32DE9F0436FF00E0885B0B9
:107F50000646174601F10F04A8EB010800F1EF09EE
:107F600000F1F00554F80F0C54F80B1C54F8072CD2
:107F700054F8033CEC46ACE80F003146A4F10F0086
:107F800000F0F2FCA4F110034A4613F801CF12F8F6
:107F9000011FA3428CEA010C83F800C0F5D1EC4626
:107FA000BCE80F00103408EB040C674528606960DA
:107FB000AA60EB60D6D805B0BDE8F083704700BF7B
:107FC0002DE9F843074600F1F00682B36FF00E0585
:107FD000144601F10F086D1AB146CE46A8F1100300
:107FE000A8F10F090EF1FF3E13F801CF1EF8012F83
:107FF00043458CEA020C83F800C0F5D13946484667
:1080000008F1100800F026F905EB08039C42E4D8BB
:10801000D9F80000D9F80410D9F80820D9F80C30A4
:10802000C7F8F0007160B260F360BDE8F883B14654
:10803000EEE700BFDAB32DE9F0414C1E84B00646EE
:10804000A518102100F1F0074FF0000810290FD0FB
:108050000A46013104AB1A4414F8013F12F8102CFF
:10806000AC4283EA02032370F0D104B0BDE8F08192
:1080700038687968BA68FB68EC46ACE80F003146AE
:10808000684600F0E7F806F580710F2211F8013D0F
:10809000FF2B06D03244013382F8F0300121002258
:1080A000D8E7013A531C81F80080EFD1F6E770471A
:1080B00003460846194600F057BC00BF0346084671
:1080C000194600F0C7B800BF182A2DE9F04FC0F8D4
:1080D00000215ED0202A00F08880102A7FD0002363
:1080E0001D46A0F804311A461946434EDFF80CB17C
:1080F00005EB81032FE016F804A01BF8099016F891
:108100000E4016F80CE016F808C08AEA09088A1A28
:1081100005EB820915F8222088EA020883F800801E
:1081200099F801200433544003F8034C99F80220D5
:108130008EEA020E03F802EC99F803208CEA020C96
:1081400003F801CC90F8042101310132B1EB820F28
:1081500043D290F80521B1FBF2F902FB191A13F88A
:10816000048C13F8034C13F802EC13F801CCBAF1A9
:10817000000FC0D0D0F80071202FC8D1BAF1040F81
:10818000C5D116F80880345D16F80EE016F80CC05C
:10819000BDE740F20C63A0F8043105460B46844667
:1081A00000241A788CF800205A788CF801209A78EC
:1081B0008CF80220DA788CF8032090F8052101343D
:1081C0009442114603F104030CF1040CE9D390F836
:1081D00004310133B2EB830F87D3BDE8F08F40F257
:1081E0000A43A0F804310546D8E740F60E03A0F88C
:1081F00004310546D2E700BF54140A0048130A00B0
:1082000038B51D460446FFF75FFF29686A68AB680A
:10821000E868C4F8FC00C4F8F010C4F8F420C4F80E
:10822000F83038BD30B500010C1D01F11405231FD5
:1082300002EB000C19781CF801EB81EA0E0103F83F
:10824000011BA342F6D11C1DAC4200F10400EED18B
:1082500030BD00BF2DE9F04FD1F8003187B0A3F158
:108260001002102A0491824600F2C7800123934035
:1082700003F0013323F08073002B14BF0B4600235F
:1082800007EE903A17EE902A51460020FFF7CAFFFA
:10829000012302930AF104030593DFF868B10AF1A0
:1082A00010030193D0460598C6464246002312F8B3
:1082B00023101BF8011002F823100133042BF6D110
:1082C00001329042F2D198F80D2098F8011098F8F8
:1082D000023098F8090088F8092098F8062098F8E4
:1082E0000AA088F80D1088F80A3098F80E1098F84F
:1082F000033088F80E2098F80B2098F8054098F87D
:108300000F9088F80F2098F8072088F80730049B12
:1083100088F80B2088F8014088F8050088F802A04A
:1083200088F8061088F8039093F80431029A934273
:108330005AD0CDF80C809EF800508AEA090785EAE9
:10834000040C84EA0A0885EA09038CEA070600930C
:108350004FEADC104FEAD811FA09DB09744086EACB
:108360000A0A86EA0909754000EB4000009E01EB0D
:10837000410102EB420203EB430300EBC00001EBBF
:10838000C10102EBC20203EBC30383EA460380EAA6
:108390004C0081EA480182EA470283EA0909684001
:1083A000019B8EF800004C4082EA0A0A8EF80140D8
:1083B0008EF802A08EF803900EF1040E734506D0DD
:1083C0009EF801409EF802A09EF80390B3E7DDE915
:1083D000024817EE902A20464146FFF723FF204629
:1083E0000130C3B202935EE717EE902A029841462D
:1083F00007B0BDE8F04FFFF715BF002307EE903A36
:1084000040E700BF54140A00FEE700BF2DE9F04F1B
:108410004FEAA30803F00304644B03EB84194346BB
:108420001C2B86466248A8BF1C2350F824A0D9F80C
:108430000400033389B023EAE37318410590D9F8A7
:10844000080018410690D9F80C00B8F11F0FC34678
:1084500040FA03F3A8BF4FF01F0B079300205B46C1
:108460000490C346C846D1469A460EE008AC04EBD9
:10847000850555F8104C002B40EA0400B8BF644253
:10848000013A41F8044B00F08E805EF8043B23F083
:10849000004424F0030423F00045002CE6D023F030
:1084A000004424F00F0454B958F82540BBF1000FE4
:1084B000BABFCAF10005AC4044FA0AF4DBE723F086
:1084C000004424F03F0474B93A4C103D54F8255050
:1084D0004C4685FB04642546AAF10304002C57DBB7
:1084E00045FA04F4C7E76C04B4F1006FB6BF6C053D
:1084F00000250425B4F1005F009503DA009D0235E4
:10850000A4000095B4F1804F03DA009D01356400AA
:108510000095294D294E2A4FAC422A4DC8BFAC4682
:10852000294DD8BFB446294ED8BF2E46284DD8BFB6
:108530002F46284D0297284FD8BF2F46274D019729
:10854000274FD8BF2F460397254686FB0575654400
:10855000264685FB06C6039F25463E4486FB05C589
:10856000019F3D4485FB0464029F1E4D3C44009FD7
:1085700055F8275084FB0565ED004C4685FB0464E7
:108580002546194C54F82740AAEB0404002CA7DA1E
:1085900066426FF0004444FA06F7AF42FFF66BAF55
:1085A00005FA06F467E709B0BDE8F08FC4300A00A9
:1085B000B42F0A0004300A009979825A28482EB054
:1085C000B477F5FEA4F633D3A9BDA02963218510A5
:1085D000591858FF8D496C23F0CEC2271BAA575952
:1085E0008B40E946E42F0A00C42F0A002DE9F04F22
:1085F0009BBB12F0010C2DD0D0F88012D0F8802354
:10860000D0F8804149425242C0F88012C0F880231D
:10861000D0F88014D0F880259C46D0F880364942A6
:1086200052425B42C0F88014C0F88025D0F8801018
:10863000D0F88027C0F88036D0F8803864425242A3
:1086400049425B42C0F88041C0F88010C0F88027E2
:10865000C0F880386046BDE8F08F4FF00046DE403D
:1086600012F0010C06F1FF36C3F11F0547D04FF0A1
:10867000000C00F1800400F51068674654F8802C67
:1086800042FA05F94FEAE27AB9EBE27F18BF86EACF
:108690000A029A40BE4644F8802C82EAE27EAEEBA3
:1086A000E27ED0F88020524242FA05FA4FEAE27B9D
:1086B000BAEBE27F18BF86EA0B029A40B946C0F8CF
:1086C000802082EAE279A9EBE2790A684EEA090E93
:1086D0004CEA0E0C42FA05FEBEEBE27F4FEAE2796D
:1086E00018BF86EA090200F580709A40804541F87B
:1086F000042B04F58074C1D16046BDE8F08F00F111
:10870000800400F5106E674654F8802C42FA05F993
:108710004FEAE27AB9EBE27F18BF86EA0A029A4092
:10872000B84644F8802C82EAE278A8EBE278D0F8E8
:10873000802042FA05FA4FEAE27BBAEBE27F18BFEB
:1087400086EA0B029A40B946C0F8802082EAE279B4
:10875000A9EBE2790A6848EA09084CEA080C42FAEF
:1087600005F8B8EBE27F4FEAE27918BF86EA090222
:1087700000F580709A40864541F8042B04F580741A
:10878000C2D16046BDE8F08F2DE9F04F00221646B9
:1087900089B06C4B6C4C6D48CDE902223546012204
:1087A000196841B1D4F80413114204D01D6019684E
:1087B000009100991643043383424FEA4202EFD1FD
:1087C000614BD3F87C21002A6BD00022C3F87C21B6
:1087D000D3F87C3101934FF0A042019BD2F81025D1
:1087E0005B4B0292D3F810250392F3B2002B7AD19F
:1087F00000224FF0FF33574EDFF85491CDE90422A9
:10880000CDE90633A6F15A08534C002514F9010BA3
:10881000471C30D0C0F3C20E08AB03EB0E0C00F0C7
:1088200007021CF8083CD340D907C7B200F03F004C
:1088300021D508EB0003B90993F9283058F8233003
:10884000002B5CD003295CD01F2887BF07F01F07CF
:10885000CE4607464FF0A04E1CF818CC0EEB87070B
:108860002CFA02F2D7F800C7D207CCF3014C3DD462
:10887000BCF1030F54D0A642C8D18DB34FF0A04332
:108880000299D3F81035D9F81025994202D10399ED
:10889000914225D0DDE904010293069003920791ED
:1088A000B2E7F3B2D3B12D4F01250024A30003F1A9
:1088B00080432E4203F5C0434FEA45050BD0D3F861
:1088C000100557F82420D3F81015C0F30520C1F384
:1088D000014102B190470134082CE7D1002E87DB1B
:1088E00009B0BDE8F08F46F00046DCE7BCF1020FAE
:1088F000C1D1032923D0002BBDD09847BBE7032962
:10890000B9D10DF1100A4FF0010B1AF80EA00BFAB5
:1089100002FB4AEA0B0A0DF1100B0BF80EA093E7CD
:108920000329E8D14FF4003CD7F8002722F4403265
:10893000013542EA0C02EDB2C7F80027DBE74FF43D
:10894000403CF1E7006100400060004020610040D1
:10895000000300509A5301209853012040530120F6
:1089600008B502204EF0FCFE2DE9F04FD1F80031A1
:10897000A3F11002102A85B00C46804600F2368121
:108980000123934003F0013323F08073002B14BFC5
:108990000B46002307EE903A17EE902A94F8040154
:1089A000DFF850B24146FFF73DFC94F80431013B3B
:1089B000DBB2019308F10403039308F11003009361
:1089C000C2469AF801009AF80D109AF809509AF8E0
:1089D00005309AF802208AF805009AF807009AF8FC
:1089E0000A609AF806408AF80D508AF809309AF819
:1089F0000E509AF803308AF801108AF80A209AF883
:108A00000B109AF80F208AF8030003988AF80B20BD
:108A10008AF802608AF806508AF80E408AF8071031
:108A20008AF80F3057465246002312F823101BF8DD
:108A3000011002F823100133042BF6D101329042C9
:108A4000F2D1019C17EE902A51462046FFF7EAFB2F
:108A5000002C00F0C880CDF808A03A7897F8029072
:108A6000797897F803E0D3094FEAD91603EB43036B
:108A70004FEAD11C03EBC30306EB460683EA42032D
:108A80004FEADE100CEB4C0C06EBC6065FFA83FADD
:108A900086EA4906C3F3C0130CEBCC0C00EB400094
:108AA00082EA01088CEA410CC6F3C01482EA09028A
:108AB00003EB430300EBC00080EA4E00CCF3C0158B
:108AC00081EA09015FFA8CFC8EEA020203EBC30320
:108AD00004EB4404F6B283EA4A038EEA01018CEA0D
:108AE000020288EA0E0E04EBC40488EA0908C0F307
:108AF000C01984EA460486EA0E0E724005EB45056D
:108B0000C3F3C01609EB4909C0B205EBC5058AEAF3
:108B100001018AEA080809EBC90906EB460685EA5D
:108B20004C0589EA400980EA0E0E8CEA010180EAD0
:108B3000080806EBC606D8B286EA4006414080EA3D
:108B40000E00C5F3C01E0EEB4E0EF3B2EDB20EEBEF
:108B5000CE0EC4F3C0166A4085EA080806EB460646
:108B60008EEA45055FFA89FEC9F3C019E4B28EEAC0
:108B7000020206EBC60609EB4909EDB2614060400E
:108B80008EEA08085A4086EA440409EBC909E4B2AF
:108B900083EA010C83EA080883EA000189EA4E0EA1
:108BA00085EA020385EA0C0C5FFA8EF269406340A5
:108BB00085EA0805534084EA0C0C61406C407B70E8
:108BC00082EA0C0C5140009B87F800C06240B970EB
:108BD000FA700437BB427FF440AFDDE9013A581E1A
:108BE000C3B20193EDE605B0BDE8F08F002307EEB8
:108BF000903AD1E654130A0010B4D0F8C437D0F834
:108C0000C847D0F8BC2704FB03F302FB03F3002B97
:108C100011DD00220239944621F802CFD0F8C8476E
:108C2000D0F8C43704FB03F3D0F8BC47013204FB8F
:108C300003F39A42F0DB5DF8044B70472DE9F04FE7
:108C400089B00593002800F058810D460968174641
:108C5000814661F08DFE061EC0F24C8129683144C8
:108C60002960484662F016FBB0F10008C0F273813B
:108C70002B6843442B603B6806EB08041B1B3B60DE
:108C8000D9F8B827002A7CD0D9F8B02742B1D9F852
:108C9000B44748465EF0FCFD2044C9F8CC073B6869
:108CA000129A002A00F0B980D9F8D827C9F8CC3731
:108CB000002A40F02C81002B40F32981C9F8DC37D1
:108CC000D5F8008043442B60D9F8CC273B689B1A29
:108CD0003B60D9F8C427D9F8DC4700239A420793B0
:108CE0004FEAC40440F304819B4609F5FC630493F6
:108CF000D9F8BC37002B40F3B780049BCDF80CB0FB
:108D00004FF0000A5746079EC3469A4618E0A4450E
:108D10002EDC03980197009048465EF0C5FD0028C0
:108D200007F10107C5EBC0058344C0F2C080079E70
:108D3000D9F8BC373544BB42A8EB050440F3918019
:108D4000039800905946234607AA0197484661F0C8
:108D5000F3FE079D5AF804CBC6EBC008A844834431
:108D60000028ACEB080307AA5946A4EB0808CEDAA2
:108D700048460599FFF740FF6FF0070009B0BDE8CE
:108D8000F08FD9F8B037002B81D10123C9F8B03763
:108D90002B68D7F800A003931C1B9B4601E0AAEBAD
:108DA000020A5146584600F0F7F800280BEB000382
:108DB00000F10302C0F2E4801BF800002178884231
:108DC00003F1030BEBD1587861788842E7D194F82E
:108DD00002C099788CEA010111F0FC0FDFD11CF080
:108DE000020F039A18BF03F1FF339C1A002CC9F835
:108DF000B447C0F2C980D9F8C037D9F8C8173219BA
:108E0000424403FB02F2D9F8C437D20001FB03F35A
:108E100092FBF3F2C9F8B8273BE7D9F8CC079842A0
:108E200000F3A780D9F8DC17D9F8D827914275DB71
:108E3000891A09F11C08414440462CF0B5FFD9F8C5
:108E4000D807D9F8CC27296840442CF07DFFD9F801
:108E5000CC17D9F8D8270A44C9F8DC272B680B446B
:108E600031E7D846DDF80CB0594648465FF0F8F9CE
:108E7000002845DBD9F8BC37002BC8BF002504DC2F
:108E80001EE0D9F8BC37AB421ADD2A46594648469F
:108E90005FF0FEFE002805F10105F2DA484605996B
:108EA000FFF7AAFE6FF00A0009B0BDE8F08F484650
:108EB0000599FFF7A1FE6FF0080009B0BDE8F08F3B
:108EC000D9F8C82702FB0BF202FB03F3059A4846C8
:108ED00002EB430161F0BEFC002843DB049B083336
:108EE0000493D9F8C4370BF1010B5B453FF700AF92
:108EF000002043E76FF0050040E76FF004003DE716
:108F000048460599FFF778FE6FF0090036E74846B6
:108F10000599FFF771FE6FF005002FE7024609F192
:108F20001C00084429682CF00FFFD9F8CC27D9F889
:108F3000DC3705991344C9F8DC372B6813442B60E0
:108F40003B68D9F8CC279B1A48463B60FFF754FE94
:108F50006FF0010012E748460599FFF74DFE6FF0EC
:108F600006000BE748460599FFF746FE6FF00B0039
:108F700004E748460599FFF73FFE4FF0FF30FDE656
:108F80004FF0FF33C9F8B43748460599FFF734FE70
:108F90006FF00200F2E600BF012913DD821E02EB32
:108FA000010C431EC0F1010101E063450AD0C8185D
:108FB00013F8012FFF2AF8D15A7802F0E002E02AD4
:108FC000F3D170474FF0FF30704700BF08B15FF03A
:108FD000CDBD704718B1D0F8D037032B08D000238F
:108FE000C1E90033C1E90233C1E904338B61704741
:108FF000D0F8B8370B60D0F8BC374B60D0F8C0273A
:109000001023C1E9022390F8D437D0F8D02703EB1E
:109010004303013A10B41344084CD0F8BC2734F988
:1090200013305DF8044B02FB03F30B61D0F8D0372B
:109030004B6190F8D4378B61704700BF80560A00AF
:10904000A0B138B50D461146044661F091FC0130DF
:1090500009D0D4F8D037032B05D120462946FFF795
:10906000B9FF002038BD6FF0050038BD6FF0040077
:10907000704700BF5EF0B2BB10B54FF0804386B0C2
:10908000D3F80443620703D5D3F80821002A62D13C
:10909000A30605D54FF08043D3F81421002A4FD101
:1090A000600605D54FF08043D3F81821002A3BD144
:1090B000210604D54FF08043D3F81C214ABBE205BA
:1090C00004D54FF08043D3F82021B2B9A30512D5BF
:1090D0004FF08043D3F824216AB10022C3F8242141
:1090E000D3F82421214B0592059A1B68022006B073
:1090F000BDE81040184706B010BD0022C3F820217B
:109100001A4AD3F82031049301201368049A98472F
:10911000DCE70020C3F81C01144AD3F81C31039388
:109120001368039A9847CAE70022C3F81821104A27
:10913000D3F81831029301201368029A9847B7E7D1
:109140000020C3F814010A4AD3F8143101931368BC
:10915000019A9847A4E70022C3F80821054AD3F8EA
:10916000083100931368009A984791E7E053012073
:10917000DC530120D8530120064BD3F800213AB12B
:10918000054A00205071C3F8000113689168184720
:10919000704700BF00900240B853012002480322EC
:1091A000002129F013BE00BF00B000400248042295
:1091B000012129F00BBE00BF00100140024804222B
:1091C000022129F003BE00BF004002400E480F4AB2
:1091D000904208B507D2013A121A22F003020C4954
:1091E00004322CF0B1FD0B480B4A904207D2013AF1
:1091F000121A22F00302043200212CF055FE00F076
:10920000A7F852F06BF900BF00000120B80601205A
:10921000B8640A00B8060120FC5D0120014902483B
:1092200059F01CBE905201200030004002494FF01E
:10923000402059F013BE00BFC4520120084BD3F8A0
:10924000182102B97047002282B0C3F81821D3F860
:1092500018310193019B034802B026F00DB900BFFD
:109260000030024030520120084BD3F8182102B9D7
:109270007047002282B0C3F81821D3F81831019347
:10928000019B034802B026F0F7B800BF00F002408F
:1092900054520120F0B52A4C83B00226002501A8C3
:1092A0004FF096FA05280BD0019B032B3DD02CD80C
:1092B000022BF4D101A825704FF08AFA0528F3D1CA
:1092C000204D214F4FF40C760DF102012846ADF8E8
:1092D00002604FF009FAA0B9D7F80841002CF3D08A
:1092E00023462468D3E9011228469047002CF7D181
:1092F0000DF102012846ADF802604FF0F5F90028A3
:10930000EAD00C2817D003B0F0BDA3F10902022A5D
:10931000C5D80A2B0BD0092B0BD00B2B0CBF01206F
:109320004FF0FF3059F00EFCB9E72670B7E7002088
:10933000F8E70220F6E705484CF0EAFA03B0F0BD82
:10934000EE5D012000500120E453012060AB0900D4
:1093500010B54FF08053D3F83021082A1FD0874A28
:10936000D2F8883043F47003C2F88830BFF34F8FCF
:10937000BFF36F8F4FF01023D3F80C22D20700F108
:10938000DE80D3F80022002AC0F2B380D3F8043282
:10939000002BC0F2AE807A4B7A4A1A6010BD4FF0B3
:1093A00080410020C1F80C01774AC1F81001C1F8D2
:1093B0003805D3F80414C2F82015D3F80814C2F8FD
:1093C0002415D3F80C14C2F82815D3F81014C2F8D9
:1093D0002C15D3F81414C2F83015D3F81814C2F8A9
:1093E0003415D3F81C14C2F84015D3F82014C2F871
:1093F0004415D3F82414C2F84815D3F82814C2F839
:109400004C15D3F82C14C2F85015D3F83014C2F808
:109410005415D3F83414C2F86015D3F83814C2F8D0
:109420006415D3F83C14C2F86815D3F84014C2F898
:109430006C15D3F83411D3F84434C2F870350329CD
:1094400016D8524B5B5C1BB1514B524AC3F88C2669
:10945000514B5B5C63B14FF080535049D3F83021DE
:10946000FB20C1F81805082AD3F8343104D076E778
:109470004FF08053D3F83431032B20D94FF0805371
:10948000D3F83431032B0ED8454AD35C5BB14FF08F
:109490008053444AD3F830314FF40071082BC2F89E
:1094A00040167FF45CAF4FF08043D3F80024D1071F
:1094B0007FF555AF6FF00102C3F800244FE73A4A39
:1094C000D35C002BDAD04FF080524FF08040D2F8BE
:1094D0005832D0F8E41ED2F8304103F00F0321F0E7
:1094E0000F010B43C0F8E43E082CD2F83431C9D048
:1094F00035E72E4A0123C2F80435D2F80034002B98
:10950000FBD04FF010231221284AC3F80012D2F8E2
:109510000034002BFBD04FF010231221234AC3F854
:109520000412D2F80034002BFBD000231F49C2F8EC
:109530000435D1F80034002BFBD001F03FFA1B4A70
:109540000123C2F80435D2F80034002BFBD04FF0D1
:109550001021164AD1F80C3223F00103C1F80C3265
:10956000D2F80034002BFBD000231049C2F8043598
:10957000D1F80034002BFBD0DFE700BF00ED00E0A6
:10958000000001200090D00300C0004074AB09002F
:10959000005000404881030074AB090000F0004017
:1095A00074AB09000090024074AB090000E0014078
:1095B0000149024829F062BC785201200090004025
:1095C0000149024829F05ABC8452012000A0004001
:1095D0000149024859F01ABEF8520120002000400B
:1095E0000149024859F012BE1C530120008002407C
:1095F00000205BF03BB900BF10B5084CD4F8003137
:1096000082B04BB1064B5B6898470023C4F8003129
:10961000D4F800310193019B02B010BD000001405D
:10962000B0530120022A2DE9F043464B1ED002EB35
:10963000C20C03EB0C1C0CF1480601F1440E0CF1BA
:109640008C0C00F1240750F8043B5CF8044956F8F0
:10965000045B1A4685FB028241F8042B84FB03233A
:1096600087424EF80439EED1BDE8F0838268D3F822
:1096700038C18CFB02428469D3F8205185FB046415
:1096800022440A60D3F83C71426887FB0242C469F5
:10969000D3F8245185FB046422444A600268D3F85D
:1096A000406186FB0242056AD3F8284184FB05E548
:1096B0002A448A600268D3F84451964685FB0E2EF0
:1096C000026AD3F82C4184FB02827244CA60426869
:1096D000D3F848E191468EFB0949C469D3F830219B
:1096E00082FB048409EB04020A618268D3F84C818E
:1096F00088FB0242D3F83441836984FB03931A4404
:109700004A6143698CFB03238B61036987FB032355
:10971000CB61C36886FB03230B62C36885FB03230D
:109720004B6203698EFB03238B62426988FB023222
:109730000023C1E91033C1E90E33C1E90C33CA6219
:10974000BDE8F0833C5C0A00054B18680368D3F859
:10975000402112B10022C3F8402100F0C9BE00BF71
:10976000500B0120002800F02C822DE9F84304461C
:109770000069002800F0F68194F8627094F8613076
:10978000B74E07EB4701202B4FEA410134BF4FF0A2
:10979000A04CB4468846002900F0C081002215463E
:1097A0004FF0010E01E08A4213DA835C202B38BFB0
:1097B0004FF0A04903F01F0328BFB14601320EFA53
:1097C00003F3CC45D2B245EA0305ECD00120BDE855
:1097D000F88315F07F4305F47F0005F47F41EAB27A
:1097E00018BF082308B143F0040309B143F0020392
:1097F0000AB143F00103013B0B2B00F29081DFE83B
:1098000013F00C000C0096010C008E018E018E01ED
:109810000C008E018E018E019601012284F86020D9
:1098200094F86310B4F85E6001238B40073606F4A9
:10983000FF6684F86630DBB203FB06F694F8653009
:1098400003FB06F694F8683002FB06F6E66403B103
:10985000760008EB060016F045FA03466062002821
:1098600000F0808133446361324600212CF01CFB00
:1098700094F86000012800F07881022800F0A381AC
:1098800094F86160012706F01F0307FA03F31D43F4
:10989000A36194F86230E561002284F864209BB1F2
:1098A000D4E904309B5C03F01F0307FA03F340F88C
:1098B000223094F86230511CCAB203EB4303B2EB7E
:1098C000430FEDDB94F8616094F8653094F866100E
:1098D00001229A40013A4FF47A43B3FBF1F3B3FB10
:1098E000F2F3632B94F834205D4998BF64236365D9
:1098F000236594F844300020202A84F86A0003F09D
:109900001F052CBF08464FF0A04002F01F02202B7D
:109910004FF0010303FA02F203FA05F323642CBFAC
:109920000B464FF0A0431F2E226388BF06F01F0690
:1099300000F5A162A26298BF4FF0A04103F5A162B9
:1099400006F5E07603F20C53C4E90E2300F20C5046
:1099500040F20333E06241F8263094F861201F2A78
:1099600086BF02F01F023E494FF0A0410123934001
:10997000C1F80C3594F834301F2B86BF03F01F0359
:10998000374A4FF0A04203F5E07340F2033142F84A
:10999000231094F834201F2A86BF02F01F0230499A
:1099A0004FF0A04101239340C1F80C3594F84430A6
:1099B0001F2B86BF03F01F03294A4FF0A04203F577
:1099C000E07340F2033142F8231094F844301F2B27
:1099D00086BF234A03F01F034FF0A042012606FA78
:1099E00003F3C2F8083594F862303BB31C4D0023F2
:1099F00040F203372269D25C1F2A88BF02F01F029F
:109A0000284602F5E07298BF4FF0A0404FF0A04109
:109A100040F822702269D25C1F2A84BF02F01F0224
:109A2000294606FA02F2C1F80C2594F862200133A7
:109A3000DBB202EB4202B3EB420FDBDB94F86320B4
:109A4000012101FA02F3023BDBB284F86D30002AF7
:109A500075D00020024D03460E4640F2033714E055
:109A6000000300501F2B86BF03F01F032A464FF050
:109A7000A04206FA03F3C2F8083594F863200130D7
:109A8000C3B249009A42C9B259D9D4F848C01A01A0
:109A90000CEB03131B7B202B34BF4FF0A0432B4652
:109AA00003F5A1634CF80230A36C134493F80CC087
:109AB000BCF1200F34BF4FF0A04CAC460CF20C5C54
:109AC000C3F804C0A36C03EB020C9CF80C3003F049
:109AD0001F0306FA03F3CCF80830A36C13441B7B76
:109AE0001F2B86BF03F01F03AC464FF0A04C03F5BD
:109AF000E0734CF8237094F86D300B42A36C134460
:109B00001B7BAFD11F2B86BF03F01F032A464FF0EC
:109B1000A04206FA03F3C2F80C35AEE70D46042264
:109B200007EB470784F860204FEAC70878E602226F
:109B300007EB470784F8602007FA02F870E694F80C
:109B40006120384B202A38BF4FF0A04303F5A162B3
:109B500003F20C532046C4E9012300F055FC002019
:109B6000BDE8F8830220BDE8F883236994F86160BA
:109B7000197894F8627006F01F0200FA02F2C1F33D
:109B8000C1011543C4E9062584F86410002F3FF491
:109B90009BAE002202E0236994F864109B5C656927
:109BA00003F01F03C90000FA03F3CB40AB5494F851
:109BB00062300132D2B203EB4303B2EB430FEADB74
:109BC00080E60320704794F86160236906F01F0265
:109BD000012000FA02F219781543C4E9062594F829
:109BE0006220C1F3001184F86410002A3FF46CAEC7
:109BF000002202E0236994F864109B5C656903F01D
:109C00001F03090100FA03F3CB4025F8123094F842
:109C100062300132D2B203EB4303B2EB430FE9DB14
:109C200050E600BF0003005090F86030012B05D0D3
:109C3000022B01D000F0F4B800F02ABA00F000B80E
:109C40002DE9F04F034691B0D0F8149001921A46D6
:109C500093F8683003900491406A33B192F86A3007
:109C6000D26CC3F1010302FB0300039BB3F85E2037
:109C700093F86510D31DDB10C2EBC30250FA82F2D9
:109C8000DB00062906920B9300F0C280C1F10503A8
:109C9000DBB24FF400629A400D9240229A400E923D
:109CA000012202FA03F30F93039B93F86630002B13
:109CB00000F09880019A013A12B20A9200220C92A6
:109CC000002900F088809DF8302001980992DDE994
:109CD0000E6800FB02F2520005920D9D00220792D1
:109CE0000892B646039A92F96720002AB8BF5242FA
:109CF000013A52B2541C59D0069C0199049801FBB8
:109D000002F603FB06F600EB8606D0B20290D007FF
:109D100004D5039A92F96720002A66DB059A164457
:109D2000019A03FB02F706EB47074FF0010C0022F4
:109D3000019999B31FFA8CFC04EB010A36F8121052
:109D400037F8120011EA050318BF99F8003011EA3C
:109D50000E0F1CBF99F801B043EA0B0311EA080F7C
:109D60001CBF99F802100B4328421CBF99F803103E
:109D70000B4310EA0E0F1CBF99F804100B4310EAB6
:109D8000080F1CBF99F805100B4304F8013B62440F
:109D9000544512B2D2D1039B93F86630029A013A2D
:109DA00052B2511CA9D1039A92F86510089A4FEA51
:109DB0004E0E4ABB052927D94FF001084FF4006524
:109DC000079A06980B9C01320792D2B220448A422D
:109DD0000690089286D30C9A01320C92D2B29A4223
:109DE000FFF46EAF11B0BDE8F08F099A5F1EBF1A85
:109DF00001FB07F706EB470703FB01F60A9A07EB9F
:109E000046064FF0FF3C93E76D004FEA4808D7E75E
:109E100020231025CDE90E354FF400430D9343E781
:109E20002DE9F04F914693B090F868204469436A59
:109E300001900391002A40F01281C26C0199B1F89F
:109E40005E0091F86510C51DED10C0EBC500062938
:109E50004FEAC505C6B200F01281C1F10501C9B2D1
:109E60004FF4006088400F904020884010900120FF
:109E700000FA01F11191184600212CF015F800EBC1
:109E800086030198079390F86230002B00F0DF8082
:109E9000AA000C9209F1FF3292B2511C12B204F1E5
:109EA000180B89000B9290F86670059100220D92B4
:109EB000DA46CDF80090002F00F0C080019B93F8A7
:109EC000651000230E93002900F0AE809DF8383015
:109ED000009A0A9302FB03F3DDE9109C5B000693F2
:109EE0000023DDF83C80089309939DF834300493F7
:109EF0004B46C146E0469C46019B93F9672082EAA7
:109F0000E273A3EBE273013B5BB25D1C76D0079971
:109F10000498039C82EAE27EAEEBE27E5FFA8EFE5C
:109F200000FB0E3E009800FB0EFE07FB0EFE04EB4E
:109F30008E0EDCB20294DC0701D5002A4ADB069BB8
:109F40009E44009B07FB03FB0EEB4B0B01240022FE
:109F5000009B002B35D0059BA4B2CD183EF81270A3
:109F60003BF8126017EA090318BF5AF8183C17EAC1
:109F70000C0F1CBF5AF8140C034317EA080F1CBF40
:109F80005AF8100C034316EA090F1CBF5AF80C0CC0
:109F9000034316EA0C0F1CBF5AF8080C034316EAD9
:109FA000080F1CBF5AF8040C034351F8040B224459
:109FB0000343A94212B241F8043CCFD1019B93F86C
:109FC0006670029B013B5BB25A1C14D0019A92F955
:109FD00067209DE70A9B0B9A07F1FF3BABEB030B56
:109FE00000FB0BFB0EEB4B0B07FB00FE0BEB4E0ECF
:109FF0004FF0FF34ACE7019B93F86510099B4FEAE3
:10A000004C0C3BBB052925D94FF001084FF40069E2
:10A01000089B079A0C9801330893DBB202448B42E9
:10A0200007920993FFF468AF0E9B01330E93DBB2E6
:10A03000BB42FFF448AF019B93F862300D9A0132A6
:10A040000D92D2B293420AF1180A3FF634AF13B020
:10A05000BDE8F08F4FEA49094FEA4808D8E7019A6E
:10A0600092F86A10C1F101001146D26C91F86010AB
:10A07000B2FBF1F100FB01F103EB8103DEE62021ED
:10A080001027CDE910174FF400410F91F3E600BF00
:10A090002DE9F04F95B04569019290F86820436A28
:10A0A00002900591002A40F00B81C26C0299B1F830
:10A0B0005E0091F86510C41DE410C0EBC4000629D1
:10A0C0004FEAC404C6B200F00B81C1F10501C9B268
:10A0D0004FF400608840109040208840119001208B
:10A0E00000FA01F11291002118462BF0DDFE0299D1
:10A0F00000EB4603089391F86230002B00F0D98002
:10A1000062000E92019A91F86610013A92B213928F
:10A11000013252000692002205F10C090D9200292D
:10A1200000F0BE80029B93F8650000230F93BDF9F9
:10A130004C300C93002800F0A9809DF83C30019A27
:10A140000B9302FB03F35B00DDE911EB0793109D1A
:10A15000002309930A93029B93F9672082EAE27332
:10A16000A3EBE273013B5BB25C1C79D09DF8340039
:10A1700004900898049C059F82EAE276A6EBE276BA
:10A18000F6B204FB0636019C04FB06F601FB06F65C
:10A1900007EB8606DFB20397DF0701D5002A4DDB08
:10A1A000079B1E44019B01FB03F706EB47074FF09B
:10A1B000010C0022019B002B37D0069B1FFA8CFC60
:10A1C00000EB030836F8121037F8124011EA0503C5
:10A1D00018BF39F80C3C11EA0E0F1CBF39F80AAC55
:10A1E00043EA0A0311EA0B0F1CBF39F8081C0B43A2
:10A1F0002C421CBF39F8061C0B4314EA0E0F1CBF7F
:10A2000039F8041C0B4314EA0B0F1CBF39F8021C6D
:10A210000B4330F8021B62440B43404512B220F856
:10A22000023CCFD1029B93F86610039B013B5BB2CB
:10A230005A1C12D0029A92F967209BE70B9B0C9A4A
:10A240004F1EFF1A04FB07F706EB470701FB04F656
:10A2500007EB46064FF0FF3CACE7029B93F8650026
:10A260000A9B4FEA4E0E3BBB052825D94FF0010B48
:10A270004FF40065099B089A0E9C01330993DBB2E9
:10A280002244834208920A93FFF465AF0F9B013387
:10A290000F93DBB28B42FFF44DAF029B93F8623019
:10A2A0000D9A01320D92D2B2934209F10C093FF698
:10A2B00036AF15B0BDE8F08F6D004FEA4B0BD9E714
:10A2C000029A92F86A10C1F101001146D26C91F81D
:10A2D0006010B2FBF1F100FB01F103EB4103E5E695
:10A2E00020211027CDE911174FF400411091FAE613
:10A2F000B0B110B500F0BCFA0446406A18B115F0D0
:10A30000FDFC00236362A06C18B115F0F7FC00237C
:10A31000A364206918B115F0F1FC0023236110BD7E
:10A32000704700BF2DE9F04794469DF824709DF8D2
:10A330002CA09DF830909DF834809DF838E09DF970
:10A340003C50109A002854D0052B28BF0523052F18
:10A350003E4628BF0526002D08BF0125002A48D00B
:10A36000002D80F8675080F86230B8BF6D4203EB73
:10A37000430380F84480EDB24FEA4308A0F85C1034
:10A380005FFA88F815FB01F100250446026080F8A9
:10A3900065C080F861A080F8349080F868E0A0F88B
:10A3A0005E1080F8636085644562404615F09AFC53
:10A3B0002061D8B1300115F095FC8146A064D8B178
:10A3C0002069089942462BF0BFFC67B10A9B591ED1
:10A3D0002B46A26C11F8015F02EB03120133D8B2D5
:10A3E00086421573F5D80020BDE8F0870220BDE84D
:10A3F000F0870320BDE8F087206915F07FFCC4F8E2
:10A4000010900220BDE8F08700286DD070B590F85C
:10A41000661090F865304A1E013BDBB2D2B280F87C
:10A420006B30012980F86C2088BF90F86C3090F870
:10A430006320044688BF03F1FF334FF000008CBF58
:10A44000DBB2012384F86D3084F86E00A065002A29
:10A450003DD00122254E034640F20335944612E0DA
:10A460001F2B86BF03F01F0331464FF0A0410CFAAB
:10A4700003F3C1F8083594F863100130C3B25200F9
:10A480009942D2B223D9A16C4FEA031E01EB031308
:10A490001B7B1F2B86BF03F01F0331464FF0A041EB
:10A4A00003F5E07341F8235094F86D301342A36C28
:10A4B00073441B7BD4D11F2B86BF03F01F0331468F
:10A4C0004FF0A0410CFA03F3C1F80C35D3E7206834
:10A4D00000F03CFA236801224FF47A715A60DA6086
:10A4E000C3F840151A6070BD704700BF00030050EC
:10A4F0002DE9F843836B026C1A60D0E90B231360DB
:10A50000826A1360036801255D601D64D3F84035DD
:10A51000C26A90F86B30016B1160044603F0FF08CB
:10A52000002B00F0AF80A74E2E4394F86B3094F8C8
:10A5300065200133DBB29A4284F86B300DD80022DB
:10A5400084F86B2094F86C3094F866100133DBB219
:10A55000994284F86C3040F2CF80226D236802FA71
:10A5600008F101225A604020DA60C3F840151A60F1
:10A57000B047D4E90F321A60B4F85E1094F86C302A
:10A5800094F865C094F86B2094F8600007310CFBD8
:10A590000322C910CB0000FB02F203FB02F294F885
:10A5A000683023B194F86A30E56C05FB032201287A
:10A5B00000F00A81022800F0B180636ACEB2711EF9
:10A5C0001A44CFB2D4E906506368A168002E41D086
:10A5D00002EB471C0CF1400C203252F8206C1E603C
:10A5E0001D6000BF00BF086052F81C6C1E601D603B
:10A5F00000BF00BF086052F8186C1E601D6000BFED
:10A6000000BF086052F8146C1E601D6000BF00BFE0
:10A61000086052F8106C1E601D6000BF00BF08602B
:10A6200052F80C6C1E601D6000BF00BF086052F83D
:10A63000086C1E601D6000BF00BF086052F8046C0B
:10A640001E601D6000BF00BF203262450860C4D19B
:10A6500094F865C0BCF1010F12D994F86B307BB946
:10A66000226801231364236DD2F84025C3EBC30392
:10A6700013440433626DDB08934238BF13462365ED
:10A68000BDE8F88390F863104E4E69B346F00107B9
:10A69000C14612E0A26C02EB031312589B681360D0
:10A6A0004FF40070B84794F8631009F101095FFA9C
:10A6B00089F36D009942EDB216D994F86C3094F894
:10A6C0006D2053401D42F0D094F86C205FFA89F35E
:10A6D0002A424FEA03101946DCD1A36C03EB0113A5
:10A6E000D3E901231360DBE794F86C30DBB246F06A
:10A6F000010684F86D3018E784F86C2094F86E3009
:10A7000043B194F86A30C3F10103DBB284F86A30D4
:10A7100084F86E20A36D0133A3651EE7606ACBB297
:10A7200000EB020E616894F86420581EC7B2D4E9A9
:10A730000665A06801EB4202002B8BD00EEB071CD4
:10A740000EF110030CF1200C33F8107C17800E6012
:10A7500000BF00BF056033F80E7C17800E6000BF9D
:10A7600000BF056033F80C7C17800E6000BF00BF8F
:10A77000056033F80A7C17800E6000BF00BF0560DB
:10A7800033F8087C17800E6000BF00BF056033F807
:10A79000067C17800E6000BF00BF056033F8047CA4
:10A7A00017800E6000BF00BF056033F8027C178081
:10A7B0000E6000BF00BF103363450560C4D194F83C
:10A7C00065C047E7A0620A00606ACBB200EB020EE8
:10A7D000616894F86420581EC7B2D4E90665A06881
:10A7E0000A44002B3FF436AF0EEBC70C0EF1080302
:10A7F0000CF1100C13F8087C17700E6000BF00BF3E
:10A80000056013F8077C17700E6000BF00BF05607D
:10A8100013F8067C17700E6000BF00BF056013F8C8
:10A82000057C17700E6000BF00BF056013F8047C44
:10A8300017700E6000BF00BF056013F8037C17702F
:10A840000E6000BF00BF056013F8027C17700E6039
:10A8500000BF00BF056013F8017C17700E6000BFD9
:10A8600000BF083363450560C4D194F865C0F1E6C4
:10A8700000285BD0436A002B58D030B490F86E208B
:10A8800002F0FF03002AF9D1026801245460146425
:10A89000816BD2F84025026C0A6090F86220B2B158
:10A8A000234D0269D25C1F2A29468CBF02F01F0289
:10A8B0004FF0A04104FA02F2C1F80C2590F8622092
:10A8C0000133DBB202EB4202B3EB420FE9DBB0F83B
:10A8D0005E3023B3164C00224FF0010C90F861302B
:10A8E0001F2B21468CBF03F01F034FF0A0410CFA31
:10A8F00003F3C1F8083500BF00BF90F861301F2B8B
:10A9000021468CBF03F01F034FF0A0410CFA03F364
:10A91000C1F80C35B0F85E3001329A42DED3826A5B
:10A92000036B1360C26A136030BC7047704700BF8E
:10A930000003005090F8683033B1012380F86E3086
:10A9400090F86E30002BFBD1704700BF194B984236
:10A9500012D003F58053984225D003F580539842D6
:10A9600023D003F58033984221D003F580539842D9
:10A9700008BF1B2101D0704708210023012242603B
:10A98000C0F80435C260C0F80835C0F810350A4B6D
:10A9900010B402FA01F14FF48034C0F80443196096
:10A9A0005DF8044B70470921E7E70A21E5E71A2122
:10A9B000E3E700BF0080004000E100E0BFF34F8FFD
:10A9C0000549064BCA6802F4E0621343CB60BFF34B
:10A9D0004F8F00BFFDE700BF00ED00E00400FA0567
:10A9E00070B510EE106A26F000450123B5F1FF4F57
:10A9F0002DED048BB0EE408A036024DAC5B1B5F1C9
:10AA0000E45F04460FDA002EBEBF4FF0FF33036051
:10AA1000B1EE400A2AF0F2FCB1EE408AB0EE480AEC
:10AA2000BDEC048B70BD002E14DAB5F1964F69DBD6
:10AA3000DFEDD37AB7EE007A87EE278AB0EE480AC8
:10AA4000BDEC048B70BD20EE008AB0EE480ABDEC70
:10AA5000048B70BDB5F17E5F51D0B5F1804F4ED003
:10AA60009FEDC79A730073D4C64B9D4240F3248276
:10AA7000C54B9D4240F3CE81B0EE007A37EE487A66
:10AA80009FEDBF0ADFEDC16A9FEDC16A9FEDC15A1C
:10AA9000DFEDC15A9FEDC18A67EE077AA7EEA66A7D
:10AAA000E7EE855ADFEDBE6A9FEDBE5AE6EE276AF5
:10AAB000A5EEA75A9FEDBC6ADFEDBC5AA6EEA76AC9
:10AAC000E5EE275ADFEDBA6AE6EE276A9FEDB96A2E
:10AAD000A5EEA76AA6EEA78ADFEDB76AE6EE276ABB
:10AAE00028EE078AF6EE005AA6EEA78AA7EE658A38
:10AAF00038EE008A002E91DA39EE488A8EE79FED13
:10AB0000A08A8BE7B5F17A5FC0F2E481F1EE408A6A
:10AB1000B0EE680A24F0A4FEF4EE408AF1EE10FADA
:10AB200040F0E780DFEDA57A77EEC87A17EE903A2D
:10AB300003F0010307EE903AF8EEE77A9B00062B4C
:10AB400000F22782DFE803F0588A8A54549999006A
:10AB5000B5F1824F80F2E080BDEEC87ADFED986AF1
:10AB60009FED986A9FED985ADFED985AF8EEC77AF4
:10AB700017EE103A78EE677A033BA7EEA66AE7EE87
:10AB8000855ADFED936A9FED935AE6EE276AA5EEAC
:10AB9000A75A9FED916ADFED915AA6EEA76AE5EEFE
:10ABA000275ADFED8F6A9FED8F5AE6EE276AA5EEF2
:10ABB000A75A9FED8D6ADFED8D5AA6EEA76AE5EEE6
:10ABC000275ADFED8B6AE6EE276AB7EE006AA5EE3C
:10ABD000A76A66EEA76AB6EE005A86EE868AA7EEE8
:10ABE000858A042B86D8DFE803F06A577C6D7F00E6
:10ABF000B7EE007A77EE677A9FED7E0ADFED600AA6
:10AC000027EE800A002000F0FDFEF1EE408AF5EE0E
:10AC1000408AF1EE10FA3FF40BAF68EE287A9FED10
:10AC2000750AF0EEE77A80EE270A2AF0E7FBF5EEE8
:10AC3000C08AF1EE10FA44BF4FF0FF332360B5F144
:10AC40007E5FB0EE409A00F05A81B5F1804FB1EED0
:10AC5000488A7FF407AF9FED4A8A4DE7B6EE007A47
:10AC600077EE677A9FED630ADFED450A27EE800AEB
:10AC700000F010FBF1EE408AC9E7B7EE087A77EEF4
:10AC8000C77A9FED5C0ADFED3E0A27EE800A00F0EE
:10AC900001FBF0EE408ABAE7B7EE007AB0EE080AA0
:10ACA00037EE800A20EE070AB0EE007A77EE877A58
:10ACB00027EE800A2AF0A2FB38EE008A1AE7B7EEE8
:10ACC000000AF1E7B7EE000AB1EE047A37EE877AB0
:10ACD00027EE000AB1EE007A37EE877A27EE007A87
:10ACE000DCE7B7EE000AF5E7B1EE080A37EE800AB6
:10ACF000EAE7F6EE007A68EEA78AB0EE680A24F07A
:10AD0000AFFD38EEC00A70EE007AB0EE677ABEEEA4
:10AD1000CF7A17EE103A12E7B5F1B94FB0EE480A04
:10AD200080F2E4802AF06AFBF7EE007A87EE886A08
:10AD300030EE670A9FED303ADFED303A9FED304A52
:10AD4000DFED304A9FED305ADFED305A9FED307A1B
:10AD500066EE067AF6EE006AE7EE833A78EE666A09
:10AD6000A3EEA74AE4EE274AA4EEA75AE5EE275A37
:10AD7000A5EE867AB0EE478AA6EE808ABAE600BFD4
:10AD8000000000006666663F17A6DD3FA283D3374A
:10AD900067976739752C3C384584E2383F239E3DE0
:10ADA000A1549C3A34B6053A7E02F23BC66E3D3B56
:10ADB00001F0893D1599A83C661AA53E0000004B9C
:10ADC00067FF0538B435F13ABDD7F536D6EE4B3AC4
:10ADD000E440DA3C54BF983CE6DC153E6E0F303E52
:10ADE0007ACCA63EC5D0383F5A245C3E3B2DB23FBC
:10ADF0003F239EBDDB0F4940E8C4D5BAD23D5B3A44
:10AE00005C061CBAFD0C503A610B36BBABAAAA3DDE
:10AE10001D7FD63E614B9D4274DDDFED617A9FED73
:10AE2000610A38EE678A28EE084ADFED5F5A9FED27
:10AE30005F7A9FED5F6ADFED5F6A9FED5F5ADFED3E
:10AE40005F4A64EE087AA7EEA56AE7EE876ADFED4F
:10AE50005C5A9FED5C7AE6EE275AA6EEA77A9FED44
:10AE60005A6ADFED5A6AA5EEA76AE7EE276AE7EEAF
:10AE7000854A9FED577A9FED575ADFED575AA6EE58
:10AE8000277AE6EEA75AA4EEA75A9FED546ADFEDA3
:10AE9000546AA5EE887AA5EE276A9FED528ADFED07
:10AEA000525AE6EE276AA7EE678A94EE268A38EEB3
:10AEB000658A38EE008A1DE6B0EE480A2AF09EFA4E
:10AEC0004A4B9D42B1EE400A5BDDB7EE007A37EEA9
:10AED000487AD7E59FED460ADFED320A28EE000AF0
:10AEE000002000F08FFDF0EE408A90E62AF086FA0E
:10AEF000F7EE007A30EE670A20EE088AFAE5B0EE47
:10AF0000408A8BE5F7EE007A38EE678A9FED250AD6
:10AF1000DFED386ADFED387A9FED387A9FED386AD9
:10AF2000E8EE267AA8EE076ADFED366A9FED367AFC
:10AF3000E7EE886AA6EE087ADFED347A9FED346A90
:10AF4000E6EE887AA7EE086ADFED326A9FED327A84
:10AF5000E7EE886AA6EE087ADFED307AE6EE887AC8
:10AF6000F7EE006AE7EE086A67EE887ABEEE006ADE
:10AF700087EEA67AF0EE477AE8EE067A37EE808A18
:10AF8000B8E5274B9D42C3DDDFED267A38EE678AB0
:10AF900049E7B0EE007A77EEC77A2DE61FA69D3F0F
:10AFA000C316BB3F0000000027F9A3B9F7E9AF398A
:10AFB00067F8663A85300DBA6B7BA53976F4B7BA77
:10AFC000FE7771BB9916143B3D37933CFEFC28BCC1
:10AFD0003C2117BE07E7C73B155A843D474D06BDC8
:10AFE0005EB9F73E521CE631CDCDF83D1F4A3B3FDE
:10AFF000DB0F49405E3C5B3C78756A3EDBD5523BDB
:10B00000AF72D53DB24B7A3FDFEF443FE73ABA3FEC
:10B010002D390840F400223FBE2E1D403F239EBD27
:10B0200007336D3E0C5BEC3E30B510EE103A8B4AA8
:10B0300023F0004C944587B0044664DD884A94456B
:10B0400010EE105A22DC002BDFED867A864A2CF0B7
:10B050000F0CB0EE407A40F3E780944570EE677ACB
:10B0600009BFDFED826A9FED827A9FED827A77EEEB
:10B07000E67A012077EEC76A77EEE67AC4ED006AD9
:10B0800077EEC77AC4ED017A07B030BD7A4A9445AD
:10B0900040DCDFED7A6ADFED735AF0EEC07AB6EE8F
:10B0A000007AA7EEA67ADFED726ABDEEC77A17EED8
:10B0B000100AB8EEC76A1F28E6EE657A26EE267AF1
:10B0C000F1EE465A6CDC6E4A411E23F0004352F802
:10B0D000212023F0FF03934262D077EEC76AC4EDCC
:10B0E000006A77EEE67A002D77EEC77AC4ED017A32
:10B0F000CADAF1EE666AF1EE677AC4ED006AC4ED71
:10B10000017A4042C0E7002284ED000A426000203C
:10B1100007B030BDBCF1FF4F77DA4FEAEC52863A08
:10B12000ACEBC25307EE903ABDEEE77ADFED556A1D
:10B13000B8EEC77A77EEC77A8DED037A67EEA67A16
:10B14000BDEEE77AB8EEC77A77EEC77A8DED047A6E
:10B1500067EEA67AF5EE407AF1EE10FACDED057ABB
:10B1600060D1B5EE407AF1EE10FA14BF022301234C
:10B17000454901910221009103A8214600F00CF9F4
:10B18000002D81DA94ED007AD4ED017AB1EE477AA0
:10B19000F1EE677A84ED007AC4ED017A404273E7FC
:10B1A00077EEC76A4FEAEC5216EE903AC3F3C753F4
:10B1B000C3EBDC5CBCF1080F91DD9FED2C7ADFED79
:10B1C0002D6AB0EE675AA5EE875A77EEC57AE5EE9E
:10B1D000877AD6EE267A75EE676AB0EE677A16EE53
:10B1E000903AC3F3C753D21A192A16DDDFED276A46
:10B1F000DFED274AF0EE457AE5EEA67A35EE677A7E
:10B20000A5EEA67A96EE247A67E770EE407A0020E3
:10B21000C4ED017AC4ED007A36E7F0EE457AC4ED6C
:10B22000006A5EE70323A3E7944570EE277A09BF1F
:10B23000DFED0E6A9FED0E7A9FED0E7A77EEA67A1D
:10B240004FF0FF3077EE876A77EEE67AC4ED006A5A
:10B2500077EE877AC4ED017A16E700BFD80F493F31
:10B26000E3CB1640800FC93FD00FC93F00443537AC
:10B270004344353708A3852E800F494384F9223F84
:10B2800028160A0000008043A8160A0000A3852E95
:10B2900032318D2410EE103A23F00043B3F1485FB1
:10B2A0002CDAFDEEC07A17EE903A002B60D020EE3B
:10B2B000007ADFED317A9FED315ADFED315A9FEDA3
:10B2C000316ADFED316AA7EE275ADFED307AE7EE1B
:10B2D000055AA7EE256AE7EE067AE7EE276A67EEDB
:10B2E000266A60EEC00AF6EE007AE7EE260AB7EEAE
:10B2F000000AD7EE270A30EE600A704720EE007A87
:10B30000DFED1D7A9FED1D5ADFED1D5A9FED1D6A81
:10B31000DFED1D6A1E4AA7EE275A9342DFED1B7A26
:10B32000E5EE075AA5EE876AE6EE077AE7EE876A4A
:10B3300066EE876AD5DD174A934214DC03F17F433A
:10B3400007EE903AB7EE006A36EE676A60EEC00A22
:10B35000F6EE005AD7EE257AE7EE260A77EEE00AF7
:10B3600036EE600A7047B6EE076AF5EE027AEDE750
:10B37000B7EE000A704700BF4ED747ADF6740F31E5
:10B380007CF293B4010DD037ABAA2A3D610BB6BA5B
:10B390009999993E0000483F2DE9F04F2DED048B1F
:10B3A000DBB01C4603930691A14B6899089253F8B1
:10B3B0002150111D824604F1FF38C0F29F82D31E36
:10B3C00044BF13460433DB1002930133DB000793C1
:10B3D000DDE907239B1A0593029B15EB0801A3EBFC
:10B3E000080315D401319FED937A699819441EAA78
:10B3F000002BA4BFC45C07EE904A03F10103ACBF6D
:10B40000F8EE677AF0EE477A8B42E2EC017AEFD100
:10B41000002DC0F2E382039B1EA901EB830446AE1C
:10B420004FEA830C4046EF180AEB8301B8F1000F96
:10B43000DFED807A09DB22465346F3EC016A32EDF8
:10B44000017A8B42E6EE877AF7D10130B842E6EC1A
:10B45000017A04F10404E9D109AB0AAF03EB8509D1
:10B4600007EB8503083B9FED759ADFED738A05981E
:10B4700004930AEB0C0446AE00955AAB03EB85032C
:10B48000002D13ED140A4FEA850B16DD06EB85033C
:10B490003A4660EE097AB0EE407AFDEEE77A73ED57
:10B4A000016AF8EEE77AB342A7EEE87A37EEA60A29
:10B4B000BDEEC77AA2EC017AEBD101904CF004FF0B
:10B4C000B0EE408AB4EE000A28EE000A24F0C8F973
:10B4D000F2EE007AA0EE678A01980028FDEEC89A85
:10B4E000F8EEE97A38EE678A76DD05F1FF3EC0F1C5
:10B4F000080357F82E1041FA03FC0CFA03F3CB1A99
:10B50000C0F1070219EE901A43FA02F26144002AD0
:10B5100047F82E3009EE901A66DCB5EE408AF1EE5F
:10B5200010FA40F0BE80009B05F1FF3B5B4510DC4C
:10B5300005F18043013B07EB83030021944653F858
:10B5400004294B4541EA0201F9D16246002940F045
:10B55000F180009B013B57F82330002B40F0E58041
:10B56000049B4FF0010C53F804290CF1010C002A44
:10B57000F9D005F1010BAC44DE46039B5919029B3F
:10B5800003EB0B05699B013D1D441EAB06EB8B0BCA
:10B5900003EB810115F8013F9FED267A07EE903A03
:10B5A000F8EE677AB8F1000FC1ED007A0A4601F1B2
:10B5B000040109DB534601E072ED017AF3EC016A04
:10B5C000A342A6EEA77AF7D10EF1010EE645ABEC49
:10B5D000017ADFDD654650E740F09D806B1E57F82D
:10B5E00023201212002A98DD19EE903A002D03F163
:10B5F000010309EE903A40F397813968002940F041
:10B600008080012D26D03B464FF0010C53F8041FDB
:10B6100000297AD00CF10103C1F580719D4247F8F1
:10B620002C1016DD57F82310BB4407EB83030AE008
:10B630001C160A0000000000000080430000803B50
:10B640000000C93F1968C1F1FF0143F8041B5B45C5
:10B65000F8D1012100280CDD012800F046810228E4
:10B6600007D105F1FF3C57F82C3003F03F0347F8B2
:10B670002C30022A7FF451AFB7EE000A30EE488A30
:10B6800000293FF44AAF099201904CF01DFE38EEBC
:10B69000408A099A0198B5EE408AF1EE10FA3FF41B
:10B6A00042AF0292DDE90732B0EE480A981A0195DE
:10B6B000009D4CF009FE1FED207AB4EEC70AF1EEB2
:10B6C00010FADDE90132C0F257815FED247A059965
:10B6D00060EE277A0831FDEEE77A0591F8EEE77A19
:10B6E00003F1010BA7EEC70AFDEEE77ABDEEC00A33
:10B6F00010EE101A47F8231017EE903A47F82B3047
:10B700002FE001234FF0000C86E70CF1010CAC4553
:10B710007FF47CAF9EE7F6EE007AB4EEE78AF1EEB6
:10B7200010FA80F2F0800022F7E605F1010BDE4608
:10B73000DC4622E70599A1F1080057F82B10059087
:10B740002B46009D69B903F18043023B07EB83035D
:10B75000014653F804090BF1FF3B08390028F8D0E3
:10B76000059105980092B7EE000A4CF0ADFDBBF1D3
:10B77000000F009AC0F225814FEA8B0E46AB03EB17
:10B780000E060EF1040C1FED537A07EB0C03311D6E
:10B7900073ED017AF8EEE77ABB4267EE807A20EE2D
:10B7A000070A61ED017AF3D1002D1FED5B6A4FF0BE
:10B7B000000420DB9148DFED927AB0EE467A314604
:10B7C000002303E09C4208DBB0EC017AF1EC016A53
:10B7D00001339D42E6EE877AF4DA5AAB03EB840339
:10B7E000A34543ED287AA6F1040604F1010305D030
:10B7F000002D1C46DEDADFED827AEEE76899022939
:10B800001CDC002900F392800FD132ABDFED7C7A93
:10B810009C443CED017A634577EE877AF9D10AB111
:10B82000F1EE677A069BC3ED007A19EE903A03F0C9
:10B8300007005BB0BDEC048BBDE8F08F689B032B69
:10B84000F3D1BBF1000F00F0D1805AAB734432A9A1
:10B8500013ED287A01EB8B0373ED017AF0EE476A62
:10B8600037EE277A994277EEC77A83ED007A77EE42
:10B87000A67AC3ED017AEFD1BBF1010F40F3B68098
:10B880000BF1804B5AAB0BF1FF3B9E444FEA8B0B05
:10B890000BF104031EED287A0B4433A873ED017AF3
:10B8A000F0EE476A37EE277A984277EEC77A83ED53
:10B8B000007A77EEA67AC3ED017AEFD10BF1080B8F
:10B8C000DFED4F7A01EB0B03083133ED017A99423A
:10B8D00077EE877AF9D1002A56D10699329A339BAE
:10B8E0000A604B60C1ED027A9FE705F1FF3C57F813
:10B8F0002C3003F07F0347F82C30BAE60823079377
:10B900000023029364E519EE903A002D03F1010340
:10B9100009EE903AC8BF02223FF76FAEF7EE007A09
:10B9200037EEC88A0222F8E5002193E632A9DFED5E
:10B93000347A01EB830333ED017A994277EE877A0B
:10B94000F9D19DED327A8ABB069BBBF1000FC3EDA6
:10B95000007A77EE677A0BDD33A90123B1EC017A27
:10B9600001339B4577EE877AF8DA0AB1F1EE677A10
:10B97000069BC3ED017A58E7BDEEC00A9B4610EE68
:10B98000101A47F82310ECE6DDED326A9DED337AAC
:10B99000069BF1EE666AB1EE477AF1EE677AC3ED87
:10B9A000006A83ED017AC3ED027A3EE7069BF1EE71
:10B9B000676ABBF1000F77EE677AC3ED006ACBDCF4
:10B9C000D4E7689B022B0DDC002B14DC7FF42DAF39
:10B9D000DFED0B7A002A3FF425AF21E7039B4FEA06
:10B9E000830C39E5689B032B7FF41FAFDFED047AEE
:10B9F000002AC9D171E7DFED027AA2E7F4150A0047
:10BA00000000000010EE103A23F00043B3F1485F4D
:10BA100004DAFDEEC07A17EE903A5BB360EE007A7E
:10BA20009FED157ADFED155A9FED156ADFED156A6A
:10BA3000E7EE875A9FED147AA5EEA76A20EE275A03
:10BA4000E6EE276AA6EEA77A30B9DFED106AE7EED8
:10BA5000876AA6EE850A704727EE457AF6EE006AF9
:10BA6000A0EEA67ADFED0A6AD7EE270AE5EE260AEF
:10BA700030EE600A704700BFD3C92E2F342FD7B2E3
:10BA80001BEF3836010D50B98988083CABAA2ABE95
:10BA9000ABAA2A3E10EE103A23F00042B2F1465F04
:10BAA00010DAFDEEC07A17EE901A01BB431C134367
:10BAB00000F0A280012800F0A880BFEE007AC7EE57
:10BAC000007A76E052498A4211DBDFED527A9FED2F
:10BAD000527A002BBCBFF1EE600AB1EE400A37EE9D
:10BAE000C00A77EE607ADFED4D0A37EE800A20EE6D
:10BAF000007A9FED4B5A9FED4B6ADFED4B5ADFED1D
:10BB00004B6A434967EE077A8A42A7EE856AE7EEF9
:10BB1000A56A9FED475ADFED475AA6EE275AE6EE93
:10BB2000A75A9FED456ADFED456AA5EE276AE5EE67
:10BB3000A76A9FED435ADFED435AA6EE275AE6EE79
:10BB4000A75ADFED416A9FED416AE5EE276AA5EE4F
:10BB5000A76AF0EE667AE6EE077A60EE075AF0EE34
:10BB6000606AE7EEA56A9FED3A5AE6EE870AE5EECF
:10BB7000850A70EE207A1FDA01281AD0BFEE007A0B
:10BB8000C7EE276A334B17EE902A1A4006EE102AAA
:10BB900016EE902A134007EE903AB7EE007AA6EE22
:10BBA000277A36EE400A70EEC00AA0EEA77AE7EEDA
:10BBB000267AB0EE670A704707EE100AB8EEC77A29
:10BBC00067EEA75A77EE877A9B17C5EEA76A03F050
:10BBD0000203C3F10103B0EE006A76EEE00A07EE5D
:10BBE000903A30EE600AF8EEE77AA0EE467A67EE19
:10BBF000877AB0EE670A7047B0EEC00AB7EE007AF7
:10BC0000C7EE007AB0EE670A7047F0EE407AD0E7F0
:10BC100040A12C3FDA0F493F682122330000000089
:10BC20005FAE9BB745F4A3388453D9377AC09538B3
:10BC3000C8261A3AB937813916696B3B48DEBE3AD5
:10BC4000A427B33C1F37113C8988083ED10D5D3DC8
:10BC5000ABAAAA3E00F0FFFF70B5044640F2514087
:10BC60000D4635F029FF50B1D0E9013228469568DC
:10BC7000984704F108012B46BDE870401847224957
:10BC8000284630F011FC0646C0B190F85030D90675
:10BC900033D443F0100304F1080180F8503020F051
:10BCA0006BF994F82A3013F00C0F304618BF0121BD
:10BCB000BDE8704008BF002120F050B92846134964
:10BCC00030F0F2FB0546D8B190F82A309A0714D428
:10BCD00043F0020304F1080180F82A301FF0A8F9AC
:10BCE00094F82A3013F00C0F284618BF0121BDE844
:10BCF000704008BF00211FF049B9054836F01CF814
:10BD0000044836F019F800BFE8EB0900C0E7090065
:10BD1000386E0900486E09000DF048BB2DE9F04F60
:10BD20000B4685B069468346002401AA1846009454
:10BD300032F070FC009902294FD9DBF8040001228F
:10BD4000890025F073F8009BCBF804408146ABF8DE
:10BD50000840002B3AD0DFF88CA02546019B00223A
:10BD6000029253F8250003AA02A934F0A1FC40F284
:10BD70003D42022102982AF029FF039B40F299518B
:10BD800018682AF079FF47F6FF7240F2995351463E
:10BD900080462AF00BFF039B40F29E5158682AF020
:10BDA0006BFFAE004E44074640F29E5347F6FF72CB
:10BDB00051462AF0FBFE29F825807780009B01344C
:10BDC000A4B29C422546C9D35B009BB2CBF8049039
:10BDD000ABF8083005B0BDE8F08F014835F098FFAA
:10BDE000147109000080FFFF2DE9F04F2DED028B4B
:10BDF00093468DB0C268BDF86490DDF86880BDF8E8
:10BE00006C701D9E04468A461D46B0EE408A2AB1DB
:10BE100043689A4200F0B6800DF0DAFDB9F11F0FC9
:10BE20005BD9BAF1000F00F0838000264FF0060ABC
:10BE3000BBF1000F74D040F201230DF1180BADF8E7
:10BE400018306B1CADF81A305846002307934CF09D
:10BE500077FC00283CD19FED4F0ADFED4F6A189B1D
:10BE6000029328EE000A4D4B0690C0EE267A03FBA3
:10BE700005F54B4BCBF81400002FA3FB0535CBE9A0
:10BE80000100CBE9030008BF4FF000080796B6EEAB
:10BE9000007A77EE877A6D0BFCEEE77A0126ADF833
:10BEA0000C90ADF81470CDF810808DF818A0CDED81
:10BEB000087AADF824508DF82D6002F019FA38B9DF
:10BEC000384D5A4602A928464CF014FC00283FD0B1
:10BED0000DB0BDEC028BBDE8F08F1F2FA1D8BAF1D9
:10BEE000000F2DD0002E4AD0F0EE0C7AB4EEE78A87
:10BEF000F1EE10FA304669460AD807EE905A9FEDE7
:10BF00002A7AF8EE677AF4EEC77AF1EE10FA3BD9A6
:10BF100000F068FC6E464FF0030ABBF1000F8AD1B7
:10BF2000CDE906BB0DF1180B58464CF009FC90E723
:10BF3000002F564614BF4FF0080A4FF00A0A77E761
:10BF4000002F564614BF4FF0040A4FF0050A6FE762
:10BF50001649224604F1280006F06EFF1C9B297842
:10BF60005AB230464CF0F6FB0028B1D12878314661
:10BF70004CF0C2FB0028ABD1189BE360A8E74FF060
:10BF8000010A55E71120A3E700F02CFC6E464FF0A4
:10BF9000020A4DE70024744900401C4440420F004F
:10BFA0005917B7D1B50601206666A63F9DE9020084
:10BFB000DFED0F7A20EE270A38B5BCEEC00A049DEB
:10BFC00041600446114680ED020A1A460C304BF0DF
:10BFD000EFFE35B1224628460649BDE8384006F056
:10BFE0002BBF21460348BDE8384006F007BF00BF1D
:10BFF00000007A44B55C03002DE9F843416099469E
:10C000004B680B9F9B7980F82C3090460A9A0285EA
:10C010008D7D044605F0300605F00605002B41D164
:10C020004FF6FF73C384002E35D1089BE36194F86B
:10C030002C20099B2362002384F82D3084F82A30B9
:10C04000A384CAB1002F36D022492246384606F0D2
:10C05000F3FE4EB116F0040137D00121606884F878
:10C060002B1000220DF0F4FE25B1AA060ED50223F6
:10C0700084F82B30BDE8F88317B3174922463846B9
:10C0800006F0DAFE002DF5D06B07F0D5012384F819
:10C090002B30BDE8F8834A46414604F108004BF0D6
:10C0A00087FEC2E74B68D86807F04CFC3346E08453
:10C0B0002E461D46B7E70748214606F09FFEC8E713
:10C0C0000548214606F09AFEDCE7606801220DF083
:10C0D000BFFEC9E7692F0700DD2F070030B5044612
:10C0E00015464FF6FF7283B0A28000220846A16079
:10C0F0002361A271E26001A9E57107F095FF002DAF
:10C1000004F1040201A90CBF012002204CF040FB05
:10C11000054610B1284603B030BDA188084600F09E
:10C1200013FC284603B030BD2DE9F04F89B09DF8CF
:10C130004840002B35D081464068DFF87CB0164679
:10C140001D465FFA81F842F0E7FE002C14BF002282
:10C1500020224FF6FF7A002755452C46D9F80400D7
:10C16000069628BF544603A9CDE9044701928DF8ED
:10C170000C708DF80D80079742F0B6FF58452644A5
:10C18000034602D12D1B019AE6D1D9F80400019390
:10C1900042F0A4FE019B184609B0BDE8F04F56F0EE
:10C1A0003FBEC9B20EF0F0FE002814BF00201320DD
:10C1B00009B0BDE8F08F00BF0000AD0B2DE9F04FD6
:10C1C00085B007460C460292002A40F0198201F120
:10C1D0000C053B78D4F800A03846002B76D00AF145
:10C1E00002024FF00008AA1803925646CDF80480C8
:10C1F000292B5AD05E2B00F2C381232B3FD9243B3D
:10C200003A2B3CD8DFE813F0A6013B003B003B0093
:10C210005E013B00B00091003B003B0007013B008A
:10C220003B003B003B003B003B003B003B003B0036
:10C230003B003B003B003B003B003B003B00E4007D
:10C240003B003B003B003B003B003B003B003B0016
:10C250003B003B003B003B003B003B003B003B0006
:10C260003B003B003B003B003B003B003B003B00F6
:10C270003B003B003B0010016F003B00650026685F
:10C28000002D00F05282731C23604FF00103AB5568
:10C2900023685A1C22603A78EA54394663680133AD
:10C2A00063604B784F1C002BA2D10199384649B1ED
:10C2B00023685B1A013B5AB29A4218BF48F0010842
:10C2C00005B16B54B8F1000F40F0928105B0BDE8A4
:10C2D000F08F002D00F0908123685022591C2160BE
:10C2E000EA542668D9E77B78791C002B00F080811E
:10C2F00043F02002642A266800F0358123F004030D
:10C3000043F02003732B00F02E81002D00F0B38149
:10C31000731C23604FF00103AB55787827687B1CB2
:10C32000236057F091F8E855B8E72268B24200F070
:10C330005F817B783F2B00F0F381002D00F00F82AE
:10C3400039466223AB542368F61A0133023EEE5499
:10C3500072B2B24218BF48F0010822686368961CA6
:10C360000133266063609CE72268B24200F040819E
:10C37000002D00F06781B01C921BA919284429F0F8
:10C3800013FD2368023360222360EA542368F21A03
:10C390002B44023A5A702368023323607B7851B2EF
:10C3A000914218BF48F001083F2B00F0CB8139467D
:10C3B0006123AB552368721C9E1B023E73B2AE54C0
:10C3C000B34218BF48F001085FFA88F826680BE10D
:10C3D0002268B24200F00C81002D00F02381B01CD5
:10C3E000921B2844A91929F0DFFC2368023323603B
:10C3F0007B783F2B00F0DD8139466123AB55236804
:10C40000721C9E1B023EAE5473B2B34218BF48F07A
:10C410000108266842E72668731C2360002D3FF45C
:10C420003CAF0223AB5538E77B7826685E2B07F1DB
:10C43000010100F05781002D00F08781731C2360FB
:10C440000323AB55236801332360636801336360C2
:10C450007B785D2B00F058814FF00009002B00F035
:10C46000C7805C2B00F00A812368002D00F0328128
:10C470005A1C22600A78EA540F467B782D2B00F074
:10C480000F810B785C2B00F01481002D00F01D81D2
:10C4900023685A1C22600A78EA540F467B785D2B89
:10C4A00007F1010109F10109D8D14FFA89F34B4590
:10C4B00018BF48F00108002D3FF4F3AEAB1983F824
:10C4C0000190EEE67B7826683F2B00F02081A36880
:10C4D00003F10109C4F80890002D00F02981731CB4
:10C4E00023607E23AB554FEA4903226859B2994233
:10C4F00018BF48F00108511C2160AB546368013338
:10C5000063604FF0010B2146029A781CFFF756FE3C
:10C51000014600286CD00278292A69D1BBF1000FAE
:10C520003FF4BFAE002D00F0478123687E22581CE7
:10C530004FEA4909206009F10109EA544FFA89F3E9
:10C540004B4518BF48F0010823685A1C226005F8C3
:10C550000390A3E6002D4FD023685122591C21607F
:10C56000EA54266899E6002D00F08580731C23604C
:10C570000523AB5523685A1C22607A78EA548DE66D
:10C580007C2B7FF47CAE019800283BD02268131AE4
:10C59000013B59B2994218BF48F00108002D34D030
:10C5A0002B542268039805EB0A063146A2EB0A02D7
:10C5B00029F0FAFB2368EA186021033323609170A5
:10C5C000236801931A4601326123226005F80A307C
:10C5D0002368A3EB0A03023B73705AB226689A429F
:10C5E00018BF48F00108394663680233636058E6B3
:10C5F000002005B0BDE8F08F2668013626604CE6C5
:10C600000025E6E5002DCCD12268161DD31C019330
:10C61000A6EB0A03023B5AB226609A4218BF48F0C2
:10C620000108E0E7023222607B783F2B00F0D080E7
:10C63000931B023B16465AB239469A4218BF48F03D
:10C6400001082BE6131D2360B21A043A797850B220
:10C65000904218BF48F001083F2900F09E809A1BC5
:10C66000023A1E4653B2934218BF48F001083946B9
:10C670005FFA88F8B8E7B31C23600FE648784F1CD0
:10C680000028B5D055B3D4F800B00BF101032360F6
:10C6900056F0DAFE05F80B007B782D2B7FF4F1AE17
:10C6A000BB785D2B3FF4EDAE5C2B07F102017FF40C
:10C6B000ECAE48784F1C00289AD03DB121684B1C45
:10C6C000236056F0C1FE6854E8E60F462368013344
:10C6D0002360E3E6013323600F46CEE6236801338F
:10C6E0002360CAE6002D43D0731C23600423AB559E
:10C6F000236801332360636801336360BB785D2B7B
:10C7000007F102017FF4A8AE4FF00009D6E6BB782E
:10C710003A2B7FF4DCAE4FF0000B0237D946F2E63D
:10C72000002D31D0791C61230CE6B31C2360B4E5E5
:10C730004FEA4903B21C22605AB29A4218BF48F02D
:10C740000108DBE6791C622333E66368013363602A
:10C75000B31C23607B785D2B7FF47EAEA1E5B31A1A
:10C76000023B58B23946984218BF48F00108F5E537
:10C77000636801336360B31C2360BB785D2B07F1F2
:10C7800002017FF469AE8CE5B31A023B58B2791C02
:10C79000984218BF48F00108E0E59A1B023A1E468D
:10C7A00053B2934218BF48F00108791C5FFA88F829
:10C7B0001AE7791C622321E622684FEA4903013314
:10C7C000023222605AB29A4218BF48F0010865E569
:10C7D000931B023B16465AB2791C9A4218BF48F086
:10C7E00001085BE530B502790B780D4662F347032B
:10C7F00005F8013B85B00C468068012201A92EF0A6
:10C80000ABF8019B1A68C4F801209B88AB8005B087
:10C8100030BD00BF10B51D4AB2F80CC0D189ACEBD9
:10C8200001039BB2044692F90000402B28BF40232D
:10C83000002882B009DB8C4520D0154A0021204613
:10C8400002B0BDE8104058F091BA8C450ED0916806
:10C850000F4801931A4629F077FA0D4A019B80216F
:10C86000204602B0BDE8104058F080BA8021002276
:10C87000204602B0BDE8104058F078BA00210A46C0
:10C88000204602B0BDE8104058F070BAAC1F01203D
:10C890005C46012010B50446900882B015D001EB2B
:10C8A000800051F8043B23608142FAD112F0030268
:10C8B00001D102B010BD0023014601A8019329F067
:10C8C00043FA019B236002B010BD0846EEE700BFAB
:10C8D0005FEA920C15D000EB8C0C0B6840F8043B1F
:10C8E0006045FAD112F0030200D1704700B583B061
:10C8F0000B68019301A9604629F026FA03B05DF8A0
:10C9000004FB8446EEE700BF08B502F04DFB08B11A
:10C91000012008BD02F02CFD80B902F05FFD78B95E
:10C92000084B1B68D90707D4DA03F1D413F4801F2E
:10C930000CBF0020042008BD052008BD022008BD52
:10C94000032008BD405701202DE9F041DFF8288081
:10C9500006460D4600244FF6FF7738F81400B8421B
:10C9600004F144042A46314601D04BF015FFB4F5DA
:10C97000AA7FF2D1BDE8F08118070120034B53F8DC
:10C98000203013B19A6801329A607047EC1E012082
:10C99000114B53F82000F0B1017942791F298ABF69
:10C9A0000E4B4FF0A04301F01F01D3F810351F2AA2
:10C9B00023FA01F38ABF09494FF0A04102F01F0298
:10C9C000D1F810155B00D14003F0020301F0010122
:10C9D00019434DF087BB7047183701200003005002
:10C9E0002DE9F04F0446ABB08B4640F25340214650
:10C9F00035F062F8002800F00F83012120462DF069
:10CA0000EDFF4268CDE90D4200230F938DF86430AD
:10CA10000DAD082105A85AF00BFA002328469946C7
:10CA2000CDE90B3356F0D4FCDFF830A6C8464F46AC
:10CA30009DF86440002C00F02981284656F0C8FC7F
:10CA4000A4F10903742B00F2298201A252F823F009
:10CA500031CA020031CA02009DCE02009DCE020002
:10CA600031CA02009DCE02009DCE02009DCE020082
:10CA70009DCE02009DCE02009DCE02009DCE020002
:10CA80009DCE02009DCE02009DCE02009DCE0200F2
:10CA90009DCE02009DCE02009DCE02009DCE0200E2
:10CAA0009DCE02009DCE02009DCE020031CA020042
:10CAB0009DCE0200C1CD02009DCE02009DCE02009F
:10CAC0009DCE02009DCE02009DCE02009DCE0200B2
:10CAD0009DCE02009DCE02009DCE020031CA020012
:10CAE00025CC02009DCE02009DCE020025CC020086
:10CAF00025CC020025CC020025CC020025CC02006A
:10CB000025CC020025CC020025CC020025CC020059
:10CB100025CC020031CA02009DCE02009DCE02004B
:10CB20009DCE02009DCE02009DCE02009DCE020051
:10CB30009DCE02009DCE02009DCE02009DCE020041
:10CB40009DCE02009DCE02009DCE02009DCE020031
:10CB50009DCE02009DCE02009DCE02009DCE020021
:10CB60009DCE02009DCE02009DCE02009DCE020011
:10CB70009DCE02009DCE02009DCE02009DCE020001
:10CB80009DCE02009DCE02009DCE02009DCE0200F1
:10CB90009DCE02009DCE0200B1CC02009DCE0200CF
:10CBA00063CC02009DCE02009DCE02009DCE02000D
:10CBB0009DCE02009DCE02009DCE02009DCE0200C1
:10CBC0009DCE02003DCD02009DCE02009DCE020012
:10CBD0009DCE02009DCE02009DCE02009DCE0200A1
:10CBE0009DCE0200F1CC02009DCE02009DCE02003F
:10CBF0009DCE02009DCE02009DCE0200A7CE020077
:10CC00009DCE02009DCE02009DCE02009DCE020070
:10CC10009DCE02009DCE020095CD02009DCE020069
:10CC200063CC0200002606960DE02B2C08D02D2C9C
:10CC300006D0204656F00AFD0346002800F0558134
:10CC4000284656F0C5FB214605A859F0DBFF9DF8A4
:10CC500064402E2C03D004F0DF03452BE5D10126E0
:10CC6000EEE7002F00F01A810B9B002B00F0EB8108
:10CC7000013B0C9A0B9352F82370384630F0C2FCFB
:10CC80009DF864408046002C7FF4D7AEBBF1000FC6
:10CC900000F09481002F00F001810B9B002B40F0ED
:10CCA000FD8005A85AF050F838462BB0BDE8F08F4B
:10CCB0000021084631F0F0FF0446A7B1D04571D0FD
:10CCC000B9F1000F00F0EA804946224638462FF0BD
:10CCD00033FE0C9B4FF00009002B6AD0394609A89F
:10CCE00031F058FC204630F08DFC274680469FE608
:10CCF0009DF86430752B40F0D180284656F068FBD3
:10CD00006C2840F0CB80284656F062FB6C2840F03F
:10CD1000C580284656F05CFB002F00F03F81D045CF
:10CD200000F07081B9F1000F00F02A8149460E220F
:10CD300038462FF001FE4FF0000979E69DF8643087
:10CD4000612B40F0AB80284656F042FB6C2840F047
:10CD5000A580284656F03CFB732840F09F8028466B
:10CD600056F036FB652840F09980284656F030FB97
:10CD7000002F00F03281D04500F04981B9F1000F59
:10CD800000F0048149461E2238462FF0D5FD4FF0B1
:10CD900000094DE6002031F0D5FD0446002FA2D059
:10CDA000D0458DD12146384631F0F4FB0C9B002B49
:10CDB00094D1012109A831F03BFC0C9B1F6091E745
:10CDC0009DF864100023069351B967E005A859F057
:10CDD00019FF284656F0FCFA9DF8641000295DD032
:10CDE000222900F099805C29F0D1284656F0F0FA0B
:10CDF000A0F162030146132BE8D801A252F823F0F8
:10CE0000A3CE0200CDCD0200CDCD0200CDCD0200DB
:10CE10005DCE0200CDCD0200CDCD0200CDCD020011
:10CE2000CDCD0200CDCD0200CDCD0200CDCD020092
:10CE300059CE0200CDCD0200CDCD0200CDCD0200F5
:10CE400055CE0200CDCD020051CE020061CE0200CF
:10CE50000921BBE70D21B9E70A21B7E70C21B5E7A6
:10CE600004240026284656F0B3FA40F02000C3B24E
:10CE7000A3F13002D2B2092A84BF573BDAB2013C97
:10CE800042EA0616EED1314605A859F0D3FE2846EF
:10CE900056F09EFA9DF864100029A1D16C4834F038
:10CEA0004BFF082192E79DF86430722BF6D128469B
:10CEB00056F08EFA7528F1D1284656F089FA652881
:10CEC000ECD1284656F084FA002F00F08E80D04531
:10CED00000F09380B9F1000F55D049463E22384604
:10CEE0002FF02AFD4FF00009A2E56EB30090024634
:10CEF0000390DDE9061034F029F9039B0446BFB323
:10CF0000D04546D0B9F1000F1CD0494602463846FC
:10CF100099462FF011FD8BE5284656F059FADDE9C8
:10CF2000061031F05DFF044617B3D04531D0B9F19A
:10CF3000000F07D04946224638462FF0FDFC4FF03F
:10CF4000000975E5A14673E5DDE9061033460A22BE
:10CF500034F086FA04465FB1D0451AD0B9F1000F1B
:10CF6000F0D0494602463846B1462FF0E5FC5FE571
:10CF700030F048FB2746BBF1000F7FF48BAE1DE07D
:10CF80004FF00E0954E54FF03E0951E54FF01E09F0
:10CF90004EE52146384631F0FDFA49E50E2030F0E5
:10CFA00031FB0E27BBF1000F7FF477AE9DF86400D4
:10CFB00056F074FB40B1284656F00AFA9DF864001A
:10CFC00056F06CFB0028F6D19DF86430002B7FF4FE
:10CFD00065AF002F7FF461AE60E71E2030F012FBDA
:10CFE0001E27BBF1000FE1D057E63E2030F00AFBD0
:10CFF0003E27BBF1000FD9D04FE63E21384631F035
:10D00000C9FA15E50E21384631F0C4FA10E51E21A3
:10D01000384631F0BFFA0BE5034610AA7E212046C0
:10D02000CDE917332EF0D4FC0A4A0B4B13920121A1
:10D030004022CDE914120DAD1AA913AACDE90D5362
:10D0400016911292E5E4BBF1000F7FF42AAEB5E72A
:10D050001C8A09002C420900853308006C4F090026
:10D0600038B50388112B0C460AD0362B06D119B1DE
:10D0700082888B899A420AD0012038BD002038BDB1
:10D080004FF6FF7201238A810B74002038BDC388DC
:10D09000CB81C5894A68954228BF154600F1100129
:10D0A0002A46206828F050FE0120A560207438BD73
:10D0B000C207034621D400B510F0030283B00BD1A0
:10D0C000114A016891421BD0184630F09BFA5E224B
:10D0D000C1880E4834F024FE022AF5D10C4A0240E1
:10D0E000062AF1D030F0E2F9FCEEC07ACDED017AFB
:10D0F0009DF8040003B05DF804FBC0F347007047DF
:10D1000030F072FAC0B2F5E73C4E0900807A0900AF
:10D11000070080FF30B585B00DF10F040DF10E034F
:10D1200001940D46009311460DF10D0303AA044628
:10D1300009F0A8FD9DF80F109DF80E209DF80D3008
:10D14000CDE9002120469DF80C20294609F094FEE7
:10D1500005B030BD70B500F110050446284654F006
:10D1600045FB3F2800D870BDA178002057F062FD34
:10D170000028F8D0284654F039FB3F28A17807D979
:10D1800004F59C724023BDE87040002057F0EEBDCE
:10D19000BDE87040002057F0A3BD00BF70B500F19E
:10D1A00010050446284654F021FB3F2800D870BDE6
:10D1B000E178002057F03EFD0028F8D0284654F0D2
:10D1C00015FB3F28E17807D904F638024023BDE873
:10D1D0007040002057F0CABDBDE87040002057F0F5
:10D1E0007FBD00BFF0B5294E7388CDB03122012438
:10D1F000B3F57F7F8DF80C208DF80D4038D20546B1
:10D20000022103A801F086F8074628BB738804337F
:10D21000AB4222D821F006FC7388334404AA1F7164
:10D22000311D04465FF0A9FB00BB9DF81C30DB06F6
:10D2300016D4204616495FF092FC044657F01AFCBB
:10D24000B4B900942346022203A912480DF026FB2C
:10D2500010480DF02BFA00E0002420464DB0F0BD40
:10D26000311D204652F0E8F90028E2D057F002FCC8
:10D2700000230222009303A906488DF80D201C46C6
:10D280000DF00CFB20464DB0F0BD00BFF84801206A
:10D29000FC480120FC4501202DE9F04F0446E1B097
:10D2A0006B480DF03DFAB0F1000AC0F2AB80694E58
:10D2B0007388B3F57F7F80F0B2800433A34205D931
:10D2C00001230393039861B0BDE8F08F21F0AAFB1E
:10D2D0007388311D5A1E8C5C2F2C00F099803344CA
:10D2E00000221A715C4A04A95FF03CF9002340F265
:10D2F0005112C6E90023C6E902330390002840F02A
:10D30000998018A904A85FF01EFA002840F09980BF
:10D31000DDF80CB004E05FF016FA0BF1010B28B950
:10D320009DF87A3018A904A8002BF4D1002104A894
:10D330005FF009FAC6F808B0BBF1000F52D0DFF871
:10D3400010814FF0000918A904A85FF0FCF9BDF89E
:10D350006A30BDF86810C6F8049003F01F0252004E
:10D360000192480AC3F344120092DB0A01F01F0243
:10D3700000F2BC70C1F3431153F0CCF8374B38497D
:10D38000C018A0FB01034FF00002306142F1000021
:10D3900001FB00309DF86C30706113F010033AD03F
:10D3A0000123B261F3600DF17A004FF07BFF054677
:10D3B000708050464BF036FC85B1002427462A1B6E
:10D3C000042A28BF04220DF17A0319190097144486
:10D3D000002340460DF062FAA542F0D809F1010998
:10D3E000D945B0D104A85EF0DDFB0023B26873809C
:10D3F00050467260F360B3614BF014FC039861B067
:10D40000BDE8F08F00230393039861B0BDE8F08F6F
:10D4100000238B5466E7F360189BB361C3E740F2C7
:10D4200051233380002303934BF0FCFB039861B03E
:10D43000BDE8F08F03225046727003934BF0F2FB6D
:10D4400040E7039C04A821465FF07DF9B460C9E77A
:10D45000FC450120F8480120FC48012080436D383C
:10D4600000CA9A3B38B52D4A2D4B0446012110685D
:10D470001D6841F013FC2B4A02F1200C52F8043FC6
:10D4800013B11979A14202D06245F7D138BDDA79DA
:10D4900032BB5A699969AA1A411AC2EB02420A447C
:10D4A000D9891C8AA4B214FA81F19C894FF6FF7CB9
:10D4B0004FF6FE7E724588BF6246B1FBF4FC04FB6A
:10D4C0001C119C6824F81120198A9C8989B2A142F8
:10D4D00019D21A8A013292B21A825D61986138BDFE
:10D4E0001F2C8ABF104A4FF0A04204F01F01D2F84F
:10D4F000102522FA01F15A7901F001018A42ECD09B
:10D500000022DA71E9E7DA8992B20132B2FBF4F172
:10D5100004FB112292B2DA81DFE700BFF05801204C
:10D520000C570120F43601200003005000B50278AA
:10D5300010F801EC72B191F800C0C31C13F8021C82
:10D54000614503D813F8011C614509D2013A03F182
:10D550000203F3D1BEF1030018BF01205DF804FB04
:10D56000AEF10300B0FA80F040095DF804FB00BFA3
:10D57000007840F02003642B4FEA5012C0F34010B3
:10D5800018D0732B0FD0097821F02003413B192BC1
:10D5900008D9A1F13003092B04D95F2902D0D04367
:10D5A00000F0010070470B78202BFBD0093B042BC7
:10D5B000F8D9F4E70B78303B092BF3D9D04300F0CE
:10D5C0000100EFE72DE9F04F2DED048B00F1080B82
:10D5D00091B0824606AF58461CF0A2FD28B92C3700
:10D5E000BD46BDEC048BBDE8F08F9AF862100029AF
:10D5F00040F05981DAF80C00002800F0E0801DF0BE
:10D6000043FB3860002800F0DA80396807F1100227
:10D6100058461CF02FFB6B4609EE903A002800F0AC
:10D62000C58007F110001BF02BFE064607F1100025
:10D630009AF852501BF03CFE9AF8993084B2002BB5
:10D6400000F0C680C6F3CF037B604FF4007308EE92
:10D65000103A082618EE103A640901340733A20084
:10D6600023F00703ADEB030DD31D23F007030DF1EA
:10D67000180807F11000ADEB030D08EE902A1BF01F
:10D68000FFFD06AB09EE103A7B680446002B00F064
:10D690008D800025C7E902554BE01BF009FE9AF882
:10D6A0005230DB0813FB00F91FFA89F9FB6818EE0A
:10D6B000902A0133002119EE100AFB6028F0F4FBD8
:10D6C00018EE102A0021404628F0EEFB19EE102A31
:10D6D000434607F11C0158461CF014FB58461CF049
:10D6E000C1FA002862D058461CF0B8FA9AF8971090
:10D6F000012239B9DAF808000092DAF824500AF168
:10D700009403A847DAF80800CDF8009000224346B9
:10D710000121DAF82450A84758461CF0EFFA56F0D9
:10D720004FFABB687A6833449BB2BB60BB899A42AC
:10D730003CD9B8687B8A3A8ABA8332181A440344BF
:10D7400000219BB29AF899007962FB83B98A3984E7
:10D75000B44223442CBF7A847B849AF893209AF8AD
:10D760009210049007F11C000390002002909AF898
:10D77000970001904FF48073009358461CF0E8FA2C
:10D780009AF85230A41B072BA4B207F11C0084D8CE
:10D7900007F11C001BF08CFD9AF852900823B3FB94
:10D7A000F9F9B0FBF9F01FFA80F97FE73B6819EE51
:10D7B000902A9B683B609546002B7FF426AF584625
:10D7C0001CF0B0FA2C37BD46BDEC048BBDE8F08FE1
:10D7D00007F110001BF06CFD2023B3FBF5F5B0EB57
:10D7E000C51F4FEAC5181CD864090134A30008EE10
:10D7F000903A073323F00703ADF5007D0DF11808CB
:10D8000007F11000ADEB030D1BF03AFD06AB09EE7E
:10D81000103A01237B604FF4007308EE103A04467F
:10D8200037E707F110001BF0EDFD9AF85230B8FB16
:10D83000F0F6012E38BF0126072B0BD89AF8592095
:10D8400042B90822B2FBF3F3B6FBF3F203FB126317
:10D85000F61AB6B207F110001BF012FDB0FBF6F09D
:10D8600084B207F110007C601BF00AFDB0FBF6F3F8
:10D8700003FB16039BB21BB1234601339BB27B60B3
:10D8800007F110001BF0BEFD16FB00F084B2B4FBE4
:10D89000F5F305FB13459AB20DB1531C9BB29B00E7
:10D8A00008EE103AD6E60023CAF844300AF13C03E9
:10D8B0003B60AAE62DE9F04F2DED088B8FB0C36ECB
:10D8C00000AF054600F170045B6878612146806E08
:10D8D00098472B6F002B00F027812B460833184602
:10D8E00008EE903A1CF01CFC95F8621049B97B696F
:10D8F000D868002800F014811DF0C6F9786030B9AE
:10D900000EE17A690023536402F13C037B607D6978
:10D91000B5F84A2007326B46D2100BEE103AD31DF1
:10D920006946DB08A1EBC3039D460021684628F049
:10D93000BBFAEB6EA86E5B6821469847E9464FF04C
:10D94000010A796818EE900A07F120021CF092F99A
:10D950006B460AEE903A002800F0D0807A6992F87F
:10D960005230072B16D892F859209AB1B7F92420D3
:10D970000821B1FBF3F31A4499B2013A92FBF3F296
:10D9800012FB01F2BA84B7F9202092FBF3F202FBFA
:10D9900003F33B8407F120001BF072FC7B69B86144
:10D9A00007F1200093F852402023B3FBF4F41BF05E
:10D9B0007FFC054607F120001BF07AFCB0EB441F0A
:10D9C0004FEA441600F2BD80C5F34A1301339B00B1
:10D9D00009EE103A073323F00703A0B06A4607F1B7
:10D9E0002000ADEB030D08EE102A1BF049FC6B463E
:10D9F0000AEE103A0123BB60802309EE903AF861E9
:10DA00004FF00008C7F810804146B88C7A8CFD6949
:10DA100038860023B8697B633B8CBB8553189BB267
:10DA2000A842FB8500F2868043181A44FB607A8680
:10DA3000D7E906239B1A9BB219EE102A00211AEE91
:10DA4000100AFB6128F030FA19EE902A002118EE36
:10DA5000100A28F029FA18EE103A1AEE102A07F1E7
:10DA60002C0118EE900A1CF04DF97B69B7F92C00D7
:10DA700093F85210B7F93020B3F88E60B7F92E4002
:10DA8000B3F88C50121A11FB00F301FB02F2002BC9
:10DA9000796906FB0455B8BF073305EBE3030D6F47
:10DAA0001D44B7F93230002AA4B2B8BF0732A342EE
:10DAB0004FEAE20B18DD18EE108AE20804F00703C3
:10DAC00019F802100AFA03F30B4309F80230414631
:10DAD00028465A4628F038F90134B7F93230A4B252
:10DAE0009C42D8443544E8DB3C6901343C6156F043
:10DAF00067F8BA68B989A3B29A4286D87B681AEEE9
:10DB0000902A9B687B609546002B7FF41AAF7A6958
:10DB1000D36E906E9B68494698471BEE103A9D461F
:10DB200018EE900A1CF0FEF83C37BD46BDEC088BA1
:10DB3000BDE8F08FFA6913447B86BB690B44FB6038
:10DB400076E707F120001BF05DFC7A69B6FBF0F088
:10DB500092F852300128014638BF0121072BB961E4
:10DB600003D892F85920002A48D007F120001BF072
:10DB700087FBBD69B0FBF5F086B207F12000BE60FF
:10DB80001BF07EFBB0FBF5F303FB15039BB21BB14F
:10DB9000334601339BB2BB6007F120001BF032FC1F
:10DBA000BB6913FB00F083B2B3FBF4F204FB123445
:10DBB00092B20CB1013292B25B099200013399002A
:10DBC000D31D23F00703ADEB030DCB1D09EE902A07
:10DBD000DB086A46A2EBC3039D4607F1200009EE6D
:10DBE000101A08EE102A1BF04BFB6B460AEE103A97
:10DBF000BB68F861002B7FF403AF7FE70820B0FB20
:10DC0000F3F3B1FBF3F003FB1010081A83B2BB610E
:10DC1000ABE700BF2DE9F0414368DB6884B0044600
:10DC20000D4640F2514053F8211033F045FF0746AE
:10DC3000002858D062684368D26852F82500984797
:10DC4000BB6801A95B6880469847BB6806469B682D
:10DC500040460021984763682449DB6853F8250053
:10DC60002EF022FC074668B190F850306FF3041391
:10DC700001A980F850301DF05FFE002106463846AD
:10DC80001EF07AF963681A49DB6853F825002EF014
:10DC90000BFC054668B190F82A306FF3410301A9E7
:10DCA00080F82A301CF08CFF0021064628461DF023
:10DCB000BFF97EB194F82A30DB070ED504F11802C3
:10DCC00001A910461BF050FB94F82A3043F00103E1
:10DCD00084F82A3004B0BDE8F08104F1180101A8ED
:10DCE0001BF0A0FAF0E70646B5E700BFE8EB090035
:10DCF000C0E70900F8B50D4F0D4B4FF0000C04467E
:10DD00000D46164687F800C04FF0FF0C83F800C0A0
:10DD100001F0AEF8324629462046F9F7F1FF3246C7
:10DD200029462046BDE8F84001F056BB205F01209F
:10DD3000215F01202DE9F043364F86460D462846E7
:10DD400015F8014BE65D16F00806F8D12D2C2FD101
:10DD50002C780126851C002B57D0102B09D1302C94
:10DD600007D1287800F0DF00582849D16C781023BB
:10DD700002354FF0FF380027B8FBF3F803FB08F932
:10DD80006FEA09093846A4F1300CBCF1090F14D828
:10DD90006446A34222DD002F1DDB80451BD301D149
:10DDA000A14518DB00FB0340012715F8014BEAE70A
:10DDB0002B2C04BF2C78851CCDE7A4F1410CBCF1C1
:10DDC000190F01D8373CE4E7A4F1610CBCF1190F3D
:10DDD00004D8573CDDE74FF0FF37E6E7002F07DABE
:10DDE0002223CEF800304FF0FF3032B9BDE8F08387
:10DDF00006B14042002AF9D007B1691E1160F5E76B
:10DE00003024002BB5D10823B3E7302CA9D00A2346
:10DE1000AFE700BFB5630A0010B59A42A2EB030456
:10DE20008E46A4B202D24189641AA4B2B0F804C0EA
:10DE3000A44507D2944515D941896144521A91B23B
:10DE4000018264461CB914E0A3EB0C039BB29C4511
:10DE5000FAD9C2880168704602FB031127F074FFEB
:10DE6000012010BD8489A2EB0C0189B28C42E7D25B
:10DE7000E2E7204610BD00BF2DE9F04782B005461D
:10DE8000BDF828C09DF82C00A3EB0C0463450E469A
:10DE9000A4B202D26989641AA4B2B5F804E0A64516
:10DEA0000BD29E455ED9698971445B1A99B2298269
:10DEB000B5F810C074461FFA8CFC002C4ED094426A
:10DEC00028BF1446E64505D8ACEB0E0C1FFA8CFCB7
:10DED000E645F9D9EA882968A4EB0E036344AEEB62
:10DEE0000C0E13FB02F39FB201281EFB02F302FB90
:10DEF0000C181FFA8EFE1FFA83F93AD1744544D9E3
:10DF000029F0030A1FFA8AFA524641463046FEF7C4
:10DF1000C1FC19F0030952D008EB0A01C9F1040849
:10DF20001FFA88F8B84528BFB846A7EB08034A4649
:10DF30009FB201A80023019327F006FF01AB2D68D3
:10DF400003EB09005FFA88F2B8F1000F03D029460D
:10DF5000154427F0F9FE019B33609FBB204602B0B9
:10DF6000BDE8F087AC89A3EB0E0189B28C429ED24A
:10DF700099E7744514D804FB02F24146304627F075
:10DF8000E3FE204602B0BDE8F08714FB02F2304603
:10DF900092B24146FEF77EFC204602B0BDE8F08713
:10DFA00041464A46304627F0CFFE29683A4606EBFE
:10DFB000090027F0C9FE204602B0BDE8F0872D68B1
:10DFC000002FCBD03A4629463046FEF763FCC5E722
:10DFD0002DE9F04F0546C789008A8846297A83B023
:10DFE000BFB280B200293ED1391A8742AC8889B2CB
:10DFF0004DD3661AB6B2964228BF1646301BEA8841
:10E0000080B2A742BC4605D3ACEB040C1FFA8CFCD3
:10E01000A445F9D2604410FB02F0A4EB0C011FFAF6
:10E0200080F9286811FB02FA012B02FB0C0489B26B
:10E030001FFA8AFA22D18E4232D816FB02F292B22D
:10E0400041462046FEF744FCF3199BB29F4202D89A
:10E05000AA899A4202D26A8913449BB23046EB8164
:10E0600003B0BDE8F08FAC88A24214D3161BEA8837
:10E07000074602FB068800202646C2E78E4242D8A9
:10E0800006FB02F24146204627F05EFEDCE7688987
:10E09000091A89B2ADE7101B164680B2EA88B0E7CC
:10E0A0002AF0030B1FFA8BFB5A4641462046FEF727
:10E0B0000FFC1AF0030A32D004EB0B00CAF104047F
:10E0C000A4B24C45D8F80030019328BF4C465246C4
:10E0D00001A927F039FEA9EB040901AB03EB0A0102
:10E0E0001FFA89F9D5F800A0E2B21CB1504692445B
:10E0F00027F02AFEB9F1000FA6D04A464146504605
:10E10000FEF7E6FBA0E741465246204627F01CFEFC
:10E1100028684A4608EB0A0127F016FE94E7D5F86E
:10E1200000A0E7E72DE9F84343689A68002A33D056
:10E13000DFF88880204F064600240FE072684368AD
:10E14000D26852F824009847AB6806F108019B6832
:10E15000984773689A68013494421DD2DB6840F294
:10E16000514053F8241033F0A7FC4FEA84090546C8
:10E170000028E3D17368DB68414653F824002EF091
:10E1800093F9394650B106F108011DF0F5FE7368A8
:10E190009A6801349442E1D3BDE8F8837368DB6880
:10E1A00053F809002EF080F90028D2D006F10801BA
:10E1B0001CF03EFFCDE700BFC0E70900E8EB090017
:10E1C00090F95030234910B5002B836AB4BF428ABE
:10E1D000028AB0F90CE0002B08BF0B46997BD9B13D
:10E1E00093F90540B3F802C004FB0ECC0FFA8CFC87
:10E1F000A0F846C00EEB020193F905205C8812FBE3
:10E2000001F323441BB29C45D2BFA0F84A30A0F8CA
:10E210004AC0A0F8463010BD93F90440B3F800C0DE
:10E2200004FB0ECC0FFA8CFCA0F844C00EEB0201EC
:10E2300093F90420B3F800E012FB01F373441BB21E
:10E240009C45D2BFA0F84830A0F848C0A0F84430A0
:10E2500010BD00BF9803012090F95030234910B53C
:10E26000002B836AB4BF028A428AB0F90EE0002B09
:10E2700008BF0B46997BD9B193F90440B3F800C0AD
:10E2800004FB0ECC0FFA8CFCA0F844C00EEB02018C
:10E2900093F904201C8812FB01F323441BB29C4514
:10E2A000D2BFA0F84830A0F848C0A0F8443010BD54
:10E2B00093F90540B3F802C004FB0ECC0FFA8CFCB6
:10E2C000A0F846C00EEB020193F90520B3F802E076
:10E2D00012FB01F373441BB29C45D2BFA0F84A3035
:10E2E000A0F84AC0A0F8463010BD00BF9803012036
:10E2F00000B589B00822694606F098F910B909B04E
:10E300005DF804FBC2B2002168464AF007FA09B082
:10E310005DF804FB70B582B005460E464DF038FD41
:10E3200018B90024204602B070BD044656F07AFBAE
:10E330000028F6D105236B7032460090034629462B
:10E3400001480CF0ABFAEDE7FC45012008B510EEF2
:10E35000102A22F00043B3F17E5F2DED028B09D32A
:10E3600052D070EE407A9FED5E7A87EE270ABDECC0
:10E37000028B08BDB3F17C5F07D2B3F14A5F4ED880
:10E38000BDEC028B9FED570A08BD002AB7EE008A4C
:10E390006ADB38EE400AB6EE008A20EE088AB5EE57
:10E3A000408AF1EE10FA00F18D80B1EEC87ADFED0F
:10E3B0004E7ADFED4E6A9FED4E0A9FED4E6AE8EE13
:10E3C000276A17EE103A23F47F6323F00F03A8EEB9
:10E3D000260A07EE903AF0EE485AF7EE006AE8EEA9
:10E3E000066AE7EEE75A28EE008A37EE876A85EE7E
:10E3F000860A88EE266ABDEC028BA6EE070A37EE87
:10E40000800A30EE000A08BDBDEC028B9FED3A0A8F
:10E41000DFED337A002AA8BFB0EE670A08BD20EE10
:10E42000007ADFED316ADFED317ADFED315AE7EE68
:10E43000267ABDEC028BE7EE275ADFED2E6ADFED80
:10E44000297AB7EE006AA7EE266A27EE257ADFED75
:10E450002B6AC7EE065AB0EE667AA0EE657A30EE09
:10E46000470A37EEC00A08BD30EE080AB6EE008A49
:10E4700020EE088AB5EE408AF1EE10FA29D4F1EECA
:10E48000C85ADFED197A9FED196ADFED196A9FED21
:10E49000150AA8EE276ADFED177AE8EE066AB7EEEE
:10E4A000007AA8EE277A28EE268ADFED157AC8EEE4
:10E4B000076AE6EEA57A77EEA57A30EE670A30EEC7
:10E4C000000A54E7B0EE480A4CF0E8FEB0EE407A9D
:10E4D0006DE7B0EE480A4CF0E1FEF0EE405AD0E7AE
:10E4E00000000000DA0FC93F6BD30DBCBA132FBD7B
:10E4F00075AA2A3EAEE534BFDA0F49406821A2333F
:10E500006821A2B308B510EE103A5A002DED028B27
:10E51000B0EE408A28D523F00042B2F18B4F08D3E9
:10E5200026F06CFFBDEC028BDFED207A30EE270A7F
:10E5300008BDFFEE007AE0EE007A70EE008AF5EE9C
:10E54000407AF1EE10FA26D4B1EEE70A38EE008AEE
:10E55000F7EE007A87EE880A38EEC00ABDEC028B2F
:10E56000BDE8084026F04ABFB7EE000A38EE408A00
:10E5700078EE087AE8EE087AF5EE407AF1EE10FAD5
:10E580000ED4B1EEE70A38EE000ABDEC028BBDE80E
:10E59000084026F07BBEB0EE670A4CF07FFED5E760
:10E5A000B0EE670A4CF07AFEEDE700BF1872313F1B
:10E5B00070B588B00D460C2000211646039327F055
:10E5C00017F80F4B036005AB01930E4B039A0093B2
:10E5D000044603233146284628F0AAFA9DF818205D
:10E5E0000599204608F04CF99DF81C3013B92046D7
:10E5F00008B070BD204608F065F9204608B070BD2F
:10E6000038C0090084C0090010B5044608F03CF980
:10E61000204610BD08B5086808F092F90E2008BD24
:10E6200010B58EB003AB51F8044B0193184B009317
:10E630000138032328F00EFA606806AA40F26E4102
:10E640002DF0C6F9227A049B03980599520042F0F6
:10E650000102089240F62612CDE909025B006FF034
:10E66000004243F0010391420B930ED0490041F068
:10E67000010140F2E643CDE90C31022106AA022055
:10E6800029F052FF0E200EB010BD0121F6E700BFA9
:10E690006CC0090010B58EB003AB51F8044B019368
:10E6A000184B00930138032328F0D4F9606806AAB8
:10E6B00040F297512DF08CF9227A049B039805992A
:10E6C000520042F00102089240F62612CDE90902FA
:10E6D0005B006FF0004243F0010391420B930ED0B8
:10E6E000490041F0010140F2E643CDE90C3102213D
:10E6F00006AA022029F018FF0E200EB010BD01213D
:10E70000F6E700BFCCC0090030B597B003AB51F8B5
:10E71000044B0193314B00930138062328F09AF9FA
:10E72000606809AA4FF4B3612DF052F9227A039878
:10E73000059B0699520042F001020B92049A5B007D
:10E74000CDE90C026FF0004243F0010344F2A61041
:10E750009142CDE90E0338D0490041F0010144F265
:10E7600086120923CDE910214FF00B0E4FF00A0C51
:10E770001C46032116AA02EB8300079B02EB8C0CBC
:10E780005B0043F00103089A43F6960540F8345CB9
:10E790004CF8343C6FF000439A420FD016AB03EBB9
:10E7A0008E0E03EB8404520042F00102013143F665
:10E7B00076034EF8343CC9B244F8282C09AA032049
:10E7C00029F0B2FE0E2017B030BD07234FF0090E1E
:10E7D0004FF0080C1C460221CCE700BF9CC009008A
:10E7E00070B58EB00D46182000211646059326F010
:10E7F000FFFE174B036007AB0193164B059A00937E
:10E80000044607232846314628F092F91249089811
:10E81000079D40F29E2228F01FFA9DF834209DF8B3
:10E8200030309DF82C10CDE902320A9A9DF8243040
:10E83000CDE900212046089A294608F091F8089869
:10E8400018B1002201210DF091FA20460EB070BDE2
:10E8500018C1090034C1090088DD090008F092B828
:10E8600008B5086808F0D6F80E2008BD2DE9F0417B
:10E87000054682B001F134000E4603F00FFC2B88F0
:10E88000102B31D0112B2BD10022A888364F1346E4
:10E8900037F81210814202F1440203D00133052BF4
:10E8A000F6D1042303EB031307EBC3042F482146DF
:10E8B0004FEAC30804F0DAFAE36D4FF6FF7227F867
:10E8C00008200E2B4FF0000284F85A2002D05A6024
:10E8D0002A7A1A7200230120B36102B0BDE8F081E8
:10E8E000002002B0BDE8F08100231F4F1A464FF60A
:10E8F000FF7037F81310814203F1440303D0013253
:10E90000052AF6D1042202EB0212D400AB883B5355
:10E9100007EBC2020E234FF0000804F16000D3653C
:10E92000384482F85A80A2F87680104904F084FABC
:10E93000C6F81880286969696C34274403C768469B
:10E9400049F0FAFEBDF800302A8A9A4202D86A8A53
:10E950009A4203D2A888694649F0D6FE00230120D6
:10E96000F36002B0BDE8F0811807012001620400E5
:10E9700070B50E46C18A044601318900006915460A
:10E9800026F06CFEE38A2061591CE18200EB8302D1
:10E99000002120F823109670D57070BD10B5038843
:10E9A000102B0C4606D0262B0CD108460BF010F885
:10E9B000012010BD81880022032049F0CBFE2046B3
:10E9C0000BF006F8002010BD30B5830787B0044671
:10E9D00021D1134B154602689A421CD108460122E8
:10E9E00069462BF0B9FF03A9284602222BF0B4FF99
:10E9F000019D049A2946204656F060FF009903982D
:10EA00002A4627F0A1F92046DDE9031208F0F4FABE
:10EA10000E2007B030BD0348F32133F081F900BF69
:10EA200060C30900A86B090030B5830787B00446AE
:10EA300021D1134B154602689A421CD10846012287
:10EA400069462BF089FF03A9284602222BF084FF98
:10EA5000019D049A2946204656F030FF00990398FC
:10EA60002A4627F071F92046DDE9031208F0D6FAAC
:10EA70000E2007B030BD0348F32133F051F900BF39
:10EA800060C30900A86B090008B5830709D1074BCB
:10EA900002689A4205D190F80C01400040F0010054
:10EAA00008BD0348F32133F03BF900BF60C3090000
:10EAB000A86B0900F0B58BB0234C009405AD084657
:10EAC000019511461A46052328F032F800214FF42B
:10EAD0008A7026F08DFD1D4B0360044601220598C7
:10EAE00002A92BF039FF039E26F00803102B01D05A
:10EAF000202E22D1069D029F022D0DDD062D0DD167
:10EB0000079870B102A901222BF012FF48B1039BB4
:10EB1000102B15D1029B05E0002DF1DC0C4833F0E1
:10EB2000F7F800230095089D0195204632463946A6
:10EB300008F056FA20460BB0F0BD064833F0E8F86E
:10EB40000548102133F0ECF8B4C3090060C3090094
:10EB5000D87109000C6E0900006D09002DE9F04123
:10EB60000C4684B0012201A905466068D4F80080F3
:10EB70002BF0F2FEDDE901760FB326F00803102B2F
:10EB800001D0202E18D1022D09D80023404632464C
:10EB9000394608F055FA0E2004B0BDE8F081012294
:10EBA000A06801A92BF0D8FEDDE90132102AEDD0D2
:10EBB0000448102133F0B4F8034833F0A9F80348AF
:10EBC00033F0BAF8006D09000C6E0900686F090097
:10EBD000830710B5044615D10C4B02689A4211D137
:10EBE00008462EF0B9FC0228014606DD062806D1AB
:10EBF000204608F041FA0E2010BD0028F8DC044839
:10EC000033F086F80348F32133F08AF860C3090033
:10EC1000D8710900A86B09002DE9F04F87B002AF49
:10EC200007F10C03214C01930094012381468A468D
:10EC3000002027F00FFF5146484656F041FFFE687E
:10EC400030462FF06FFC4510AB00073323F007036D
:10EC5000ADEB030D02AB7B60EDB1DFF85C8001AC86
:10EC60004FF0000B08E0026842450FD10BF1010B99
:10EC70005D4544F8040F0ED04FEA4B01042241F0E9
:10EC80000101304631F052FC8307ECD0084840F2D5
:10EC9000271133F045F8514648467B682A4608F06C
:10ECA00085FA0448002133F0A9F800BFC0C4090068
:10ECB000A86B0900AC47090088DD090038B510B918
:10ECC0000E24204638BD0D46044656F0F9FE29466E
:10ECD000204608F0F5F904464AF000FC204638BD0D
:10ECE000D0B110B50D4B0E4C93F800E084460439BA
:10ECF000002301E09C450DD051F8040F820703F179
:10ED00000103F7D10268A242F4D142681279724538
:10ED1000F0D110BD0E2010BD0E207047215F0120E4
:10ED200008C5090070B588B00D460C2000211646B4
:10ED3000039326F05DFC0F4B036004AB01930E4B75
:10ED4000039A0093044631462846042327F0F0FE38
:10ED5000049856F07BFE01469DF81C0000909DF83B
:10ED600018309DF81420204608F0E0F9204608B03D
:10ED700070BD00BF08C5090034C5090008B508F01A
:10ED8000E9F9002808BF0E2008BD00BF08B508F04B
:10ED9000E3F9002814BF3E201E2008BD10B5044C26
:10EDA000237803B110BD17F077F90123237010BD4C
:10EDB000E95D01200E4A0F49506810B50E4C002342
:10EDC0000009C4E9001310D00C49D26891F800E0A2
:10EDD00002F1040C01E0834207D05CF83320117982
:10EDE000714503F10103F6D16260034810BD00BF15
:10EDF00048AE090008C50900A8470120215F01208D
:10EE0000F8B5184F184E00240125D7E90023D6E99C
:10EE10000010A4F1200CC4F1200E05FA0CFC25FA18
:10EE20000EFE114303434CEA0E0C05FA04F20A40AD
:10EE300003EA0C031343E0B207D048F0A5FC2046D8
:10EE40003EF05EFE20463EF08DFF0134402CDCD1CA
:10EE5000064900220023C1E90023C7E90023C6E9CF
:10EE60000023F8BD200B0120300B0120400B0120B6
:10EE70002DE9F04F89B0079000296BD0444BDFF8A3
:10EE8000249118685B680293D9E90087414B424D91
:10EE90000190043A002602EB810C19685B6803912B
:10EEA0000493B34605964FF0FF314FF0010E0696DE
:10EEB000009701E0944530D052F8043F9807F9D10B
:10EEC0001868A842F6D159681E7A0979A1F1200084
:10EED000C1F12004002E40D0009F05962EFA04FABE
:10EEE0000EFA00F646EA0A0637430EFA01F60097D4
:10EEF00046EA08085B7A0EFA00F0002BDAD0069397
:10EF00002EFA04F4049B20430343039804930EFA5F
:10EF100001F3184394450390CED1059B069E009FB4
:10EF20000BB1C9E90087BBF1000F04D0184B019A5F
:10EF30001A60029A5A6026B1164B039A1A60049A14
:10EF40005A60013106D0079BE3B11449144A0023EB
:10EF50000B60137009B0BDE8F08FA1F12000C1F182
:10EF60002004029F0EFA00F62EFA04FA46EA0A0678
:10EF700037430297019F0EFA01F6374301974FF08E
:10EF8000010BB7E709B0BDE8F04F17F085B800BF37
:10EF9000300B0120400B012008C50900405701201B
:10EFA000E95D0120200B0120054B1B78012B01D0CE
:10EFB00000207047034B1878FF3818BF01207047B6
:10EFC000205F0120215F012008B500F009F8FFF75C
:10EFD00017FF00F0C1F9BDE8084000F0FBB900BF21
:10EFE00038B5174C174D236823F47F0323F47F4370
:10EFF000AB4223D04FF480720021201D26F054FF35
:10F000004FF080434FF440320021C3F8042984F8C4
:10F010000411C3F8142984F805114FF47C11C3F8C6
:10F020002429C3F83429C3F84429C3F85429C3F860
:10F030006429C3F87429C3F88419256038BD00BF5A
:10F040001C5E0120AF0000ADF0B5144687B0002A69
:10F0500070D011F0030706460D4603D1464B0A68EF
:10F060009A422FD03046376808F0C0F82A46014649
:10F07000002338462BF07AFC042C054615D0204698
:10F080002EF06AFA4223FF220021044627F08EFD6B
:10F09000012303AA294630468DF80C4008F0AAF84F
:10F0A000002844D00E2007B0F0BD014601233046B1
:10F0B00003AA08F089F89DF80C00400040F0010018
:10F0C00007B0F0BD08F092F829466A4633F0AAFB73
:10F0D000002847D0042C32D0DDE90035ED1AA30713
:10F0E0002AD12368254A934208D0254A934205D065
:10F0F000244A934202D0244A93421DD1012203A9FB
:10F1000020462BF029FC049BAB4231D19DF8141012
:10F11000039C0022402027F0F7FD012825D100990B
:10F120002B462246304608F065F80028BAD1174829
:10F1300032F0DAFD1046B6E7154832F089FDDDE918
:10F140000034E41A3946204626F052FA0099054662
:10F1500002462346304608F037F8294620462FF06D
:10F1600065FBA0E70B4832F073FD0B4832F0E4FD7D
:10F170000A4832F0E1FD00BF68570900B4410900B8
:10F180002C42090068420900F0570900E87509009F
:10F1900010790900C4860900488D090048720900E9
:10F1A00010B50446084608F021F8042C09D0052CB7
:10F1B00005D1074B03EA400040F0010010BD0020DC
:10F1C00010BD80B2002814BF3E201E2010BD00BF1D
:10F1D000FEFF010090B130B4094C0246043900230F
:10F1E00051F8040F850703F1010302D10568A54218
:10F1F00002D09A42F4D10E2030BC70470E207047E6
:10F2000084C5090038B5084BD3E9004554EA050325
:10F2100005D011F0ADFE201A65EB010138BD4FF0AD
:10F22000FF30014638BD00BF480B012070B52DED01
:10F23000028B8AB00D46082000211646039326F063
:10F24000D7F9324B036005AB0193314B039A00931E
:10F25000044602232846314627F06AFCDDE905050D
:10F26000B0F10E0218BF0122B5F10E0318BF012341
:10F270009A4245D00E2840D02EF018F9B0EE408AC0
:10F2800011F076FEF8F7A6F9DFED227A07EE100A04
:10F290000E2DC7EE278A21D006982EF0D5FE054602
:10F2A00048F09AFE07A94EF01FF99DF822109DF82C
:10F2B00021209DF82030BDF81C00CDE900219DF8EB
:10F2C0001F209DF81E1051F0A3F9134B281A034478
:10F2D00007EE903AB8EEE78A38EE288AB4EEE88A6C
:10F2E000F1EE10FA0FD42046B0EE480A07F096FF70
:10F2F00020460AB0BDEC028B70BD9FED088ABFE7C7
:10F30000074832F019FD074832F016FD84C50900A0
:10F31000A0C5090000007A4480BC92C7000000002C
:10F320009C7209009874090008B507F07BFF10EE85
:10F33000103A23F0030040F00200A0F1FF4008BDA6
:10F34000704700BF0248034A0260002343607047D1
:10F35000A847012084C5090008B5012045F060F8E0
:10F36000024B00200021C3E9000108BD480B012029
:10F37000034B1878A0F10200B0FA80F04009704702
:10F38000205F012070B586B00D460820002116468A
:10F39000039326F02DF90B4B036005AB01930A4B49
:10F3A000039A0093044631460123284627F0C0FB08
:10F3B000059856F04BFB0146204607F037FF2046E4
:10F3C00006B070BDE0C50900FCC509004068704783
:10F3D0000E207047704700BF704700BF0020704785
:10F3E00008B5054B1B6813B1044A934201D102488A
:10F3F00008BD034832F078FCC0090120E853090039
:10F40000C074090008B5064BD3F8C03013B1054AE3
:10F41000934201D1024808BD034832F065FC00BFA9
:10F42000C0090120E8530900D074090010B500F0AC
:10F4300009F8044628B1002000F0D8F808B10834D3
:10F44000046010BD2DE9F0473C4F3B6804460E4672
:10F450009046002B48D0DFF8EC905D68D9F80000AA
:10F46000083325F003051D44002846D0621C04BF64
:10F47000441B083CCCB1A30717D19EB93B6844F0AC
:10F48000010C13B915E01B689BB15A686245FAD1AB
:10F490005C60B8F1000F02D044F002045C601846D2
:10F4A000BDE8F087D9F80030E9E700231846BDE849
:10F4B000F08704F1080A431B53450BDA06B33B6897
:10F4C00044F0010113B923E01B680BB35A68914261
:10F4D000FAD1DDE7BEB12AF00303C31AD9F8002040
:10F4E0001A60C9F80030D3E744F0D0FFDFF8549039
:10F4F0000546D9F800000028B8D144F0CBFFB5E7A5
:10F50000D9F80030DCE73B682B602B463D60BFE755
:10F51000B8F1000FC9D021F0C5F80028C5D00121ED
:10F52000504626F089F803460028BED0044AD2F897
:10F5300000110160C2F800014460ADE7FC4F0120FA
:10F54000E4530120F04F0120002211464FF0FF301C
:10F55000FFF76CBF70B58AB044F096FF78B145F004
:10F5600045F81D4C206045F045F823681B491C4AAE
:10F57000C01A086010601B4A1A600AB070BD0446C9
:10F580006846F7F73DFD184E054645F033F83368F9
:10F59000451B03F58060224628440121FFF746FF02
:10F5A00070B10F4B32681A600B4C0368236021F076
:10F5B00015FE0A4A236810600A4A1A600AB070BD34
:10F5C0000246012105F5C840FFF730FF044B4FF418
:10F5D000C0421A60E8E700BF84570120805701202D
:10F5E000004D0120EF2978016003012000B50E4B8A
:10F5F0001968B9B10D4B002808BF19460B1F01F15E
:10F600003C0CC1F1040101EB030E53F8042F8242BC
:10F6100004D06345F7D100205DF804FB0348704433
:10F620005DF804FB0149E9E708570120B4470120D0
:10F630000D4A01230021C2F8003582B0C2F8101132
:10F64000D2F8101100910099D360D2F81031002B3C
:10F65000FBD00023C2F81031D2F8101101910199AA
:10F66000C2F8003502B070470070004008B5086865
:10F6700007F006FE0E2008BD08B507F001FE0E20BB
:10F6800008BD00BF38B51C46084611464FF00212AF
:10F6900027F0A6F9206807F083FE00210546082020
:10F6A00025F0A6FF034B03600446294607F0CCFD76
:10F6B000204638BD70C6090010B5044607F0FCFDB1
:10F6C00090B9204607F0FEFDB5EEC00AF1EE10FA43
:10F6D00008D910EE103A23F0030040F00200A0F128
:10F6E000FF4010BD0E2010BD46F0CEFDE9E700BF83
:10F6F00010B5044607F0E0FD30B9204607F0E8FDFC
:10F70000400040F0010010BD46F0BEFD204607F06D
:10F71000DFFD400040F0010010BD00BF08B50868E3
:10F7200007F048FE0E2008BD08B507F043FE0E2086
:10F7300008BD00BF38B51C46084611464FF00212FE
:10F7400027F04EF9206856F081F900210546042083
:10F7500025F04EFF034B03600446294607F022FEC6
:10F76000204638BDE8C6090038B504460D4607F006
:10F7700023FE70B928462DF0EFFEA2234FF6FF724C
:10F78000002127F013FA81B2204607F017FE0E2061
:10F7900038BD46F079FDEDE701B97047F0B511F0DD
:10F7A000030683B01D4603D14F68FBB2934204D0D9
:10F7B0002B4603B0BDE8F04018473F0A08D00C1DA7
:10F7C000019054F8041F0136A847B7420198F7D1B9
:10F7D00003B0F0BD2DE9F04F2DED088B91B00BABD0
:10F7E000814C01930094052327F034F900210B98F4
:10F7F0003BF090F8002183460C983BF08BF80546CF
:10F8000000210D983BF086F8EB790390012B40F036
:10F81000E780C379012B40F0E380A968012940F219
:10F82000DF808368012B40F2DB80994240F0D88072
:10F830006621DBF808003DF05DF9EC692979079055
:10F8400020463BF05BF9AB68A8692979013B00FBD6
:10F850000340F0EE408A3BF051F90E98039B0E28CE
:10F86000DC69F0EE409A00F0A0802DF01FFE0F98AA
:10F870000E28B0EE409A00F0A2802DF017FEF0EEB8
:10F8800040AA039AEB69D26906930592DBF8083027
:10F89000079ADBF81C60D76953B34FF0000809E002
:10F8A00087ED009ADBF8083008F10108434507F1BD
:10F8B00004071DD930469BF804103BF01FF9DBF814
:10F8C0001830F4EEC08AF1EE10FAB0EE408A1E4411
:10F8D000E6DCF4EEC09AF1EE10FA0FD5C7ED00AAFF
:10F8E000DBF8083008F10108434507F10407E1D8C7
:10F8F000079811B0BDEC088BBDE8F08FAC68013CF7
:10F90000012C69D908962E46069D0997A2464FF00C
:10F9100000096408B069317904EB090700FB07505E
:10F920003BF0ECF8B4EEC08AF1EE10FA86BFAAEB19
:10F930000704B946BA46012CEBD83546DDE908671D
:10F94000CDF810A0069CA869297900FB09403BF07E
:10F95000D5F8049BA869297900FB0340F0EE40BA72
:10F960003BF0CCF8039C0599A06900FB09102179B4
:10F97000B0EE40AA3BF0C2F8DDE90421A06900FB2B
:10F9800002102179B0EE40BA3BF0B8F838EE6B8A3D
:10F9900030EE4B0A3AEE6BAA28EE008A88EE0A0A8D
:10F9A00030EE0BBA87ED00BA7CE7204619793BF0C0
:10F9B000A5F80F980E28B0EE409A7FF45EAF039B37
:10F9C00098681A469B691179013803FB00403BF0A7
:10F9D00095F8F0EE40AA54E704944FF00009B1E71F
:10F9E000024832F0A9F900BF98210A00CC81090031
:10F9F0002DE9F0472DED048B86B003AB574C0193F6
:10FA00000094032327F026F8039800213AF082FFA0
:10FA10008368012B6FD9C579012D044640F09A8087
:10FA200000793BF009F8049BE6690E2B804668D00C
:10FA3000002118463AF06EFFC579012D824640F04C
:10FA40008680A26883689A4240F081800079DFED69
:10FA5000448A3AF0F1FF81463046DAF81C70C0471C
:10FA6000A36938461E44B0EE409AC847DAF8183009
:10FA70001F44A368012BF0EE409A28D93046C047B6
:10FA8000A3693846B0EE498A1E44B0EE409AC84792
:10FA9000B0EE697A39EE088A30EE477AB0EE686ADD
:10FAA00007EE905A97EE086AA368DAF81820F8EE85
:10FAB000676A0135C6EE267AAB421744F0EE409AEB
:10FAC00078EEA78ADAD8F6EE007A68EEA78A013BCC
:10FAD00007EE903AF8EE677A67EEA87A17EE900A8A
:10FAE00020F0030040F00200A0F1FF4006B0BDECA2
:10FAF000048BBDE8F0871B4806B0BDEC048BBDE865
:10FB0000F08705989FED169A2DF0D0FC3046F0EE68
:10FB1000408AC047A368012B16D92A462179E0699B
:10FB2000B0EE408A3AF0A6FF07EE905A30EE088A0F
:10FB3000B8EE677A38EE498AA368C8EE077A0135CD
:10FB4000AB4239EE279AE8D868EE898ABBE70648C7
:10FB500032F0F2F8054832F0EFF800BF80210A00D9
:10FB60000000000002008080F48A0900088B090070
:10FB70001E280ED03E280CD010F001030AD18207B7
:10FB800008D1036804481B1AB3FA83F35B091846CB
:10FB900070470123184670473C4E090008B50146DE
:10FBA000FFF7E6FF18B901F00303022B00D008BDF0
:10FBB00002480840063818BF012008BD070080FF32
:10FBC00070B5426832F0FF0582B004460B460ED095
:10FBD000D4E90221207927F045FDD4E901320E2035
:10FBE0000132A3F58073C4E9013202B070BD2A4628
:10FBF00001910179402027F087F8A16862680831F7
:10FC0000064600FB01F1082060F31F226260E068F5
:10FC100025F024FD6268E0602946C2F31722A5683A
:10FC2000013A06FB02F205FB0666304426F03CF979
:10FC3000019BCDE72DE9F04106468CB00C461546F8
:10FC4000242820D8DFE800F024242424241F1F1FA8
:10FC50001F1F1F1F1F1F851F131F1F1F1F1F1F1F5A
:10FC60001F1F1F591F131F1F1F1F1F1F910012F05F
:10FC7000010040F08B8012F0030104D17F4B126829
:10FC80009A4200F08380002420460CB0BDE8F08149
:10FC9000012206A9204600F0B1F9012209A928464F
:10FCA0002AF046FE00286CD0089A012A00F0BD8098
:10FCB0005A2A40F3A68000210B9B012B00F0B8804C
:10FCC0005A2B00F3B7802033934240F0908023F00A
:10FCD0000203642B00F08B80022E02D0002800F07B
:10FCE0008680DDE90930DDE906120090304632F009
:10FCF000C5FC002845D03E24C6E706A901222046BF
:10FD000000F07CF909A9284601222AF025FE9DF879
:10FD100020100022402026F0F7FFA1680A9E054629
:10FD20009DF82000B6FBF5F6314400F0DFF90446FB
:10FD3000DDE90612C06826F007F8E068079B09991C
:10FD400006FB05F2184425F0FFFF20460CB0BDE885
:10FD5000F0814B4B0A689A4295D02946204600F024
:10FD600015F920460CB0BDE8F081012203A9284610
:10FD70002AF0DEFD90B3A20703D1424B22689A42DB
:10FD800042D01E2420460CB0BDE8F08128462DF05C
:10FD9000E3FB012209A90746204600F02FF9102EA7
:10FDA000DDF8288048D0A1689DF82C0007FB01F100
:10FDB00000F09CF9C5680446B8F1000F3FF464AF49
:10FDC0007E1E002F3FF460AF099928464246013E4F
:10FDD00025F0BAFF711C4544F6D155E7EB0706D470
:10FDE00015F0030306D1254B2A689A42C9D1002099
:10FDF00031F02EFF022BC4D1234B2B40062BF6D122
:10FE0000BFE72032014657E7012209A92046012415
:10FE100000F0F4F8DDE90323DDE9090100941FF0A7
:10FE20000BF900287FF467AFABE76222014643E796
:10FE3000622349E7084647E721790022402026F05F
:10FE400063FFA36807FB03F300FB03F1E06825F001
:10FE500005FCA36807FB03F3C4E9023063686FF392
:10FE60001F2305466360002F3FF40EAF013F45445A
:10FE7000B8F1000F3FF408AFA2E700BF3C4E090005
:10FE8000684209002C420900070080FF2DE9F0417B
:10FE9000012884B080460C4633D08B072AD02046F8
:10FEA0002EF050FB00284CD045102946404600F06B
:10FEB0001DF90021064620462AF0AEFD0024074623
:10FEC00038462AF0E9FF48B165B901463046FFF7E8
:10FED00077FE38462AF0E0FF0028F5D1304604B01E
:10FEE000BDE8F08122460346F168404627F0BAFBA0
:10FEF0000134E5E70B68154A934202D0144A934255
:10FF0000CDD1012201A920462AF012FD0028C6D039
:10FF100041460022402026F0F7FE029BB3FBF0F1A1
:10FF200000FB01F4A3420ED1404600F0DFF8019936
:10FF300006462246C06825F007FF304604B0BDE8FB
:10FF4000F0810546B1E7034831F0F6FEF0570900AD
:10FF50002C420900247A090000B5012883B00B4621
:10FF600008D0844600226146074830F0B3F903B058
:10FF70005DF804FB0A6840F61623CDE900234FF034
:10FF8000020C6B46EEE700BF545A090070B50446F8
:10FF900084B00846012201A92AF0DEFC0022217962
:10FFA000402026F0B1FE6368029DB5FBF0F5B5EB8D
:10FFB000132F0646C3F3172212D8521B62F31F23D6
:10FFC000E0686360A368019903FB060005FB06F285
:10FFD00025F0BAFEA3680E202B44A36004B070BDC8
:10FFE000D4E90210294406FB01F125F037FB6368D0
:10FFF000E0606FF31F236360E4E700BFF8B50379A7
:020000023000CC
:1000000004460D46164603F07F010022402026F0EC
:100010007BFEE7682F60A1680E4A00FB01F1696072
:10002000217901F07F01A9602168914201D000206F
:10003000F8BD94F90420002A034603DBB20701D57A
:100040000120F8BD6268C2F3172203FB02732B6024
:100050000020F8BD6842090010B44268C468916885
:100060008C420CD20346D16810799A68224401343C
:10007000DC605DF8044B00F07F0026F0C1BF00207B
:100080005DF8044B704700BF084A0023C1E9023302
:10009000C1E90020064B02689A4201D00846704729
:1000A0004368C3F317238B6008467047F04109008B
:1000B0006842090038B50C461D46114620460A4ADA
:1000C00026F08EFC286830F0DBF8012C05D069683A
:1000D0000078BDE83840FFF7D9BEBDE83840007869
:1000E000002100F003B800BF040002007828F8B532
:1000F00020D005460E4600220146402026F004FE90
:1001000000210746102025F073FA04460571866029
:1001100062680A4B6FF31F226260094A012D18BF03
:10012000134606FB07F00021236025F061FAE0602A
:100130002046F8BD034831F0FFFD00BF2C42090006
:10014000B4410900B0790900F8B50D79012D0C46CC
:10015000064632D020492A4631F0A0FCA3682BB9CC
:1001600030461E49BDE8F84031F02CBC1C493046F1
:1001700031F028FCA368B3B11A4F00252A46E16884
:10018000207926F03DFF0122014630462FF0A6F8E7
:10019000A3680135AB4206D9002DEFD03946304671
:1001A00031F010FCEAE71049304631F00BFC3046E4
:1001B0000A49BDE8F84031F005BC0C4931F002FCB9
:1001C000D4E9022130462B4632F0FCFF3046034989
:1001D000BDE8F84031F0F6BBC04009000855090001
:1001E000CC400900D4400900D0400900B4400900C7
:1001F0002DE9F04387B0002A37D011F003060446FA
:100200008C46154603D1874B0A689A4232D0A168C2
:100210002068002362462AF0A9FB834B216899429B
:1002200002460ED0042D11D094F804C0E1682B468C
:100230000CF07F0027F016FA0E24204607B0BDE828
:10024000F0836368042D00EB132208D12079E16864
:1002500000F07F0007B0BDE8F04326F0D1BE94F96E
:10026000043094F804C0002BE0DB0024204607B0E3
:10027000BDE8F08380686A4632F0D4FA002800F0C6
:10028000CA802179042D324601F07F014FF04000F1
:100290006DD026F039FD15F00307064602D06348FD
:1002A00031F0D6FC286833F0DFF8614B834200F070
:1002B0009C80604B2A689A42F1D1012E40F0AE80BA
:1002C000324603A928462AF047FBDDE90398564A3F
:1002D0002368E768DDE900019342A1EB0005A8EB84
:1002E000050524D0002D2DDD6368B5EB132F58D8FC
:1002F000A36840442B441A1A06FB017106FB02F264
:1003000006FB007025F050FD009806FB08F24946F8
:1003100000FB067025F048FD6368C5EB132262F30D
:100320001F23A26863602A44A2600E2485E794F923
:100330000430002B99DA002D70D16368C3F31723C2
:1003400006FB0377494606FB08F206FB007025F022
:100350002BFD0199A2680098521A404406FB02F254
:1003600006FB017106FB007025F01EFDD4E726F0A8
:10037000CBFC2D4B22689A42054622D0DDE90031A4
:100380002079C91AFFF7B2FEDDE90013E6685B1AAF
:10039000044605FB03F205FB0161C06825F0D4FCAF
:1003A0004BE7A1682944384606FB01F125F056F9D0
:1003B0006368E06065F31F2363600746DDE90001C1
:1003C00096E73146102025F013F9054694E80F0012
:1003D00085E80F00009A02EB112060F31F2169608D
:1003E000019B9B1A2C46AB6027E729793A4601F01E
:1003F0007F01402026F088FCB0420FD10A4A2B68CA
:100400009342D5E902897FF463AF6B68C3F3172386
:1004100006FB03995CE7084831F01AFC074831F005
:100420008BFC00BF68570900684209001079090079
:10043000F1010300F0570900C48609004C8309004C
:10044000042808D0052804D18868400040F0010045
:100450007047002070478B68002B14BF3E201E2081
:10046000704700BF10B510EE104A24F00043B3F1FE
:100470007E5F2DED028B0BD319D070EE407ADFED4D
:100480003F6A86EEA77ABDEC028BB0EE470A10BD3C
:10049000B3F17C5F35D2A3F50003B3F1645F11D2F1
:1004A000BDEC028BB0EE407AB0EE470A10BDDFED36
:1004B000347A9FED347ABDEC028BA0EE277AB0EE51
:1004C000470A10BD60EE007A9FED2F7A9FED2F6AEC
:1004D000DFED2F6ADFED2F5AA7EE876ABDEC028BA6
:1004E000E7EE866AB7EE007AA7EEA57A67EEA67AFF
:1004F000C7EE876AB0EE407AA0EE267AB0EE470AE1
:1005000010BDB7EE008AB0EEC00A38EE400AB6EE73
:10051000008A20EE088AB5EE408AF1EE10FA26D461
:10052000F1EEC87A002CDFED186A9FED187A9FED86
:10053000186ADFED185A9FED120AA8EE267AF7EE38
:10054000006AA8EE076AE8EE256A28EE068A9FEDA3
:10055000127A88EE266AF0EE005AE6EE277AA7EEC7
:10056000A57A30EE477A8EDAB1EE477A8BE7B0EEB5
:10057000480A4AF093FEF0EE407AD3E7000000000C
:10058000DA0FC93F000080036BD30DBCBA132FBD37
:1005900075AA2A3EAEE534BF6821A2B310B52DED91
:1005A000028B84B08DED010A019B23F00042B2F171
:1005B0008B4F08EE102A4FEAD3742ED25B0012D470
:1005C000B2F1665F32D2DFED2B7A78EE277ACDED8D
:1005D000037A039B0CB1B1EE488AB0EE480A04B02E
:1005E000BDEC028B10BDB7EE000AA8EE080A78EE4B
:1005F000088AB5EE400AF1EE10FA36D4F1EEC07A70
:1006000038EE278AF7EE007A87EE880A30EE280A5D
:1006100024F0F4FEB0EE408ADCE700EE102A24F06D
:10062000EDFE9FED158A30EE088AD3E768EE088A62
:10063000B7EE000A38EE800AB5EE400AF1EE10FA85
:100640000ED4F1EEC07AB7EE007A77EE877A88EEB4
:10065000A70A30EE080A24F019FEB0EE408AB9E786
:100660004AF01CFEF0EE407AEDE74AF017FEF0EE9D
:10067000407AC5E70000807B1872313F08B5054B12
:100680001B6833B1044A1B68934202D0042047F030
:1006900067F808BD84570120EF29780148B110B5EB
:1006A0000E2884B0044602D00EF0AAF810B104B0AF
:1006B00010BD7047204601A94FF4EB7403AB02AAAA
:1006C000039420F00DFE0399014831F03DFB00BF7B
:1006D0004C6A0900F4EE400AF1EE10FAF0EE407AAE
:1006E00053D610EE902AB2F17E5F10EE103A47D04A
:1006F00010B5940F04F0020444EAD37433F00043BD
:1007000008D1022C3ED09FED380A032C18BFB0EE62
:10071000670A10BD32F0004228D0B2F1FF4F1BD063
:1007200002F15061994221D3B3F1FF4F1ED0A107CE
:100730002ED503F15063934243D29FED2C0A022C35
:1007400046D0002CE5D09FED2A7ADFED2A7A30EEF4
:10075000070A30EE670A10BDB3F1FF4F04F1FF3412
:1007600027D0022C1FD99FED210A10BDDFED227A80
:100770009FED220A14F0010F18BFB0EE670A10BDFA
:1007800000F044B89FED1B0A10BD30EE800A7047A0
:1007900087EEA00AB0EEC00A00F038F8012CCED1E6
:1007A000B1EE400A10BD164B03EB840494ED000A31
:1007B00010BD022C15D8134B03EB840494ED000AF2
:1007C00010BD87EEA00AB0EEC00A00F01FF8B6E731
:1007D0009FED077ADFED077A30EE070A37EEC00AA1
:1007E00010BD9FED090A10BDDB0F49C000000000DD
:1007F0002EBDBB33DB0F4940DB0FC9BFDB0FC93F49
:100800007C170A0070170A00DB0F493F10EE102A10
:1008100022F00043B3F1994F4FEAD2710DD3B4EEF9
:10082000400AF1EE10FA11D6DFED4B7A9FED4B0A3C
:10083000002908BFB0EE670A70474948834206D8CE
:10084000B3F1665F39D212F0FF4F7DD07047454A51
:100850009342B0EEC00A4BD9434A93426BD8F7EEAD
:10086000087AB7EE006AA0EE276A70EE677A9FED0D
:100870003F7A9FED3F0AC7EE866A66EEA65A9FED65
:100880003D6ADFED3D4A9FED3D4A9FED3D5A65EEE5
:10089000A57AE7EE864AA7EE845A9FED3A6AA7EE5C
:1008A000A46A67EE857AE5EE867A97EEA67A77EE09
:1008B000667A30EE670A71BB704760EE006A9FEDA2
:1008C0002D7ADFED2D5A9FED2D5A9FED2D6A66EEA4
:1008D000A67AE7EE875AA7EE856A9FED2A7AA7EEF9
:1008E000A57A67EE867AE6EE877AA7EEC00A7047A9
:1008F000A2F5D002934211D8F0EE007ABFEE006A62
:10090000A0EE276A70EE277A9FED1F7A9FED1F0AEF
:10091000C6EE276AB1E7B1EE400A7047F7EE007AFB
:1009200030EE676A70EE277A9FED197A9FED190A0B
:10093000C6EE276AA1E7FFEE007AC7EE806A9FED58
:10094000167A9FED050A98E760EE007A82B0CDED49
:10095000017A019B02B07047DA0FC93FDA0FC9BFB5
:10096000FFFFDF3EFFFF973FFFFF1B40B40F143335
:100970005E987B3F25AC7C3D0DF5113E4712DABDFC
:1009800098CA4CBEA9AAAA3E6937AC313863ED3E7D
:1009900068212233DA0F493F6821A23310B584B0B1
:1009A0008DED010A019B23F00042B2F17C5F00EE65
:1009B000102A4FEAD37422D2B2F13E5F0CD213F068
:1009C000FF4F04D160EE007ACDED037A039B0CB1AA
:1009D000B1EE400A04B010BD30EE007AF7EE007AB6
:1009E00077EEC07A67EE006A86EEA70A30EE070A55
:1009F00024F04CFCF6EE007A20EE270AE7E7F7EE4B
:100A0000007A77EEC07A80EE277A37EE070A24F074
:100A10003DFCF6EE007A20EE270AD8E7014B186875
:100A20001FF030BFFC47012010B584460C46BCF1D6
:100A3000010F1346086888BF221D0CF1FF3198BFD3
:100A4000002248F0B3FD206810BD00BF38B5044C4B
:100A5000044B206800251D6024F0C8FD256038BDCA
:100A6000FC4701200448012000B583B0019001A893
:100A700048F00CFE0E2003B05DF804FB08B506F04C
:100A8000E3FC0E2008BD00BF30B589B004AD144CA6
:100A900001950846009411461A46042326F048F8AA
:100AA000049854F0D3FF0546059854F0CFFF024652
:100AB0000698039254F0CAFF0021034628200293AF
:100AC00024F0BEFD2946074D05609DF81C50009599
:100AD000DDE90232044606F073FC204609B030BD61
:100AE00088C7090080C8090008B5086806F0ACFC92
:100AF0000E2008BD10B5044605F036F9204606F074
:100B0000D5FC002814BF3E201E2010BD10B50446A1
:100B100005F02AF9204606F0CFFC002814BF3E203D
:100B20001E2010BD10B5044605F01EF9204606F043
:100B3000C3FC20B1204606F0D3FC0E2010BD0148B6
:100B400031F0D2F81870090070B50C4686B054F830
:100B5000046B03920546304605F006F904AB019399
:100B6000084B039A00932146681E022325F072FF6A
:100B700030469DF81420049906F0BAFC0E2006B009
:100B800070BD00BFA8C7090010B5044605F0ECF819
:100B9000204606F08BFC08B90E2010BD204606F05A
:100BA000ABFD0E2010BD00BF10B5044605F0DCF80B
:100BB000204606F0A9FD0E2010BD00BF08B506F0C6
:100BC000FBFD0E2008BD00BF2DE9704F2DED028BFF
:100BD0008CB005AD2D4C01950846009411461A467F
:100BE000072325F0A5FF059854F030FF80460698AE
:100BF00054F02CFF00218146082024F0F9FC244BFE
:100C000003609DF82050DDF81CA06A073AD19DF8DA
:100C10002860730733D104460B989DF824B040B385
:100C20002CF044FCB5EEC00AF1EE10FAB0EE408AAA
:100C300022D4F7EE007AB4EEE70AF1EE10FA1BDCEC
:100C400053464A4641462046CDE901B6009506F096
:100C50006BFD9FED100A28EE008AFCEEC87A17EEB5
:100C6000900A29F021FF20460CB0BDEC028BBDE8B4
:100C7000708F9FED098AE3E7084831F05DF8084876
:100C800031F05AF8074831F057F800BF9CC8090006
:100C900040C9090000007A44AE47E13D6C6E09008E
:100CA000EC700900C08D090008B5086806F084FDE5
:100CB0000E2008BD10B5044606F092FD30B920465E
:100CC00006F098FD400040F0010010BD45F0DCFA50
:100CD000204606F08FFD400040F0010010BD00BF2F
:100CE00070B584B006460C46154606F079FDC8B9C5
:100CF0004FF46E71284625F0BFFF4FF46E7200214D
:100D0000054625F07BFFA30703D11F4B22689A42BB
:100D100031D0022201A9204629F00AFE28B90E206E
:100D200004B070BD45F0B0FAE2E79DF80C10029CEB
:100D30000022402025F0E8FFB4FBF0F0A8421DD3CC
:100D4000304606F055FD039B482B05D0102818D0DF
:100D5000422B03D0012B01D0082809D001992A4643
:100D6000304606F04BFD400040F0010004B070BD7D
:100D7000064830F0E1FF064830F06AFF054830F0E1
:100D8000DBFF054830F0D8FF10970900047D09000B
:100D90005C8F0900DC6A0900247D090008B506F0B3
:100DA0007DFD0E2008BD00BF10B4019CA4468468E0
:100DB000CCF8004089B1817BB2FBF1FC01FB1C2225
:100DC00090F80CC041685DF8044B4FEADC00D2B2E9
:100DD00002FB00121A600020704742685DF8044B65
:100DE0001A600020704700BF4FF0010C82F800C06D
:100DF000427B1A70009A83681360019B09B190F8D6
:100E00000EC083F800C0704730B58BB0204C009402
:100E100004AD0846019511461A46032325F088FEC5
:100E20000021142024F0E4FB1A4B03600446012245
:100E3000049807A929F090FD099B622B1DD023F08F
:100E40002002A3F16800B0FA80F0482A4FEA50105F
:100E500011D0422B14D0012B14D106999DF81420E7
:100E60000090CDE901212046DDE9071206F008FDDA
:100E700020460BB030BD0223EFE701200346ECE72C
:100E80000123EAE704484FF4227130F05DFF00BF10
:100E90008CC9090024CA09001072090008B5086845
:100EA00006F0FCFC0E2008BD10B5044606F0FAFC66
:100EB00030B9204606F000FD400040F0010010BDB2
:100EC00045F0E2F9204606F0F7FC400040F0010052
:100ED00010BD00BF38B504460D4606F0E3FC40B92E
:100EE00028462CF039FB0146204606F0E7FC0E2090
:100EF00038BD45F0C9F9F3E7704700BF08B506F003
:100F000093FD0E2008BD00BF2DE9F04383B00446D9
:100F10000A9E9846002970D1856B0F46226A636B42
:100F2000C2B9AB426FD0A28B01351544ED1AEB0765
:100F30004FD4E368C8F8003023693360002F4FD1E5
:100F4000A36B0133A363206A003818BF012003B0EC
:100F5000BDE8F083AB42E6D1E36A9A4228BF1A4665
:100F6000A38BD8074CBFE1686168C8F80010206BFC
:100F700001AB083091465BF036FB00284AD1019B5B
:100F8000994547D1226AD21A22628AB913F0030026
:100F90000ED0A17E0344082901933FD0102907D128
:100FA000D8F8001023F00103194421F8022C019B0A
:100FB0003360A28BD1074CBF2361A3600132636B06
:100FC00092B2013501331544ED1A6363EB07A28336
:100FD000AFD56368C8F80030A3683360002FAFD086
:100FE000012FB0D1E26BA17E0132E263D8F800306C
:100FF00003EBD103C8F80030A5E7012A856B08BFD1
:10100000C56B17468AE71046C8F80020326003B067
:10101000BDE8F083022003B0BDE8F0834FF0800EFE
:10102000D8F800106FEA020C0B44013203F80CE010
:101030009042019BF4D1BBE74FF0000C82F800C056
:10104000827E082A94BF002201221A70009A4FF46F
:1010500000731360019B19B190F824201A70704737
:1010600001221A70704700BFF0B51F460E4685B0CA
:1010700011463046274A25F0B3FC3C68264B2340F6
:10108000062B0DD014F003013AD1244B22689A426A
:1010900006D0402024F0ACFA214B036005460FE057
:1010A000214644F296621F4827F014FA00210446B4
:1010B000402024F09DFA1A4B0360A307054625D172
:1010C000194B22689A4221D1012E09D800231E46CD
:1010D00028463246214606F0F3FB284605B0F0BD0F
:1010E0007868022201A929F037FC4FF42273DDE968
:1010F00001604FF48062082125F08CFD0346E7E78C
:101100000021402024F074FA054B0360074830F0BA
:10111000FFFD00BF040002000F0080FF545A0900C9
:1011200020CB090030950900109709004C7E09007A
:1011300008B5086806F078FC0E2008BD10B5044616
:1011400004F01CFE204606F079FC400040F001004F
:1011500010BD00BF10B5044604F010FE204606F096
:101160006FFC400040F0010010BD00BF10B5044608
:1011700004F004FE204606F067FC400040F0010049
:1011800010BD00BF38B50D46044604F0F7FD2846F3
:101190002CF0E2F90146204606F058FC0E2038BD3E
:1011A00038B5044609B1012A0BD0206B636923626C
:1011B0000025228B08302B465AF09CFEC4E90D55C1
:1011C000E56338BD08B506F06FFC0E2008BD00BF12
:1011D0002DE9F04F2DED028B8BB0CDE90623169C47
:1011E000C3690646C9B9F2682260B26906919A429B
:1011F0001CD0737C002B00F0E180079AB368136069
:10120000069B002B40F0C780F3690133F361012096
:101210000BB0BDEC028BBDE8F08F069A012AF26894
:1012200008BF036A2260B2699A42E2D17368727C95
:101230001946B368002A08BF1946079A0891116039
:10124000737C96F8242083F001037374F3689B0881
:101250000593002A00F0A581002306F128010493DC
:1012600003914FF0802B9A46039B53F8044F03934E
:10127000A368002B68D0059B002B63D004F11003FA
:101280006269089F059D08EE103AFAB9637B3BB985
:10129000237B002B00F07681A068114600F044FE0D
:1012A000A068002800F0B780002204F11403009326
:1012B000114618EE103A00F005FE6269A0F1010037
:1012C000B0FA80F040099208607362619542294645
:1012D0002369B4F818E096F810C028BF1146BAF197
:1012E000000F6FD1BCF1100F40F0978096F812C03C
:1012F000BCF1000F00F02881C9B14FEA0E42043B57
:10130000A7F1040ED44653F8040F32FB00F832FB69
:1013100010F028F3CF3820F3CF30C8EA00400CF1AA
:10132000010C61454EF8040FEDD1D4E9043203EB12
:101330008103521A6D1A2361626107EB8107A4D100
:1013400096F824204FF0010A049B01339A4204933B
:101350008ADCBAF1000F00F02481B37CA3B9337C9E
:10136000102B059B00F02C8173B1089B059903EBB2
:101370008102043A043B4FF0803053F8041F81FA95
:1013800040F193421960F8D1B3690133B361069B10
:10139000002B3FF439AF069B012B7FF438AF336A43
:1013A0000799327C013333620B68012003EBD203CF
:1013B0000B600BB0BDEC028BBDE8F08F079A736831
:1013C00013601DE7BCF1100F5BD196F812C0BCF1A1
:1013D000000F00F098800029A9D04FEA0E42043B8C
:1013E000A7F1040E4FF0000C53F8048F32FB08F005
:1013F00032FB18F820F3CF3028F3CF38C0EA08408A
:101400005EF8048F90FA18F00CF1010C6145CEF8EB
:101410000000E9D189E7626958E7480087D04FEAC0
:101420000E42CDF824A0D646023BA7F102088A4618
:10143000814633F8020FB17C4FEA004C00020CF0F9
:101440007F4C80B24CEA000009B990FA4BF032FBB5
:1014500000F132FB10F021F3CF3120F3CF30C1EA9D
:101460000040010C01F47F41C0F307200EF1010E92
:101470000843CE4528F8020FDBD15146DDF824A001
:1014800053E748003FF453AF4FEA0E42CDF824A093
:10149000023BA7F102084FF0000E8A46814633F85E
:1014A000020FB17C4FEA004C00020CF07F4C80B27E
:1014B0004CEA000009B990FA4BF032FB00F132FB24
:1014C00010F021F3CF3120F3CF30C1EA004C38F8CF
:1014D000020F0104000280B201F07F4101439CFA37
:1014E00011FC4FEA1C4101F47F41CCF3072C0EF1B3
:1014F000010E41EA0C0CCE45A8F800C0CFD15146F0
:10150000DDF824A011E700293FF411AF4FEA0E40A7
:10151000043BA7F1040E53F8042F92FA4BF230FB70
:1015200002F830FB12F228F3CF3822F3CF32C8EAA8
:1015300002425EF8048F92FA18F20CF1010C614538
:10154000CEF80020E7D1F0E600293FF4F0AE4FEAF4
:101550000E42043BA7F10408D64653F8040F90FA54
:101560004BF032FB00FC32FB10F02CF3CF3C20F3AD
:10157000CF30CCEA00400EF1010E714548F8040F5F
:10158000EBD1D2E6A260BAF1000F7FF4D9AE002D04
:101590004FEA8502514608BF0422384624F084FCF5
:1015A000CEE6059B002B3FF4D8AE059B08989A0029
:1015B000002124F079FCB37C002B7FF4E5AECEE66D
:1015C000002B3FF4E1AE089A02EB83010439131FAC
:1015D0004FF0802053F8042F92FA40F299421A609B
:1015E000F8D1D1E64FF0000C82F800C0827C1A706E
:1015F000009AC3681360019B11B1C27C1A707047D6
:1016000001221A70704700BF2DE9F0438BB0314CB6
:10161000009404AD0846019511461A46062325F0AC
:1016200087FA40F28353FF220121049825F0BEFA85
:1016300040F29A23022201210746069825F0B6FAC5
:1016400040F2B34204460121099825F0A3FADDF8DF
:101650001C80B8F1080F054602D0B8F1100F35D143
:1016600007F10B000021800023F0C2FF1A4A02603C
:101670009DF820200092E4B2CDE90145059A5FFA79
:1016800088F3F9B2064606F0E3F9002F13DDDFF820
:101690005080D8F80C9006F1280500240023194644
:1016A0001A464046C847013445F8040F314606F053
:1016B0009FFAA742F2D196F8240006F12C012DF0F2
:1016C0003FFCB06230460BB0BDE8F083034830F019
:1016D00033FB00BF8CCB0900ACCC0900C4790900F6
:1016E0009CCD090008B5086806F0DEF90E2008BD9B
:1016F00010B5044604F04CFB204606F0E3F9002840
:1017000014BF3E201E2010BD10B5044604F040FB5F
:10171000204606F0EFF9400040F0010010BD00BF88
:1017200010B5044604F034FBA06A10BD70B50C4639
:1017300088B054F8045B03920646284604F028FB60
:1017400005AB01930E4B039A009321460323701EB1
:1017500025F080F995F824209DF818309A420AD98E
:1017600005EB83059DF81C20E86A059906F0D6F97B
:101770000E2008B070BD40F2825025F05DF900BF28
:10178000C4CB090070B50C4686B054F8045B0392D4
:101790000646284604F0FCFA05AB01930C4B039A6D
:1017A000009321460123701E25F054F995F824205A
:1017B0009DF814309A4207D905EB8305E86A06F0D4
:1017C00019FA0E2006B070BD40F2825025F034F9AF
:1017D000BCCB090038B590F824306BB10024054625
:1017E000234605EB83030134D86A06F003FA95F823
:1017F0002420E3B29A42F4D838BD00BF10B50846A1
:101800001146002225F0ECF800211C2023F0F0FE08
:10181000034B0360044606F06FF9204610BD00BF7D
:101820009CCD090008B506F06DF910EE103A23F0D2
:10183000030040F00200A0F1FF4008BD08B506F02B
:1018400067F9002814BF3E201E2008BD10B584B0E3
:1018500002AB51F8044B0193074B0093013802236C
:1018600025F0F8F820469DF80C20029906F056F96C
:101870000E2004B010BD00BF08CD090010B584B023
:1018800003AB01930F4B51F8044B00930138012334
:1018900025F0E0F803982BF009FEB7EE007AB4EEDD
:1018A000C70AF1EE10FA0ADCB5EEC00AF1EE10FA42
:1018B00005D4204606F090F90E2004B010BD024871
:1018C00030F03AFAF8CC09003C83090010B584B036
:1018D00003AB51F8044B0193054B009301380123EE
:1018E00025F0B8F8204606F085F90E2004B010BDAA
:1018F00000CD090008B506F0CDF90E2008BD00BFE7
:1019000070B5044684B08069089D00286DD039B355
:10191000206B286094F93F001146884227D094F844
:101920003C10B1FA81F14909C2F1010284F83F206B
:1019300004EB810284F83C1084F84010566A1E6063
:10194000204624F0B9FF204624F096FF10BB286003
:1019500094F83E30002B14BF0020022004B070BD6C
:10196000206B286094F93F0088420A46D7D194F949
:10197000401004EB81010120496A01EB4202FF2182
:101980001A6084F83F102A68636C03EB52036364A7
:1019900004B070BDD4E90710A26933460026091AC5
:1019A0000244009602910392606802AA03A9F7F725
:1019B00045F9E369029A9B1A236218B130462E60FA
:1019C00004B070BD2A68636C03EB52036364204665
:1019D00024F072FF204624F04FFF236AB3F5007F06
:1019E000054606D2284604B070BD2860022004B027
:1019F00070BD04F108000349224600F04BFB284665
:101A0000F1E700BFCD6905004FF0000C10B482F87B
:101A100000C001221A70019C036B2360029B09B174
:101A200090F83D201A705DF8044B7047F0B51F46E2
:101A30000E4685B011463046254A24F0D1FF3C6859
:101A4000244B2340062B0DD014F0030137D1224B39
:101A500022689A4206D0482023F0CAFD1F4B03603B
:101A600005460FE0214644F296621D4826F032FDFD
:101A700000210446482023F0BBFD184B0360A30758
:101A8000054622D1174B22689A421ED1012E08D852
:101A9000002328461A46214606F0B0F8284605B02D
:101AA000F0BD786801A9022228F056FF2846DDE93A
:101AB0000123214606F0A2F8284605B0F0BD00211A
:101AC000482023F095FD054B0360074830F020F9CE
:101AD000040002000F0080FF545A090018CF0900CB
:101AE00030950900109709004C7E090008B5086878
:101AF00006F0D0F80E2008BD10B5044604F052F9E7
:101B0000204606F0DBF8400040F0010010BD00BFA9
:101B100010B5044604F046F9204606F0D1F840001E
:101B200040F0010010BD00BF10B5044604F03AF9C2
:101B3000A06B10BD10B5044604F034F9204606F041
:101B4000C3F810EE103A23F0030040F00200A0F1B9
:101B5000FF4010BD10B5044604F024F9204606F0FD
:101B6000F1F8400040F0010010BD00BF10B5044680
:101B700004F018F9204606F0E7F8400040F00100B4
:101B800010BD00BF10B582B00446019104F00AF9FF
:101B90000199064844F2966226F09CFC01462046D4
:101BA00006F0D4F80E2002B010BD00BF3095090039
:101BB00038B50C46054604F0F5F8A30709D1064BE5
:101BC00022689A4205D12846214606F0BFF80E2029
:101BD00038BD024830F09CF8109709004C7E09008F
:101BE00038B50D46044604F0DDF828462BF0B4FC69
:101BF0000146204606F0FCF80E2038BD10B504461C
:101C000009B1012A1BD000F075FAA06B0022002355
:101C100008305AF06FF9E169216200224FF47F43E6
:101C20006264E387204624F0D3FE204624F044FE7D
:101C3000204624F021FEBDE8104000F05DBA10BD42
:101C400008B506F011F90E2008BD00BF30B589B007
:101C500005AD114C01950846009411461A46032320
:101C600024F066FF059853F0F1FE0546069853F000
:101C7000F5FE002102462420039223F0B9FC074B15
:101C80000360BDF81C30039A2946044606F0B2F8FA
:101C9000204609B030BD00BF7CCF090064D00900E8
:101CA00008B5086806F0E0F80E2008BD10B5044637
:101CB00004F082F8204606F007F9002814BF3E2001
:101CC0001E2010BD10B5044604F076F8204606F03C
:101CD000FDF8002814BF3E201E2010BD10B504469C
:101CE00004F06AF8204606F0F1F820B1204606F02C
:101CF000F9F80E2010BD01482FF0F6FF187009000A
:101D000070B50C4686B054F8046B03920546304615
:101D100004F052F804AB0193084B039A0093214658
:101D2000681E022324F096FE30469DF81420049984
:101D300006F0E0F80E2006B070BD00BF94CF090099
:101D400010B5044604F038F8204606F0BDF808B98E
:101D50000E2010BD204606F08BF90E2010BD00BFEE
:101D600010B5044604F028F8204606F091F90E203C
:101D700010BD00BF3A4BD3F80021D00052D52DE959
:101D8000F047384DDFF8D88005F1100601274FF0F5
:101D9000000955F8044BA4B1E37F33B9A268D2F827
:101DA000041111B16377C2F80431637F4BB1A37F93
:101DB0005BB1A368D3F8102132B3D3F814215AB31E
:101DC0005F60B542E5D1BDE8F087E37F002BF8D135
:101DD00094F822A0BAF1000FF3D1A368D3F8082138
:101DE000002A34D1D3F80C314BBB94F91C30002BB2
:101DF000E7DB5A09603203F01F0307FA03F3B54229
:101E000048F82230C5D1DEE7D3F80821002AD8D11E
:101E1000D3F81421002AD3D1D3F80C21002AD0D131
:101E20005F60CEE7D3F804219107A8D4D3F804214A
:101E30005207A4D4D3F804319B04A0D470470021E6
:101E400020461CF0FFFEA368C3F80C91CDE70121EA
:101E500020461CF0F7FEA368C3F808A1A368C1E7F9
:101E600000E100E09847012070B5074C002604F11E
:101E7000100554F8043B0BB14CF030FAAC4244F876
:101E8000046CF6D170BD00BF9847012010B5014623
:101E900004464FF48A602FF01DFE034620469B68DF
:101EA000BDE81040184700BF10B5014604464FF486
:101EB0008A602FF00FFE03462046DB68BDE8104025
:101EC000184700BF70B582B004460D4601464FF476
:101ED0008A60069ECDE900322FF0FCFD0696466929
:101EE000DDE9003229462046B44602B0BDE8704024
:101EF000604700BFF0B583B00446089E099F0D46B9
:101F000001464FF48A60CDE900322FF0E3FDCDE9C0
:101F10000867DDE90032866929462046B44603B0E9
:101F2000BDE8F040604700BF30B5044683B00D46C1
:101F30004FF48A60214601922FF0CCFD019A03698B
:101F40002946204603B0BDE83040184710B5014689
:101F500004464FF48A602FF0BDFD034620465B68BF
:101F6000BDE81040184700BF38B511B90025284614
:101F700038BD044604F016FE05460028F6D020467B
:101F8000002104F00BFF284638BD00BF10B5044601
:101F90000121406804F002FF6068BDE8104005F0D0
:101FA00009B800BF014B00221A707047D95D0120AB
:101FB0000349044B0120002208701A60704700BFDB
:101FC000D95D0120F84F0120014B1878704700BF00
:101FD000D95D0120024B1868003818BF01207047F6
:101FE000F84F012010B50C4C206818B10B4B1B6842
:101FF0000BB1002010BD4DF0C5FA23688342236861
:102000008ABFDB43C01AC01840F2EE23984294BF47
:102010000020012010BD00BFF84F0120F44701202F
:10202000014B00221A607047F84F0120024A1368E2
:1020300023EA000010607047F4470120024A136849
:1020400018431060704700BFF447012008B50D4BDE
:102050001B6813B90C4B1B7803B908BD4DF092FAFD
:102060000A4B18601A6812B91A6801321A60012006
:102070004CF060FE064B03F16C025A62BDE808406A
:1020800042F0BEBAF4470120D95D0120F84F01208B
:10209000E4530120C0E9001200F000B810B5044676
:1020A0000CF034FBE368A3B910490A68A24210D0CF
:1020B0000F4AA36010681368E0600BB113689C605E
:1020C0000B6853B114600CF05BFBBDE8104042F0AC
:1020D00097BABDE810400CF053BB0C6014600CF0D4
:1020E0004FFBBDE8104042F08BBA00BF0048012012
:1020F000084801200CF00ABB0CF042BB10B5054BA0
:102100001C682CB160681EF0BDFBA468002CF9D1DE
:1021100010BD00BF00480120024B1868003818BFEE
:102120000120704700480120F0B5194F83B000240A
:1021300001940CF0EBFA3A683AB3164D01A8264622
:10214000D5F8B0111346926829B1994203D8D5F851
:10215000B411994212D803601C4603F108009E6036
:10216000002AEDD1019A0C490C4B3A6000220C6018
:102170001A7003B0BDE8F0400CF002BB1E605E6058
:102180009E60DE60002ADBD1ECE71446EBE700BF7F
:1021900000480120E453012008480120E25D0120AD
:1021A000F0B5144D2B6883B013B3134F0CF0AEFA97
:1021B0003E78C6B92C68114B2E6001223A701E6021
:1021C0007CB12346A4681D6858680190C3E9026683
:1021D0000CF0D6FA019805B1A8470CF097FA002C3C
:1021E000EFD100233B7003B0BDE8F0400CF0C8BA5B
:1021F00003B0F0BD00480120E25D01200848012045
:1022000008B52BF0FFF903460348D98897290CBF7E
:10221000422297222FF084FD8C7A090030B589B0D4
:1022200004AD114C01950846009411461A4604234A
:1022300024F07EFC049853F009FC0546059853F001
:1022400005FC002102462020039223F0D1F9074B20
:102250000360079B0093039A069B2946044647F0B8
:1022600031FA204609B030BDC8D00900C8D10900F4
:1022700008B5086847F058FA0E2008BD08B547F0C1
:1022800053FA0E2008BD00BF10B5044603F09EFDB2
:10229000204647F0DFFA002814BF3E201E2010BD64
:1022A00010B5044603F092FD204647F0E5FA0E20F3
:1022B00010BD00BF70B50C4688B054F8045B0392A3
:1022C0000646284603F082FD284603F07BFE04AB59
:1022D0000193094B039A00932146701E042324F0B6
:1022E000B9FB079C049900942846DDE9052344F0D6
:1022F00015FC0E2008B070BD20D1090070B5054650
:1023000003F064FD284603F05DFE002108462CF032
:10231000C3FC0824064602E00134782C0ED0E1B25A
:10232000284647F019FA0028F6D0610041F0010173
:10233000304601342CF02EF9782CF0D1304670BDA7
:1023400070B50C4688B054F8045B039206462846E4
:1023500003F03CFD284603F035FE04AB01930A4B25
:10236000039A00932146701E042324F073FB0799FF
:102370000124CDE900142846DDE90523049955F030
:102380005FF90E2008B070BDA8D0090070B50C46EA
:102390008CB054F8045B03920646284603F016FD01
:1023A000284603F00FFE05AB01930E4B039A0093F2
:1023B0002146701E072324F04DFB0999089B069ABD
:1023C0000020CDE900100599284655F039F90B9CFD
:1023D0000A9B079A05990094284644F09FFB0E201B
:1023E0000CB070BDE8D0090070B50C4688B054F848
:1023F000046B03920546304603F0F2FC304603F0CE
:10240000EBFD04AB0193154B039A00932146681E24
:10241000042324F01FFB059840F23F4301220021D2
:1024200024F0C4FB4FF48663044601220698002181
:1024300024F0BCFB4FF41E730546092207980821BF
:1024400024F0B4FBC3B2009330460499EBB2E2B27D
:1024500047F046FA0E2008B070BD00BF84D20900D4
:1024600030B589B005AD134C01950846009411466E
:102470001A46032324F05CFB059853F0E7FA05465F
:10248000069853F0EBFA02460798039253F0E6FAE7
:10249000002103462420029323F0AAF82946064D82
:1024A0000560DDE90232044647F036FA204609B0FD
:1024B00030BD00BF04D2090030D3090008B5086858
:1024C00047F082FA0E2008BD08B547F07DFA0E20CD
:1024D00008BD00BF10B5044603F082FC204647F05B
:1024E000A5FB002814BF3E201E2010BD10B50446D9
:1024F00003F076FC204647F0B1FB0E2010BD00BF74
:1025000070B50C468EB054F8046B03920546304605
:1025100003F066FC304603F05FFD0AAB0193144BF9
:10252000039A009321460423681E24F093FA0A9824
:10253000022207A928F010FA0B98089B059006AA1A
:102540000C99069305A83BF0C3F9069A12B90E2020
:102550000EB070BD079805999DF83430014430469F
:1025600047F05AFA0028F2D105202FF085FB00BF72
:102570004CD2090070B50C468CB054F8046B039231
:102580000546304603F02CFC304603F025FD06AB33
:102590000193134B039A009321460323681E24F0F2
:1025A00059FA0698012209A928F0D6F907980A9B3A
:1025B000049005AA0899059304A83BF089F9059AA7
:1025C00012B90E200CB070BD0999049B3046194415
:1025D00047F04CFB0028F4D105202FF04DFB00BF45
:1025E0006CD2090070B50C4694B054F8046B039299
:1025F0000546304603F0F4FB304603F0EDFC0EAB2D
:1026000001931E4B039A009321460623681E24F073
:1026100021FA0E98012208A928F09EF91098099B2A
:102620001199049005AA04A805933BF051F90F985D
:1026300002220BA928F090F912980C9B069007AA89
:102640001399079306A83BF043F9059B079A934219
:1026500011D113B90E2014B070BD0B99069A0898C9
:102660000A4404990144304647F064FA0028F1D145
:1026700005202FF001FB02482FF05EFB1CD2090061
:102680000C7A090009F0D6BCF0B50E2A83B052D0FE
:1026900017468A0706460D4603D12B4A0968914220
:1026A00046D0EB072ED4022101AA28462AF096FE36
:1026B000019B18682AF050FF019A84B250682AF0F2
:1026C0004BFF0546304609F015FDA042ADB235D9A5
:1026D000304609F0CFFCA84230D9042F1ED038462E
:1026E0002AF03AFF0746304609F0A2FC37FA00F319
:1026F00027D130463B462AB221B209F0FDFC0E201C
:1027000003B0F0BD304609F0F5FC6D10042F95FBC9
:10271000F0F200FB12539CB295B2E0D12AB221B282
:10272000304609F0A9FC400040F0010003B0F0BDC4
:1027300006482FF08DFA06482FF066FA05482FF06C
:1027400073FA05482FF0F8FA685709005872090023
:10275000108F0900BC870900CC87090070B52DEDEA
:10276000028B88B0374C009402AB0193062324F00F
:1027700071F93549029840F2EA2224F06DFA3249A3
:1027800040F2F2420546039824F066FA2E490446C8
:1027900040F2F342049824F05FFA069B0E2B0646A3
:1027A0003DD018462AF082FE07980E28F0EE408AA7
:1027B0003AD02AF07BFEB0EE408A0599234814F007
:1027C00003F8696862689142C3B235D1AA7BA07BE5
:1027D000904231D1706881422ED1B17B91422BD190
:1027E000591E082925D8DFE801F005240524052411
:1027F00005241500102A22D12846F0EE480AB0EE32
:10280000680A3246214605F055FC0E2008B0BDECA2
:10281000028B70BD082AEFD00D482FF08DFA079873
:102820000E28F6EE008AC4D1B7EE008A38EE688A28
:10283000C3E708482FF080FA07482FF07DFA0748D1
:102840002FF07AFAB4D40900C8DF090058E1090072
:10285000646C0900A0760900CC8D0900806C090029
:102860002DE9F04F93B0304C00940BAB019307234C
:1028700024F0F0F82D490B9840F2762224F0ECF980
:102880000122044608A90C9828F066F80F9D109EB6
:10289000DDE90DAB6A1C08BFA588731C08BFE6887C
:1028A000BAF1000F3ADBBBF1000F37DB554535DBE2
:1028B0005E4533DBA388AB4230DBE388B3422DDBDC
:1028C000A6EB0B039DF82810A5EB0A070022402079
:1028D00003FB07F724F018FA80461198099BB3FB15
:1028E000F8F90E2814BF0123002315D007932AF00E
:1028F00033FE079B4F4514D8CDE903300899029663
:1029000020460195CDF800B05346424605F0DAFC6A
:102910000E2013B0BDE8F08F0020EBE704482FF045
:1029200083F904482FF080F9F4D30900C8DF0900C7
:10293000BC870900D880090070B586B0274C009488
:1029400002AB0193042324F085F82549039840F253
:10295000F14224F081F940F2EA2221490546029829
:1029600024F07AF9059904461E4813F02DFF0499C6
:1029700006461D4813F028FF61686B688B4224D11E
:10298000A17B1029F6B2C2B201D0012920D1511E7B
:10299000082917D8DFE801F00516051605160516F3
:1029A0001000AB7B102B16D120463346294605F08C
:1029B00001FE0E2006B070BDAB7B082BF4D00B4897
:1029C0002FF0A6F90A482FF0A3F90A482FF0A0F932
:1029D00009482FF09DF909482FF09AF99CD3090076
:1029E000C8DF090090D5090058E10900BC89090039
:1029F000D48B0900B87909008C890900A4890900E1
:102A000013460A46014640F2772013F0C9BE00BFC4
:102A100010B588B003AB1C4C01930094052324F03F
:102A200019F81A49039840F2EA2224F015F9817B3B
:102A3000069B01228A4093421FD2079C6FF00041FF
:102A40008C4201D0A2421BD9BDF91010BDF914204F
:102A500000290FDBB0F804C061450BDA002A09DB5E
:102A6000B0F806C0624505DA009405F085FC0E203A
:102A700008B010BD06482FF05FF906482FF05CF94A
:102A800005482FF059F900BF5CD40900C8DF0900E0
:102A90009C870900408C09009479090030B51A4BD5
:102AA00089B002ACCDE90034062323F0D3FF0298AD
:102AB000079D827B012393409D4222D2BDF90C10D9
:102AC000BDF91020BDF91430BDF91840002918DBFC
:102AD000002B16DB002A14DB002C12DBB0F804C03C
:102AE00061450EDA9C450CDDB0F806C0624508DA97
:102AF000A44506DDCDE9004505F0DCFE0E2009B059
:102B000030BD02482FF018F92CD409009C87090029
:102B100010B5104B88B002ACCDE90034062323F089
:102B200099FF02980799827B0123934099420ED224
:102B3000BDF91840BDF91430BDF91020CDE90041B0
:102B4000BDF90C1005F07AFF0E2008B010BD024848
:102B50002FF0F2F884D409009C8709002DE9F04396
:102B60002DED028B534B9FB011ACCDE900340D23FA
:102B700023F070FFDDE91154AA7BA37B9A42C0F0D9
:102B8000968013980E2800F08F802AF0E5FC06B29C
:102B900014980E2800F085802AF0DEFC07B2179802
:102BA0000E2879D02AF0D8FC0FFA80F818980E2851
:102BB0006DD02AF0D1FC0FFA80F9169B00930DF12D
:102BC0003A0302930EAB159901930DAA0DF136034A
:102BD000284652F0EFFD1A9B00930DF14203029339
:102BE00010AB0193204619990DF13E030FAA52F044
:102BF000E1FD1B980E2844D02AF058FCF0EE408AE4
:102C00001C980E2808D02AF051FCB5EEC00AF1EE4F
:102C100010FAB0EE408A01D5B7EE008A1D980E2852
:102C200032D02AF099FC0023CDE90A03BDF93A30ED
:102C3000BDF93820CDF81490CDE90234BDF94240F9
:102C40000994BDF94040BDF936300894BDF93E40C5
:102C50000794BDF93C40CDF81080CDE900322846FC
:102C6000BDF934300694B0EE680AF0EE480A3A46F0
:102C7000314606F053F80E201FB0BDEC028BBDE8C4
:102C8000F083DFED0D8ABBE701230020CCE7B4F829
:102C900006904FEA590990E7B4F804804FEA5808C3
:102CA00084E7EF887F087AE7AE88760870E7034804
:102CB0002FF042F8E4D40900000000006C890900FC
:102CC00010B58CB0484C009405AB0193072323F05A
:102CD000C1FE4649059840F2762223F0BDFF089CCC
:102CE0000699631E012B28D9042C78D1079B5A1E04
:102CF0001F2A6BD8DFE802F012126A126A6A6A129F
:102D00006A6A6A6A6A6A6A126A6A6A6A6A6A6A6E77
:102D10006A6A6A6A6A6A6A12012C5BD19DF82C2081
:102D200002929DF8282001929DF8242000922246CC
:102D300005F0C4FE0E200CB010BD079B5A1E1F2AC2
:102D400044D80FF2080C5CF822F000BF1D2D0300E0
:102D50001D2D0300CD2D03001D2D0300CD2D0300DF
:102D6000CD2D0300CD2D03001D2D0300CD2D03001F
:102D7000CD2D0300CD2D0300CD2D0300CD2D03005F
:102D8000CD2D0300CD2D03001D2D0300CD2D0300FF
:102D9000CD2D0300CD2D0300CD2D0300CD2D03003F
:102DA000CD2D0300CD2D0300192D0300CD2D0300E3
:102DB000CD2D0300CD2D0300CD2D0300CD2D03001F
:102DC000CD2D0300CD2D03001D2D0300084819460D
:102DD0002EF0BAFF0748182221462EF0B5FF06480C
:102DE00021462EF0B1FF00BFBCD30900C8DF0900A7
:102DF00000820900248209003882090038B50D4B91
:102E0000D3F8083104460D4613B908E01B6833B106
:102E10009A68A242FAD15868A842F7D138BD012178
:102E20000C2022F0E5FB2A462146BDE8384000F0A0
:102E300003B800BFE453012070B40B4DD5F808412E
:102E40005CB1234601E01B683BB19E688E42FAD11B
:102E50005E689642F7D170BC7047C0E9004281605D
:102E6000C5F8080170BC7047E45301200B4AD2F842
:102E700008318BB102F5847C02E09C461B685BB193
:102E80009A688242F9D15A688A42F6D11968CCF818
:102E9000001000221A607047704700BFE453012001
:102EA00038B50C4DD5F8084114B912E0246884B146
:102EB000D5F8B031002BF9D061688B42F6D8D5F83F
:102EC000B4319942F2D2A068FFF7D0FF2468002CF9
:102ED000EED138BDE45301200349044A0023C1F870
:102EE00008311370704700BFE4530120EE5D0120EC
:102EF00008B5084B1B780BB9002008BD064806F042
:102F00006DFE0028F8D1044806F0C8FE003818BF4E
:102F1000012008BDCB5D0120D8450120044BDB8C8E
:102F20004FF6FF709BB2181A18BF0120704700BF00
:102F30002C46012000B50C4883B006F04FFE70B956
:102F40000A4A12785AB1034601220DF107010648D8
:102F500006F04AFE9DF8070003B05DF804FBFF2071
:102F600003B05DF804FB00BFD8450120CB5D012014
:102F70002DE9F041074682B013480D4607F090FB5B
:102F8000F8B9124B1B78E3B1DDB10F4E0446804611
:102F90000CE092B239190023CDF80080304607F0DA
:102FA0007DFC002804440CDBA5420AD9304607F01A
:102FB000B7FB2A1B8242ECD3304607F0B1FB82B24A
:102FC000E8E702B0BDE8F0812C460120CB5D01208E
:102FD00008B50348012106F02BFA0E2008BD00BFFA
:102FE000AC48012010B586B004AB51F8044B0193F6
:102FF0000A4B00930138022323F02CFD40F24122BA
:103000000749049823F028FE039005982AF04EFA09
:103010000399204606F0AAF806B010BDACB109002D
:10302000C4B3090008B506F049F90E2008BD00BF79
:1030300008B512211DF02CFCBDE808400148AA216A
:103040001DF026BC1807012006F03AB908B506F0B5
:1030500055F9002814BF3E201E2008BD08B506F013
:1030600053F9002814BF3E201E2008BD06F060B9A9
:1030700008B506F08BF9002814BF3E201E2008BDBD
:1030800030B5002485B00B4605460DF10E012046F3
:10309000ADF80630ADF80E4045F042FB0DF10601EB
:1030A000284645F03DFB18B9BDF80E0005B030BD0F
:1030B000204605B030BD00BF08B501482EF0C8FD60
:1030C000F08E0900F8B5036905460BB106F0A6FCC1
:1030D000EB6813B1284606F07BFC0B4C0023AB6178
:1030E00004F52A774FF6FF760E252388B342204653
:1030F00001D006F085FFE5658834BC42F5D1BDE816
:10310000F8404CF05DBA00BF1807012008B506F082
:103110006FF908B10E2008BD01482EF02BFE00BF4C
:10312000506A090010B5044608462BF0CDF9014657
:10313000204606F07DF90E2010BD00BF10B50446F4
:1031400008462DF09DF80146204606F0CFFA0E20E5
:1031500010BD00BFF0B52DED028B93B00AAB51F856
:10316000044B0193354B00930138082323F072FC84
:103170000A98012204A927F0EFFB0B9800230E28E0
:10318000CDE90733099303D0012207A927F0E4FB17
:103190000F9800283ED02AF089F9DFED297AB4EEA5
:1031A000E70AF1EE10FAB0EE408A3BD4DFED257A63
:1031B000B4EEE70AF1EE10FA34DC059A9DF83050CF
:1031C0009DF834600E9F1F2A1CD811980E2827D016
:1031D0006DB31D4940F2F62223F03EFD07AB03908C
:1031E0000193204604AB109C0093B0EE480A3B4686
:1031F00032462946029406F08DFA0E2013B0BDEC3B
:10320000028BF0BD4DB1089AA2B911980E28E0D1F9
:103210001046E3E70D480F90BDE7119B0E2B06D13A
:103220000020DBE70A4A0B490B482EF08DFD0B48C6
:103230002EF0A0FD0A482EF09DFD00BF2CB1090024
:103240000AD7A33C0AD72341C4B30900CECC4CBE55
:103250001CB1090024B10900E08109009470090043
:103260003C8F090010B52DED048B90B008AB51F8E0
:10327000044B01933D4B00930138082323F0EAFBF4
:103280000B980E2855D02AF011F90C98B0EE409A00
:10329000002853D00D9B002B55D02AF007F9DFED05
:1032A000347AB4EEE70AF1EE10FAB0EE408A4FD469
:1032B000DFED307AB4EEE70AF1EE10FA48DCB5EE55
:1032C000409AF1EE10FA04D0B4EEC09AF1EE10FA82
:1032D00046D40D982AF0EAF8B4EEC08AF1EE10FA5E
:1032E000F0EE408A39D408980023069300282DD0A8
:1032F000012205A927F030FB05981DF029FD0028C3
:1033000031D0069A9DF83C100E9B09980090CDE9AB
:103310000131B0EE681A9DF828300599F0EE480AA0
:10332000B0EE490A204606F08BFA10B0BDEC048BD3
:1033300010BD0C989FED109A0028ABD10D9B0F4843
:103340000C90002BA9D10D4B0D93A6E70246D9E7AF
:103350000B4A0C490C482EF0F7FC0C482EF0ECFC04
:103360000B482EF0E9FC0B482EF0E6FC6CB109008E
:103370000AD7233B66D6234200000000CECC4CBEC9
:1033800008B1090014B10900E0810900588C090056
:10339000C48509002871090008B506F019FB0E2044
:1033A00008BD00BF08B506F033FB0E2008BD00BF06
:1033B00002280AD1930770B5164604D1104B0C466B
:1033C0001168994203D01E2070BD0020704720462E
:1033D00006F040FB0546304606F03CFB0146284619
:1033E00029F0BCFA0028EED0204606F035FB044652
:1033F000304606F031FB8442E5D13E2070BD00BF6F
:10340000C4B3090006F026BB08B506F025FB400052
:1034100040F0010008BD00BF30B589B0154C0094E4
:1034200003AD0846019511461A46022323F080FB9E
:1034300000210C2022F0DCF80F4B0360044601222F
:10344000039805A927F088FA069B062B0AD1049A4F
:10345000032A0BD820460599D2B206F0F1FA20468D
:1034600009B030BD054806212EF06EFC40F2432025
:1034700023F0E2FA54B30900C4B3090078870900C5
:1034800010B5044688B0084606F0E4FA05A9012202
:1034900027F062FA059920460C780B794A79039453
:1034A0004C7802948C780194CC78009402492EF0E8
:1034B000F5FA08B010BD00BF2CB30900062801D0F2
:1034C0000020704770B5084682B00C4606F0C2FA7C
:1034D0000E4B0340062B054613D0466846B12046E6
:1034E00006F0BAFA7040400040F0010002B070BD32
:1034F00001A928462CF09CFE019942F005FD0646E4
:10350000EDE7000942F032FE0646E7E70F0080FFD4
:1035100031291DD8102918D91139202914D8DFE8EC
:1035200001F01E2113131313131313131313131387
:10353000131324111313131313131313131313134C
:1035400013131B0022230370704721B901707047C9
:103550004129FBD070477047312303707047112316
:103560000370704712230370704721230370704764
:1035700000F0E2BE2DE9F04F97B0434C00940DAB44
:10358000043101380193092323F064FA3F490D986F
:1035900040F2CD4223F060FB3D49064640F27652B0
:1035A0000E9823F059FB0F9CE3B214F0C00408936B
:1035B00066D19DF840800746404606F04FFA9DF8D8
:1035C0004490484606F04AFA2146129840F2D33217
:1035D00023F0E0FA149B9DF84CA00E2B04462BD050
:1035E0000DF1280B18460122594627F0B5F90B9B1F
:1035F000A34231D8BAF1000F2CD115980E282ED045
:103600002CF03EFE09900021282021F0F1FF214AF4
:103610000260099ACDE905B2089A0092CDE9034A01
:10362000CDE901893B4631460022054606F06CFB98
:10363000284617B0BDE8F08FBAF1000F12D0E0B9FC
:1036400015480DF1280B0122594627F085F90B9BEF
:103650009C4201D39C42D0D010482EF06DFB002339
:103660000993D0E70DF1280B0B480122594627F0AA
:1036700073F90B9B9C42C0D2EEE72BF00FF9E0E709
:1036800040F24E4023F0D8F9ACB40900D0BB090099
:10369000D0BC0900DCB50900E0570900F88009003A
:1036A00008B506F087FA0E2008BD00BFF8B505463C
:1036B0000E4614461F4602F04DFB284606F056FA09
:1036C00080B1032E04D016233B604FF0FF30F8BDCD
:1036D00014F00100FBD0284606F0E0FA003818BFCD
:1036E0000120F8BD01482EF097FA00BF0C700900C8
:1036F00030B589B005AD184C0195084600941146C7
:103700001A46032323F014FA40F29B22134905982A
:1037100023F0A2FA40F234510546B7EE000A0698AB
:1037200023F088FA07988DED030A40F289220121DF
:1037300023F030FA002102462020029221F058FFA7
:10374000074B03609DED030A029A2946044606F0E2
:1037500019FA204609B030BD18B60900DCB50900D9
:1037600098B6090010B5044602F0F4FA204606F0B7
:1037700095FA400040F0010010BD00BF10B50446AE
:1037800002F0E8FA204606F0BDF90E2010BD00BF99
:103790002DE9F04105460E4614461F4602F0DAFABE
:1037A000284606F0E3F958B114B92046BDE8F08187
:1037B0003B46224631462846BDE8F04106F014BAA1
:1037C00001482EF029FA00BF0C70090008B5014825
:1037D0002EF03EFAF08F090006F006BB08B506F0A1
:1037E0000FFB400040F0010008BD00BF08B506F027
:1037F00009FB002808BF0E2008BD00BF00B5ADF5CD
:10380000017D4FF40072694606F0FEFA69462AF01F
:10381000FBFF0DF5017D5DF804FB00BF8B688BB1EC
:1038200070B50C460546164608492EF037F9A168D2
:103830002846324600F0FCFC28460549BDE87040A9
:103840002EF02CB903492EF029B900BF74B4090039
:103850000855090084B4090010B584B002AB51F8D2
:10386000044B0193074B00930138022323F0F2F835
:1038700020469DF80C209DF8081006F0E9FA0E206D
:1038800004B010BDF4B4090010B584B004460122A0
:10389000084601A927F060F8204601A906F024FB9C
:1038A0000E2004B010BD00BF10B400230A4C1A460D
:1038B00034F81310814203F1440306D00132052A83
:1038C000F6D100205DF8044B704702EB021204EBC6
:1038D000C2005DF8044B70471807012000234FF623
:1038E000FF724360028080F85A308370083000F025
:1038F00067BE00BF08B5406806F082FB0E2008BD19
:1039000010B584B003AB51F8044B0193074B0093FF
:103910000138012323F09EF8204600F009F80399AE
:10392000204606F071FB04B010BD00BFF0B60900E0
:1039300008B506F097FC00B108BD01482EF06CF9FF
:103940004090090018B143680BB1188870474FF6D2
:10395000FF70704708B506F085FC002814BF3E20B4
:103960001E2008BD10B50446FFF7E2FF606806F0B0
:1039700083FC10EE103A23F0030040F00200A0F1A7
:10398000FF4010BD10B50446FFF7D2FF606806F097
:103990008DFCBDE810402BF0EDB800BF08B506F077
:1039A0008DFC002814BF3E201E2008BD10B5044623
:1039B000C06D0E2800D010BD00210C2021F018FE93
:1039C000024BC0E90034E06510BD00BFC8B7090074
:1039D00010B584B003AB51F8044B0193084B00932E
:1039E0000138012323F036F82046FFF7A1FF606875
:1039F0009DF80C1006F06CFC0E2004B010BD00BF4A
:103A0000E8B6090010B5044682B0084629F04EFD1C
:103A100020468DED010AFFF78BFF60689DED010ADE
:103A200006F090FC0E2002B010BD00BF2DE9F04F53
:103A30008FB007AB384C0193043107230138009451
:103A400023F008F83549079840F29B2223F004F947
:103A5000334940F276520646089823F0FDF89DF867
:103A600024900746484605F0F9FF9DF828A05046E7
:103A700005F0F4FF0B9840F2D332002123F08AF8CE
:103A80000D9B9DF830B00E2B054626D00DF1100889
:103A900018460122414626F05FFF059BAB422AD81B
:103AA000BBF1000F01D09D4225D10021182021F04B
:103AB0009FFD1C49016004464B463A463146CDE91C
:103AC00002B8CDE900A506F05FFC3046214605F0BE
:103AD000D7FF20460FB0BDE8F08FBBF1000F0DD02F
:103AE000B8B911480DF110080122414626F034FF03
:103AF000059B9D42D7D20D482EF01EF90DF11008FE
:103B000009480122414626F027FF059B9D42CCD261
:103B1000F1E72AF0C3FEE5E734B80900DCB5090097
:103B2000D0BC0900E0B80900E0570900F88009009E
:103B300006F058BC08B506F057FC002808BF0E2058
:103B400008BD00BF00B5ADF5017D4FF400726946B8
:103B500006F04CFC69462AF057FE0DF5017D5DF834
:103B600004FB00BF8B688BB170B50C46054616464A
:103B700008492DF093FFA1682846324600F058FB13
:103B800028460549BDE870402DF088BF03492DF057
:103B900085BF00BF04B809000855090010B8090026
:103BA00010B584B004460122084601A926F0D4FECF
:103BB000204601A906F040FC0E2004B010BD00BF55
:103BC00030B5130683B004460D4601D4022A06D050
:103BD0002946204603B0BDE8304029F00BB940F239
:103BE0002F20019242F0E2FA014620462DF0EAFE33
:103BF000054920462DF0E6FE019A2946204603B0ED
:103C0000BDE8304029F0F6B82CBD090008B506F033
:103C100035FD0E2008BD00BF08B506F05DFD00288B
:103C200003DB400040F0010008BD01482EF084F89D
:103C3000406F090008B506F073FD002803DB400063
:103C400040F0010008BD01482EF076F8406F0900F1
:103C5000F0B587B0194C009403AD084601951146A4
:103C60001A46032322F064FF1549039840F29B2271
:103C700022F0F2FF40F2892206460121049822F048
:103C800089FF0746304606F0B9F8059B0E2B12D087
:103C9000184629F061FC04460021302021F0A8FCE0
:103CA0002346084C04603A463146054606F0A4FC1B
:103CB000284607B0F0BD0446EEE700BF2CB9090066
:103CC000DCB50900BCB9090030B585B004460D4625
:103CD00006F0E6FC80B9022201A9284626F03CFE47
:103CE000DDE90112204606F073FD011E07DB4800E6
:103CF00040F0010005B030BD42F0C6FAEBE70248E3
:103D000049422EF021F800BF4C8E090010B58AB050
:103D10000C4602AB17490193013800910223211D83
:103D200022F098FE2468204606F0BAFCF0B902980A
:103D3000012204A926F010FE039800230E28089300
:103D400012D0012207A926F007FE08980090DDE9AD
:103D50000412079B204606F0A1FD20EAE070400017
:103D600040F001000AB010BD1846EFE742F08CFAAF
:103D7000DDE700BF1CB9090010B50B4C0B4B2360ED
:103D8000204605F003FB00B910BD4BF0A3FB204615
:103D9000FFF798F92046002105F04AFB00F0B8FC37
:103DA000BDE810404BF05AB8AC48012010B30900F0
:103DB0002DE9F04F83B09DF83040CDE9004383B347
:103DC0008B4619B307469246002606F101081AF8F9
:103DD000066000240AEB08093D5D0134324649467D
:103DE00038193DB1AE4202D821F09CFF90B12C446D
:103DF000A345F1D8009B83B1019B4644B342E4D86C
:103E0000009B83F0010003B0BDE8F08F084603B0CB
:103E1000BDE8F08F009B002BEED0009803B0BDE80A
:103E2000F08F012003B0BDE8F08F00BF06F0F2BDB7
:103E300010B58AB005AB51F8044B01930C4B0093BD
:103E40000138022322F006FE9DF8183005980393EE
:103E500007A9012226F080FDDDE90712039B204619
:103E600006F0E4FD002814BF3E201E200AB010BD5D
:103E7000E4B9090038B54FF6FF72002304468360A9
:103E80000D468280194618462AF006FF012320615C
:103E9000E380E56038BD00BF06F026BF08B506F038
:103EA00029FF002814BF3E201E2008BD08B506F0DB
:103EB00023FF002814BF3E201E2008BD08B506F0D1
:103EC0001DFF002808BF0E2008BD00BF30B587B019
:103ED00004AD104C01950846009411461A46022381
:103EE00022F026FE0C49049840F2765222F0B4FEED
:103EF0009DF81420039205460021182021F078FB3C
:103F0000064B0360039A2946044606F0D9FE204674
:103F100007B030BD40BB0900D0BC0900D0BB0900D0
:103F20008B688BB170B50C460546164608492DF0D6
:103F3000B5FDA1682846324600F07AF928460549C1
:103F4000BDE870402DF0AABD03492DF0A7BD00BF0C
:103F500010BB0900085509001CBB090008B5014841
:103F60002DF076FE2C70090008B5064805F050FDCE
:103F7000044805F02DFDFEF793FFBDE8084049F029
:103F800035BC00BFAC48012002280BD130B59307E7
:103F900089B0144603D11C4B12689A4204D01E20EB
:103FA00009B030BD0020704708460D4606F0C2FE3D
:103FB000102804D1204606F0BDFE102819D069460D
:103FC000284606F0BDFE04A9204606F0B9FE009A78
:103FD000049B9A42E3D1019A059B9A42DFD1029A4F
:103FE000069B9A42DBD1039A079B9A42D7D13E2087
:103FF000D6E7284606F0B2FE034620461C4606F0E9
:10400000ADFE8442CBD1F2E7D0BC090008B58B7875
:1040100023B10B8883808B78837108BD01482DF014
:10402000A9FE00BF0876090083880B8083798B7016
:10403000704700BF08B506F07DFE400040F001006B
:1040400008BD00BF10B584B0044606F073FE80289A
:1040500009D16946204606F073FE102168462AF011
:1040600005FC04B010BD01482DF0CEFDD48509003B
:1040700008B506F073FE400040F0010008BD00BF27
:104080002DE9F0410C468EB0114605464FF0021264
:1040900020461C4622F0A4FC0021082021F0A8FAAA
:1040A000056007462068C2073AD483072AD1026810
:1040B000434B9A4234D0434B0340062B26D0424B0D
:1040C0009A4223D0012206A926F032FC00286ED0A5
:1040D000079B102B6ED1069B02AD186859689A6831
:1040E000DB682C460FC4BDF81410002338462A465E
:1040F0008DF814308DF8153006F002FE38460EB0FB
:10410000BDE8F0812F4B0340062BDBD101A92CF039
:104110008FF8019B242B064610D02C482DF00CFE66
:1041200029F01AFAB0F5803F014646D238460022FF
:1041300006F0E6FD38460EB0BDE8F081037A2D2B7F
:10414000EBD1437B2D2BE8D1837C2D2BE5D1C37D97
:104150002D2BE2D1451E4FF000082C4615F8010F1B
:104160004FF0B0FA30B10EAB43442A7803F8202C5C
:1041700008F10108019AA31C9B1B9A42EDD8B8F1E3
:10418000200FCAD106AC0DF117060DF138082078C2
:104190004FF0B6FA054660784FF0B2FA023440EAC2
:1041A0000510444506F80109F1D102AD9BE7084826
:1041B0002DF0C2FD07482DF0BFFD07482DF0BCFDD6
:1041C0003C4E09000F0080FF545A09007C7509001D
:1041D000947509006C8E09006C75090030B589B0C2
:1041E00003AB51F8045B01930F4B0093013802239A
:1041F00022F030FC0398022205A926F0ADFB2846E8
:10420000049C06F097FD069B04EBD000984207D86B
:1042100005992846214406F0A3FD0E2009B030BDC3
:1042200002482DF089FD00BF5CBC0900148E090016
:1042300030B5054693B008460C4606F07BFD1028C5
:1042400037D00EA9204606F07BFD9DF838209DF85A
:1042500039100D929DF83A209DF83B409DF844306E
:104260009DF845000193CDE90B219DF83C209DF878
:104270003D100090CDE909249DF83E209DF83F4077
:104280009DF84630CDE907219DF840209DF841106A
:10429000CDE905249DF842209DF843400294CDE9E4
:1042A000032128469DF8472007492DF0F7FB13B05E
:1042B00030BD204606F052FD04490246284613B0A0
:1042C000BDE830402DF0EABB0CBC0900FCBB090086
:1042D000062801D00020704710B5084684B00C466F
:1042E00006F028FD102812D06946204606F028FD69
:1042F000ADF102030DF10E01002033F8022F9942B7
:104300001044FAD1400040F0010004B010BD204636
:1043100006F024FD400040F0010004B010BD00BFD5
:1043200008B549F063FABDE80840FFF721B900BFBE
:10433000704700BF704700BF2DE9F04F2DED028B95
:10434000DFF878A289B0002500AFAAF1080B05EBD1
:1043500005130BEBC3034FEA051893F87830002BD5
:1043600040F0A08008EB05030BEBC30393F8793012
:1043700053B90135052D0AF1880AE8D12437BD4625
:10438000BDEC028BBDE8F08F1AF8069CB9F1000F66
:1043900000F0AC80BAF82E30FB60FA680121484684
:1043A0001AF01EFE0446002800F0FE80C288502A43
:1043B00005D15146083021F0B5FC00286AD0002311
:1043C000BB6107F1180320460122194608EE103A96
:1043D00044F02AFA1AF8069C002039F0BDF9044688
:1043E000002834D00AF14903BB6004E0204639F0CC
:1043F000B3F9044658B36678012EF7D1237803F059
:1044000001034B45F2D1E388502BEFD1B9687B60B3
:10441000062204F1510021F085FC7B6884461A468F
:104420006346514604F10800C7F804C0002BDDD1F3
:1044300021F078FC7B680028D8D018EE101A32469C
:104440002046BB6144F0F0F91AF8069CCEE7FB6801
:104450007B834FF000033B763AF8083CBB833B8BF1
:1044600049F48079502403F0FE0329F0FE0943EA61
:1044700009092046FC83A7F818901AF003FE18EEED
:10448000101A0646022244F0CFF922465146304621
:1044900052F0CAFEA8440BEBC8084FF0000388F89E
:1044A000793066E74BF08CF8DAE91E23801A61EB6D
:1044B0000301B0F57A7F71F10003FFF453AF4FF0C1
:1044C0000003FB823AF8080C032307F116020021CF
:1044D00044F064F96C4668B108EB05030BEBC303C9
:1044E0004FF00002A54683F878203BE7BAF8123077
:1044F000FB6052E7FB8A3AF8080C0733DB08A4EBB1
:10450000C3039D4607F116020323694644F046F9AA
:104510006E460028E0D11AF8069CBAF85020FA60DE
:10452000022148461AF05CFDFA680346002840D094
:10453000F98AC2888A4208D100F10801F860684609
:1045400021F0F0FBFB680028C6D018460023BB61B1
:1045500007F118030122194608EE103A44F064F9F5
:104560001AF8069CBAF850207A834FF000033B7685
:104570003A8BF88AF88349F4007302F0FE0223F0C4
:10458000FE0313433B833AF8083CBB831AF07AFDE1
:1045900018EE101A8146022244F046F9FA8A314692
:1045A000484652F041FE97E707F1180308EE103A2B
:1045B00012E707F1180308EE103AD5E720070120AB
:1045C0005022002121F070BC10B54FF46A2482B053
:1045D000200B04F5805444F013F9B4F5722FF7D191
:1045E000074B019301A901224FF46A2044F01CF902
:1045F000012201A9034844F017F902B010BD00BF21
:1046000031304442FC1F0F0010B50C4602211AF055
:10461000E7FC48B1C28800F108010323204644F0BA
:10462000BFF8B0FA80F0400910BD00BF70B5154664
:10463000F2B100240646204601E0A54216D939F021
:104640008BF898B14378013BDBB2FD2BF5D80378AA
:1046500003F00103B342F0D1C388502B00F14002B4
:1046600004D141F824200134A542E8D8204670BD89
:104670001446FBE710B50C461346012122461C46A2
:104680001AF0AEFC18B1C288502A01D0002010BD2B
:1046900000F10801204621F057FB012010BD00BFAA
:1046A00070B50546002039F057F80446B8B14E1CE5
:1046B00004E0204639F050F8044680B16378012BBD
:1046C000F7D1237803F00103AB42F2D1062204F1C3
:1046D0005100314621F026FB0028EAD1243420463F
:1046E00070BD00BF08B50021084639F035F860B14B
:1046F0004378013BDBB2FD2BF7D80378DB07F4D41A
:10470000013139F029F80028F2D1084608BD00BF70
:104710004FF46A23064A1B68934205D14FF4712275
:10472000D2F8FC2F9A4201D0FFF74EBF704700BF6E
:10473000313044421E3918BF0121490041F00101C6
:1047400022F0D0BC38B50C462046114602221D4648
:1047500022F046F90CB91E2038BD286829F0B4FEB5
:104760000028F8D03E2038BD032A04D01E2907D0E7
:1047700006492DF027B91E2905D005492DF022B98B
:1047800004492DF01FB904492DF01CB96CEE080046
:1047900014370900D83709001C370900052807D04D
:1047A0001E3918BF0121490041F001012EF074BEED
:1047B00000207047136803B17047406827F02EB996
:1047C00000B583B08C46D0E90101009313466246E0
:1047D00024F01EF803B05DF804FB00BF00230122A3
:1047E00000F000B82DE9F047054688B008680C468F
:1047F0001F46914628F006FF012202A98046206844
:1048000026F0AAF86068012205A926F0A5F89DF80F
:104810001C100022402022F077FA012835D1DDE972
:104820000261022D06EB010A14D9A2680E2A04D0F7
:104830000346404626F09AF80644032D0AD0E26863
:104840000E2A07D0DDE902414046012326F08EF80A
:1048500004EB000AB24505D2D7B94FF0FF3008B0DB
:10486000BDE8F087069B059ACDF80090AAEB0601FB
:1048700030461AF0E1FB0028EED0029BC01A40003F
:1048800040F0010008B0BDE8F08703482DF040FA81
:1048900002482DF051FA00BFA8780900048A0900E7
:1048A00001231A46FFF79EBF00234FF0FF32FFF7A8
:1048B00099BF00BF01234FF0FF32FFF793BF00BF46
:1048C000174B0120002210B51146C3F81405C3F898
:1048D0001005930003F1804303F51C330132082ACD
:1048E00059609962F5D10E4B0E4C59629964C3F828
:1048F0005811D3F80004D3F800240B490243C3F83D
:104900000024D3F80023C3F808232046C3F8041377
:10491000DC22002121F0C8FA4023A382238110BDAC
:1049200000700240C41F01200514C00170B588B09A
:104930000D460C2000211646039320F059FE104B23
:10494000036004AB01930F4B039A00930446314676
:104950000423284622F0ECF8049851F077F8014639
:104960000598039151F072F80246DDE9063003998B
:104970000090204606F002FA204608B070BD00BF45
:1049800088D7090088D6090008B5086806F0C0FA7B
:104990000E2008BD08B506F0BBFA0E2008BD00BF0A
:1049A00010B5044601F026FA204606F077FB0028F1
:1049B00014BF3E201E2010BD10B5044601F01AFAA7
:1049C000204606F073FB0E2010BD00BF70B50C46EC
:1049D0008EB054F8045B03920646284601F00AFAAA
:1049E000284601F003FB0AAB0193154B039A009391
:1049F00021460423701E22F02DF80B98022207A9ED
:104A000025F0AAFFDDE90C310898059005AA06A853
:104A1000069338F05DFF4FF422720121059822F0D1
:104A2000EDF8DDE90620059BBDF828100244284674
:104A300006F0F4FA10B90E200EB070BD2DF01CF97E
:104A4000E0D6090070B5054601F0D4F9284601F01A
:104A5000CDFA002108462AF01FF90824064602E094
:104A60000134782C0ED0E1B2284606F08DFA0028E9
:104A7000F6D0610041F001013046013429F08AFD91
:104A8000782CF0D1304670BD70B50C468EB054F81D
:104A9000045B03920646284601F0ACF9284601F073
:104AA000A5FA0AAB0193124B039A00932146042303
:104AB000701E21F0CFFF0B98012207A925F04CFFB3
:104AC000DDE90C310898059005AA06A8069338F090
:104AD000FFFEDDE90620059BBDF8281002442846AC
:104AE00006F0E8FA10B90E200EB070BD2DF0C4F833
:104AF00068D6090070B50C4696B054F8045B039272
:104B00000646284601F076F9284601F06FFA0FAB09
:104B100001931F4B039A009321460723701E21F037
:104B200099FF1098012209A925F016FFDDE912313D
:104B30000A98059005AA06A8069338F0C9FE1198B0
:104B400002220CA925F008FFDDE914310D98079029
:104B500007AA08A8089338F0BBFE40F217420121CB
:104B6000079822F04BF8DDE90814DDE906200C9BDC
:104B70001944CDE90010059BBDF83C10224428469D
:104B800006F0A0FA10B90E2016B070BD2DF074F822
:104B9000A8D6090070B50C4688B054F8045B03929F
:104BA0000646284601F030F9284601F029FA04AB00
:104BB0000193174B039A00932146701E042321F0A2
:104BC00049FF40F23F4301220021059821F0EEFF0A
:104BD0004FF48663012200210446069821F0E6FF87
:104BE0004FF41E73092206460821079821F0DEFFC4
:104BF000C0B200900499F3B2E2B2284606F07AFA05
:104C000010B10E2008B070BD05202DF035F800BFA2
:104C10004CD8090070B588B00D460C20002116460E
:104C2000039320F0E5FC154B036004AB0193144B98
:104C3000039A0093314604230446284621F078FF66
:104C4000049850F003FF0646059850F007FF05460C
:104C5000069850F003FF034650B19DF81C200092C7
:104C600020462A46314606F07BFA204608B070BD41
:104C7000002DF2D103482DF05FF800BF18D90900CC
:104C8000C4D70900986E090008B5086806F0F6FA5E
:104C90000E2008BD08B506F0F1FA0E2008BD00BFD1
:104CA00010B5044601F0B0F8204606F005FB4000C0
:104CB00040F0010010BD00BF08B506F0B3FB0028AE
:104CC00014BF3E201E2008BD10B5044601F09CF81C
:104CD000204606F0AFFB0E2010BD00BF70B50C469D
:104CE0008EB054F8046B03920546304601F08CF800
:104CF000304601F085F90AAB0193144B039A0093F7
:104D000021460423681E21F0A5FE0A98022207A965
:104D100025F022FE0B98089B059006AA0C99069395
:104D200005A838F0D5FD069A12B90E200EB070BD58
:104D3000079805999DF834300144304606F028FB69
:104D40000028F2D105202CF097FF00BF14D80900ED
:104D500070B50C468CB054F8046B0392054630468F
:104D600001F052F8304601F04BF906AB0193134BBA
:104D7000039A009321460323681E21F06BFE0698D8
:104D8000012209A925F0E8FD07980A9B049005AACD
:104D90000899059304A838F09BFD059A12B90E20D6
:104DA0000CB070BD0999049B3046194406F046FBCF
:104DB0000028F4D105202CF05FFF00BF34D8090093
:104DC00070B50C4694B054F8046B03920546304617
:104DD00001F01AF8304601F013F90EAB01931E4BA7
:104DE000039A009321460623681E21F033FE0E9895
:104DF000012208A925F0B0FD1098099B1199049093
:104E000005AA04A8059338F063FD0F9802220BA9A8
:104E100025F0A2FD12980C9B069007AA1399079300
:104E200006A838F055FD059B079A934211D113B996
:104E30000E2014B070BD0B99069A08980A44049984
:104E40000144304606F0B4FA0028F1D105202CF0D8
:104E500013FF02482CF070FFE4D709000C7A090018
:104E6000F8B50D4614461E4630F0BAFF074600F06E
:104E7000D5FF032D05D0162333604FF0FF352846AC
:104E8000F8BD14F0010509D16307F8D5384606F0DE
:104E90004DFD0028F3D045F00405F0E7384606F054
:104EA0004DFD051E18BF0125EEE700BF2DE9F04FAF
:104EB0002DED028B99B00CAD3B4C0195084600944A
:104EC00011461A460C2321F033FE0D9850F0C6FD12
:104ED00007460C9850F0C2FD054600285BD04FF401
:104EE0001E7309220F98052121F060FE109B2F4AA6
:104EF00093425FFA80FA53D02D4A93420CBF0223AB
:104F000000230B93962302220121119821F04EFEDB
:104F10000446129828F0CAFAFDEEC07A40F23453E3
:104F200017EE900A64220021B0EE408A21F03EFE86
:104F3000149850F093FD0A90159850F08FFD80461C
:104F4000169850F08BFD012181462C209DF85CB015
:104F500020F076FBE4B22946164D056006940B9CC2
:104F60000A9BCDF80080CDE904A4BDF84C4007941D
:104F70000E9C03940024CDE9019BCDE90844B0EEDA
:104F8000480A3A46064606F0C5FA304619B0BDEC66
:104F9000028BBDE8F08F002FA1D107482CF0CCFE8A
:104FA00001230B93AEE700BF60D9090084DA090042
:104FB000A8DA0900F0DA0900188B090008B50868BA
:104FC00006F0D6FB0E2008BD08B530F009FF06F04C
:104FD000CFFB0E2008BD00BF10B530F001FF044626
:104FE00000F01CFF204606F001FC400040F00100EC
:104FF00010BD00BF10B530F0F3FE044600F00EFF08
:10500000204606F09BFC400040F0010010BD00BFB0
:1050100010B530F0E5FE044600F000FF204606F033
:10502000E7FB10EE103A23F0030040F00200A0F17D
:10503000FF4010BD10B530F0D3FE044600F0EEFE88
:10504000204606F037FA0E2010BD00BF38B50D46D9
:1050500030F0C6FE044600F0E1FE284628F07CFA57
:105060000146204606F06EFC0E2038BD38B52DED09
:10507000028B0D4630F0B4FE044600F0CFFE284609
:1050800028F014FAFDEEC07AB0EE408A17EE900ACE
:1050900040F234536422002121F088FDB0EE480A2A
:1050A000204606F075FCBDEC028B0E2038BD00BF1B
:1050B00010B50B4C40F2451240F2791382B08C428D
:1050C00008BF134640F2D512CDE90023054940F24E
:1050D0001E234FF423722CF0E1FC02B010BD00BF80
:1050E00084DA090054D909002DE9F04114460E462E
:1050F0001F4630F075FE054600F090FE14B92046BC
:10510000BDE8F0813B46224631462846BDE8F041E5
:1051100006F07ABB10B584B0CDE90221019330F0DE
:105120005FFE044600F07AFEDDE901320399204675
:1051300004B0BDE8104006F037BC00BF30B50C46E7
:1051400083B01146204606221D4621F049FC0CB3CF
:105150002868C20711D5012C23D128F0FDF901469A
:1051600001902046FAF7C2FF019A04460021C06868
:1051700020F09AFE204603B030BD830703D10A4BCE
:1051800002689A42E7D00146012003B0BDE83040F2
:10519000FAF77CBE2146012003B0BDE83040FAF7A3
:1051A000A5BF02482CF0B4FD3C4E0900D08C09008C
:1051B00000B5012883B00B4608D084460022614622
:1051C00007482BF087F803B05DF804FB0A6840F647
:1051D0001623CDE900234FF0020C6B46EEE700BF2B
:1051E000545A090010B5044682B0806801A92BF01A
:1051F0001FF8E368019A934207D2C05C4000013374
:1052000040F00100E36002B010BD002002B010BD0C
:1052100032B9084611B1194600F008B80248704783
:1052200008B521F011FC00BFE057090070B50A680D
:10523000930790B00E46044625D111684D4B994214
:105240001ED04D4B1340062B21D04C4B99421ED003
:10525000012C40F0868012F0010535D0521000F18B
:10526000868011460CA8019251F000FE019A0E981A
:10527000002120F019FE3F480CA929F0E5FD024667
:10528000104610B070BD3C4B1340062BE0D1A01E61
:10529000012866D810460CA92AF0CAFF3268364B9E
:1052A0001340062B054623D05468DCB100211020A2
:1052B0000C9E20F09DF92F4B03600246C0E9026569
:1052C0004460104610B070BD1046B12103AA26F00C
:1052D000A5FB039B8BB103AA2946284623F024F99A
:1052E0000246CDE70C99284640F00EFE0446DDE765
:1052F000100940F03BFF0446D7E73068224605A975
:1053000025F016FB30BB306829F01CF908ADE0B180
:105310004110284651F08CFD30680CA925F07CFB2B
:10532000044607E028F018F9FF281DD8C1B2284626
:1053300051F068FC204625F0AFFD0028F2D10D4861
:10534000294629F081FD02469AE71021284651F0AE
:105350006FFDE1E7DDE90512064829F055FD02463B
:105360008EE707482CF0D4FC06482CF0E5FC002022
:105370002CF0E2FCF05709000F0080FF545A09009E
:10538000D08C0900307A0900F0B585B01546064684
:105390000C4628F037F96946074630462AF048FFA0
:1053A000042D12D1A307064603D1124B22689A425C
:1053B0000ED0009900232246384625F0D7FA305CFB
:1053C000400040F0010005B0F0BD002005B0F0BD88
:1053D000009801AA21462DF025FA40B1DDE90132FD
:1053E0003846F118D21A29F08FFD05B0F0BD0248F9
:1053F0002CF02EFC68570900C48609002DE9F047FF
:105400008F070C460646154610D001F00F03022BFD
:1054100004D0B368002B58D0BDE8F087D6074FEA18
:1054200011114ED5BDE8F0470FF0AEBD4968CBB2C3
:105430002D2B51D023D8062B39D02C2BE9D1022A81
:1054400060D1E768002FE4D017F00308E1D17B6852
:10545000DAB28E2AB94659D0312A72D0322AD8D13E
:10546000012D00F08E80022D00F09780D9F80810F1
:10547000B06A0122BDE8F047090923F04DBC2E2B8C
:1054800013D1002AC5D1A168002937D08D0704D1D6
:105490000A464968CBB2922B24D004F10802304668
:1054A0000121BDE8F04700F07FB89D2BB1D1002D60
:1054B000AFD104F108023046090ABDE8F04700F018
:1054C00073B8BDE8F04710F037B821463046354A8A
:1054D000BDE8F04710F088B8A268002A99D0002DE6
:1054E00097D15168090A022906D1D36823B19807D8
:1054F00002D11B79AC2B8CD008323046BDE8F04786
:1055000000F052B8A1680FF075FD9AE74FEA132931
:10551000022D09F1FF390DD0B9F1000F0ADD07F1B5
:10552000040A5AF8041F08F1010830460FF062FD22
:10553000C845F6D109F1020957F8299099F80420D5
:105540008AE7022D0CD03046D9F808100FF052FD32
:10555000012DB06A0DD0BDE8F047012123F09CBFBA
:10556000B06A23F007FEB06A0121BDE8F04723F0DE
:1055700093BF23F049FCB06A0021BDE8F04723F057
:105580008BBFB06A23F03CFCD9F80810B06A002247
:10559000BDE8F047090923F0BFBBB06A23F0EEFD78
:1055A00064E700BF5C7A09002DE9F04781460029D5
:1055B00047D04FF0FF3817460E46151F002401EB69
:1055C000080A02E00134A64216D055F8043F002B29
:1055D000F8D09A07F6D11A79222AF3D1B8F1FF3F11
:1055E000AAEB0402214621D1D9F82800A0460134B3
:1055F00023F074FFA642E8D1B8F1FF3F10D0002499
:10560000A0450ABF3B6839689968002248460134C2
:10561000FFF7F4FEA64207F10407F1D8BDE8F087D2
:10562000D9F82800314623F061FFE8E7D9F80820CF
:10563000002AF3D14846054ABDE8F04719460FF065
:10564000D3BFBDE8F047806A23F050BF80840900D3
:105650002DE9F84301F00F03022B0C4622D005463A
:1056600019B9AB681BB3BDE8F88311F00306F8D194
:105670000B792C2B22D02D2BF3D1A468002CF0D049
:1056800063681B0A022B33D0002BECD0271D57F880
:10569000041F2846FFF7DCFF63680136B6EB132FC3
:1056A000F5D3E0E7BDE8F84309090EF011BF214644
:1056B0002846244ABDE8F8430FF096BF89680FF0EA
:1056C00099FCE768002FCCD017F00306C9D17B689E
:1056D000DAB28E2A394614D0312A29D0322AC0D1E2
:1056E0008968A86A0222BDE8F843090923F014BBBF
:1056F000E368002BCAD09A07C8D11B79AC2BC5D15F
:10570000AFE71B0A03F1FF38B8F1000FC8BF07F17C
:10571000040907DD59F8041F013628460FF06AFC1A
:105720004645F7D108F1020857F828100A79D3E75F
:10573000284689680FF05EFCA86A0221BDE8F8439C
:1057400023F0AABEB07A09002DE9F04F074683B0D6
:105750000C461646984612E02BF0A4FC58BBDCB170
:10576000A30719D16168CBB21E2B4FEA11212BD0B0
:105770001F2B59D0202B0DD1A46886F0010620469E
:105780002BF082FC03462046002BE5D0AEB103B0DF
:10579000BDE8F08F2D2B0BD0384621460FF02AFCA8
:1057A000B86A4246314603B0BDE8F04F23F0C0BCB2
:1057B000A368002BEAD0002EE9D0B86A414603B0B6
:1057C000BDE8F04F23F0AEBB86BBD7F8109001F1D7
:1057D000FF3A09F10103BAF1000F3B6114DD04EB5C
:1057E000810586F0010204F1040B019626462C4641
:1057F00015465BF8041F4B462A463846FFF7A4FFC0
:10580000A345F6D13446019E0AF1020A384654F8FF
:105810002A1043463246FFF797FFB86A494603B05D
:10582000BDE8F04F23F090BB002ECED10029AED0C2
:10583000251D05EB810455F8041F434632463846C2
:10584000FFF782FFAC42F6D103B0BDE8F08F00BF96
:10585000137803F06003202B0ED170B594462F4AC5
:10586000BCF8043092F800E09E4507D092F8B8E802
:105870009E4540D0002070BD0020704700249CF859
:105880000130203B032BF5D8DFE803F0281F070287
:10589000A9B3022938D0012070BD81B30229FAD101
:1058A000BCF80250157105F0010686F0010102F105
:1058B00024004BF0ADFF1A4B002BECD0C5F3400297
:1058C000314620464BF0DEFFE5E70029E3D1072310
:1058D000063261464CF006F9012070BD0029F6D071
:1058E0000229D8D10F4B002BD5D02046911DAFF304
:1058F0000080012070BD02F6B8020124BFE76146B6
:105900004CF0D6F8012070BD074B002BC3D02046C9
:10591000BCF802104CF0B0F8012070BD7C0D0120E5
:105920008518080000000000791A08002DE9F043EE
:10593000244C83B000260125314641F270122046E6
:1059400020F0B2FA4FF0FF094FF4424808272B46E7
:1059500004F1380100964FF4806204F1100084F8DD
:105960000590A4F80680258127734BF0DBFE2B46BB
:1059700004F5876100954FF4806204F124004BF038
:10598000D1FE2B4604F50F6100964FF4806204F6B9
:10599000C80084F8BD98A4F8BE88A4F8C058A4F83C
:1059A000C26884F8C4784BF0BDFE00952B464FF4D6
:1059B000806204F54F6104F6DC004BF0B3FE03B0E7
:1059C000BDE8F0837C0D01202DE9F0474B79022BD7
:1059D00082B012D18B79022B0FD1DFF8DC9099F8CD
:1059E0000270064687B199F8BA38002B5DD04FF0A7
:1059F000E023D3F8F03DDB0704D40025284602B0AD
:105A0000BDE8F08700BEF8E7C846BA4640F6B803DE
:105A100003FB0AF3887809F803000C780C44092585
:105A2000617824290BD1082A02D810E0AA420ED3AB
:105A300023781C442B44617824299DB2F6D0052993
:105A40000CD06378042B02D163790A2B18D040461E
:105A5000F7F7A4FB284602B0BDE8F08721463046A0
:105A60004FF01EF90028C2D040F6B80303FB0A9A93
:105A7000A3788AF801302278AB1814449DB2E0E78D
:105A8000BA1CFB1C4A444B4430462678CDE9003210
:105A90000223A1191A464FF0A3F90028A7D005F157
:105AA0000E0316FA83F39DB2D1E709F6B80840F663
:105AB000B8074FF0010AA9E77C0D012070B5124C20
:105AC000002504F1240604F11000256025714BF037
:105AD0001DFE30464BF01AFE012130464BF098FE79
:105AE00004F6DC0604F6C800C4F8B85884F8BC58BC
:105AF0004BF00CFE30464BF009FE30460121BDE86C
:105B000070404BF085BE00BF7C0D01202DE9F84FA1
:105B1000454AD5788D420C4606461F4616D09378E6
:105B20008B426FD092F8BB388B426FD092F8BA3864
:105B30008B4270D04FF0E023D3F8F04D14F0010405
:105B400001D000BE00242046BDE8F88F15464FF076
:105B5000000905F1100ABAB205F6380150464BF0BB
:105B60008BFE324BD3B16B79FF2B17D0B7B107F651
:105B7000370BAB4405F6370802E0C3450ED06B790E
:105B800018F8012F9A42F8D150464BF0F3FD002847
:105B9000F3D1697948464BF061FFEEE7244B23B11E
:105BA00050464BF0E7FD00283AD02846F7F7F6FAC2
:105BB000AB78A34203D001242046BDE8F88F1D4BEB
:105BC00013B14846AFF3008048464BF003FF00286E
:105BD000F1D105F124004BF0BDFD0028EBD1002FE1
:105BE000E9D017F03F07E6D1A97830464FF022F808
:105BF00004460028DFD0A9783B463A4630464FF0AD
:105C0000B5F8A0E715464FF00009D1E702F6B80550
:105C10004FF001099DE702F6B8054FF00109C7E70B
:105C20004846AFF30080C0E77C0D01205D1A0800F4
:105C3000000000000000000010EE103AC3F3C7524D
:105C40007F3A162A2ADC002A10EE101A82B014DBE2
:105C5000154840FA02F21A420DD0DFED147A70EEC8
:105C6000277A0029CDED007AA8BF8918009B21EA88
:105C7000020300EE103A02B07047DFED0C7A70EECE
:105C8000277A002BCDED017A019A08DB5A00B7EE96
:105C9000000A08BF00EE103A02B0704770479FED4F
:105CA000040A02B0704700BFFFFF7F000000807B46
:105CB0000000008010B50288392A0B460AD0502A0D
:105CC00006D14A68C188928A91420DD0012010BD48
:105CD000002010BD047B012CF8D14A684189928ACA
:105CE000914209D0204610BD028A00F112011846E7
:105CF00051F0F8FB012010BDC28900F110011846D7
:105D000051F0F0FB204610BD10B586B00C46ADF842
:105D100006300DF10603CDE90432BDF820C0ADF820
:105D2000080000218DF80AC0ADF80C1002A9204629
:105D300042F02AFD48B1132809D000F081F902A9E8
:105D4000204642F021FD0028F5D106B010BD48F0F4
:105D5000EBFEEBE708B503F041FF00B908BDBDE875
:105D6000084040F091BA00BF08B501F097FB00B9B8
:105D700008BDBDE8084040F087BA00BF08B501F093
:105D800057FE00B908BDBDE8084040F07DBA00BF2D
:105D900008B501F08DFE00B908BDBDE8084040F02F
:105DA00073BA00BF08B501F083FF00B908BDBDE8B4
:105DB000084040F069BA00BF08B502F07FF800B9AA
:105DC00008BDBDE8084040F05FBA00BF08B543F029
:105DD000BDFC00B908BDBDE8084040F055BA00BFA1
:105DE00008B543F00FFE00B908BDBDE8084040F01B
:105DF0004BBA00BF08B505F0A1F800B908BDBDE871
:105E0000084040F041BA00BF08B505F04DFA00B9AE
:105E100008BDBDE8084040F037BA00BF08B505F03E
:105E2000DDFC00B908BDBDE8084040F02DBA00BF58
:105E300008B505F085FE00B908BDBDE8084040F092
:105E400023BA00BF08B505F0BBFE00B908BDBDE828
:105E5000084040F019BA00BF08B508F0E5F900B9EC
:105E600008BDBDE8084040F00FBA00BF08B508F013
:105E7000B5FF00B908BDBDE8084040F005BA00BF55
:105E800008B509F009FC00B908BDBDE8084040F0BC
:105E9000FBB900BF08B509F059FE00B908BDBDE85F
:105EA000084040F0F1B900BF08B50AF087F900B921
:105EB00008BDBDE8084040F0E7B900BF08B50BF0E9
:105EC000BFF800B908BDBDE8084040F0DDB900BF2B
:105ED00070B5830782B0054603D10B4B02689A4226
:105EE0000ED00A4CBE21A61C284601236A4625F086
:105EF000D7FD009820B9B44203D014F8011BF3E792
:105F0000012002B070BD00BF845309007D5E09000E
:105F100038B50023C3714FF0FF33C364054657F013
:105F20000EFA044630BBB5F84E224AF655239A4283
:105F300022D114490B2205F150001FF0F3FEE8B105
:105F400095F85030EB2B03D01833DBB2012B17D868
:105F50000D49032205F186001FF0E4FE40B10B4914
:105F6000052205F1A2001FF0DDFE002818BF022463
:105F7000204638BD0424FBE70324F9E70124F7E7B2
:105F80000224F5E7A8170A00B4170A00B8170A0098
:105F900008B540F20513984207D040F20F1398421B
:105FA000014605D104482BF0FBFE04482BF0F8FE17
:105FB00003482BF0DFFE00BF686D0900546D090037
:105FC0001876090008B543F0C5FB00B108BD0148CB
:105FD0002BF08AFEBC6C090008B543F017FD00B138
:105FE00008BD01482BF080FEBC6C090008B504F028
:105FF000ADFF00B108BD01482BF076FEBC6C090076
:1060000008B505F0A3F900B108BD01482BF06CFEFE
:10601000BC6C090008B5074B0340062B06D083076C
:1060200003D1054B02689A4200D008BD03482BF00B
:106030006FFE00BF0F0080FF545A0900A8780900C6
:1060400010B108B500F002F8704700BF0D2808B580
:106050000FD0014606D804280FD0072811D10A48CE
:106060002BF06AFE43F2020398420AD107482BF054
:10607000D3FD074800212BF0A1FE064906482BF06E
:106080009DFE06482BF076FEB86D09000C700900E5
:10609000F8490900F86F0900C44809003C76090076
:1060A000837A3BB310B5C37A044682B098064FF0AA
:1060B00001024CBF052035200DF1030144F0FCFF27
:1060C000A27A9DF80330134001D002B010BD062023
:1060D0008DF804308DF8052044F0B8FEE37ADA0636
:1060E00009D49B060ED501220DF10501104645F09D
:1060F00075F8EAE7704701220DF10501312045F0FE
:106100006DF8E2E7022201A9012045F067F8DCE71B
:1061100008B502484FF4EB712BF016FE4C6A0900EB
:1061200048B1882808B5014602D003482BF038FE54
:1061300002482BF035FE70472C7609007076090076
:106140002DE9F041064617461D460C4629B1186850
:1061500027F058FA7368834207D1B0682B463A4655
:106160002146BDE8F04122F0C1B901482BF0D0FD35
:10617000E87809002DE9F04F2DED028B8DB08307F3
:10618000029140F030819B4A03689342804640F080
:106190002A8111F0030A40F026810A689A4240F0F1
:1061A000228136F0F7FB002800F02081029D28466E
:1061B00036F0F0FB002800F0198198F8040034F064
:1061C0003BFC04462879029534F036FC039098F89D
:1061D000040036F09FFFD8F80C30D8F8106098F81B
:1061E000042000930AA9814698F807000B930A96A9
:1061F00036F062FC029A009BC169D269D8F81C7023
:10620000049105460792002B00F0D880CDF804A039
:10621000DDF810A00597BB4657464FF0000A002E48
:1062200000F0C9805846A0473846C8470AF1010A1D
:106230006869D8F81830564507449B44F2D106FBEC
:1062400000F006FB03FCA969019B009A081AD8F824
:1062500014100133A1EB0C0C9A4201930744E34460
:10626000DBD1029B059FD8799FED638A03F10C0176
:106270006622019136F020FCDDE901138446069088
:106280006622D879DCF81C30059336F015FCC3691A
:106290000193CDE908654FF00009079EC3464D46BE
:1062A0009846039B30469847384630EE488AA047C8
:1062B000C8EE007AC8ED007ADBE9053202FB15333F
:1062C0001F44029B9B691E44009B09F10105AB42E0
:1062D00017D09FED498ADDF804A04FF0000838463A
:1062E000A047FAEC017ADBF81830C145A0EE278A06
:1062F0001F4408F10108F2D1019BA94603EB850870
:10630000CFE7DDE90865019B68691946009B01EB51
:1063100083020192059A02EB8307049A06F1FF3883
:1063200000FB062B002E3CD0A3EB06094FEA8902A6
:1063300000929946029608F1010AD1459FED2E8AF6
:1063400035D93E465846A0470AF1010AF6EC017AD3
:10635000A969D145A0EE278A8B44F3D8009AA9EB0E
:10636000080303FB01F16FF0030317449B1A019A22
:10637000ABEB010B72ED017A58461F4437EEC88A29
:106380000192A047C8EE007A009B0433009308F105
:10639000FF38C7ED007A6B69ABEB030B029B4345FB
:1063A000C9D806980DB0BDEC028BBDE8F08FA96985
:1063B0006FF00303DBE7B446304644E7029B6622F6
:1063C00003F10C01D87901911F4636F075FB0346A5
:1063D0000690DB69F87901990593662236F06CFB2B
:1063E000C36901938FE705482BF092FC04482BF01A
:1063F0008FFC00BFB02E0A0000000000B87E09002C
:106400007C810900F8B5074628F08CF84610002E6C
:1064100010DD7600002444F00101042238462AF001
:1064200085F80546023408F0E9F9284608F096FC9C
:10643000A642F0D1F8BD00BF0279064950090123F8
:1064400002F01F02934051F82020134341F82030FE
:10645000704700BF604801202DE9F04104298AB04F
:10646000064630D02F4D0C46286819F089FE002CC6
:1064700055D02D4B9C4252D0002701ABCDE9017382
:1064800021462A4B039302A828F086FE0198043087
:1064900020F0030001223946F8F7C8FF286090B1C8
:1064A0000DF1180802680199404650F0D3FC204BCA
:1064B0000593214604A8CDF8108028F06DFE2A68C7
:1064C000019B1268D7541B4DFAF7C0FA41F0E0F86F
:1064D000FDF74AFD1DF034F941F08CF841F072F9F6
:1064E00041F086F818F0AAFAD5F8104100E0E46807
:1064F00020461AF02DFC0028F9D1C5E94344FBF7EA
:1065000013FE4DF05DFB1AF0F9F9304619F038FE34
:1065100048F058FA0AB0BDE8F04149F037B9002315
:106520002B60D0E714570120505401208D660400E1
:10653000256D0800E453012070B582B0FF230546A5
:106540000E46083001218DF8043005F0D9FB0024F7
:1065500001221444686801A904F070FFA642F7D133
:1065600002B070BD2DE9F04F804683B00F469146D2
:106570009A461BB10B8B43F008030B83A7F82090BE
:10658000D8F824201378002B39D0538D002B36D027
:106590000025AB4603E0538D0135AB422CDDD66AB6
:1065A00016F83530043B012B06EBC506F3D8788D81
:1065B0000028F0D0002401E0A04217DDFB6A13F8A8
:1065C0003420052A03EBC40304F10104F4D17168FB
:1065D0005B689942F0D1D8F828007288002322F035
:1065E0005FFD788DA0420BF1010BE7DCD8F8242089
:1065F000538D0135AB42D2DCBBF1000F09D1D8F885
:10660000280053464A46394603B0BDE8F04F22F011
:106610007DBDD8F82800CDF800A04B465A46394633
:1066200022F060FD03B0BDE8F08F00BF2DE9F04718
:106630000446806800EB010A1F460AEB4203052B63
:1066400086B00E4615464FEA42081BD84FEA80092D
:106650004A4604F10C0101A81FF076FB01AB08EBE0
:106660000602394603EB090092001FF06DFB6068DB
:1066700001AB2A46514621F039FF0446204606B0B8
:10668000BDE8F087980000211EF0B2FFA26804F177
:106690000C01920081461FF057FBA06808EB060230
:1066A0003946920009EB80001FF04EFBA16860683C
:1066B00031442A464B4621F019FF044648461EF055
:1066C00095FF204606B0BDE8F08700BF2DE9F043F6
:1066D0001D4683B090F820309DF82C609DF83070F6
:1066E000044688469146002B7ED14FEA196348F054
:1066F00040014FEA2922C9B28DF801304FEA2943FF
:106700008DF803208DF800108DF804908DF802307C
:106710000DF1010C0DF1050E002208235200D2B23A
:1067200082EA010010F0800F03F1FF334FEA4101CC
:1067300018BF82F0090213F0FF03C9B2EED1E6459B
:1067400002D01CF8011BE8E7520042F001028DF86C
:106750000520B7BB60680622694604F06FFEC827B3
:1067600001E0013F46D0FF2360680122694604F042
:106770000FFE9DF900309DF80000002BF1DBEDB11C
:106780003EB3FF238DF801300122FF2360680DEB3B
:10679000020104F0FDFD9DF80130FE2BF4D10A9AB0
:1067A0006068FF23294604F0F3FD6068FF2302229E
:1067B0000DF1010104F0ECFD9DF8000003B0BDE80F
:1067C000F083204650F0CEFB0028C3DA03B0BDE8CA
:1067D000F08360680A9AFF23294604F0D9FD9DF8EA
:1067E000000003B0BDE8F08316F0FAFA0028BFF607
:1067F0007CAFE3E76FF0040003B0BDE8F08300BFB7
:10680000DFED1C7A9FED1C7A60EE277AFCEEE77ACA
:1068100017EE903A1B0207EE903AF8EE677A30EEE8
:10682000670AB4EEC70AF1EE10FA0BD4DFED137A63
:10683000B4EEE70AF1EE10FA17D530EE470A082158
:10684000002201E010210822F0EE087A20EE270A4B
:10685000FDEEC07A17EE903AFF2BA8BFFF23C3F1DD
:10686000FF00884093401843704730EE670A0021CC
:106870001022E9E70000803B0000AA4200002A4302
:1068800041600272704700BF00B583B06A4640683D
:1068900040F24D5125F09CF800216A46084621F04F
:1068A00043FE08E048F040F924F038F9014630B9D9
:1068B0006A4621F039FE27F007FE0028F2D003B027
:1068C0005DF804FB70B59AB00446FFF7DDFF0020C9
:1068D00027F0BCFF01226946064624F03DF807A8D0
:1068E00056F046FDC0B9054603AA606840F29751CC
:1068F00025F06EF8237A06965B0043F0010303AAA5
:1069000029460220059321F00FFE36F0C3FF2046F2
:1069100000F016F81AB070BD204600F011F8089B80
:106920000549186827F09AFD18B1217A03482BF021
:106930000BFA089836F084FF184909000C6F09001B
:1069400000B583B06A46406840F2645125F040F8D3
:1069500000216A46084621F0E7FD03B05DF804FB1C
:1069600010B4019C0261C0E901149DF80C209DF84F
:10697000081003759DF8103001735DF8044B4273E5
:106980008373704710B58AB004466A46406840F287
:106990004D5125F01DF801E024F06EF900216A4602
:1069A000084621F0C1FD27F08FFD03460120002B92
:1069B000F2D060686A464FF42F7125F009F8A2689A
:1069C000217B637B520042F0010242F2D660490013
:1069D000CDE9020241F0010144F2F6305B00CDE95D
:1069E000040143F0010344F20631CDE9061342F2FB
:1069F00086701123CDE908036A460421002021F0A6
:106A000093FD206910B1217D05F07AF960680AB024
:106A100010BD00BFF0B50546006989B020B1297DE1
:106A200081F0010105F06CF9AB7B6BB905AA6868D0
:106A3000019240F2645124F0CBFF0021019A0846F4
:106A400021F072FD09B0F0BD012027F0FFFE022207
:106A500002A9064623F080FF029BFF221A70AB7B3F
:106A60006868073305AADF10A4210192DC0824F02E
:106A7000AFFF019A0796002FD9D000210120019283
:106A800021F052FD631E13F0FF04019AF5D1CEE709
:106A90002DE9F0474160154604460E461F4600F1B9
:106AA0000C0307CA83E8070082B0AB79DDF82C90AD
:106AB000DDF834A0002B3BD12B789AB203FB06986B
:106AC0000025228184F8285008EB0A008DED010A88
:106AD00027F0E4FEE061C6680A994A4630461FF096
:106AE00033F906EB08000C9952461FF02DF9A37CF0
:106AF0009DED010A4E44266263B163689B0009D094
:106B00002946FF2300E0266A735462680431B1EB22
:106B1000820FF8D34FF07E524FF48073A2616381ED
:106B2000204600F043F984F8287002B0BDE8F087F1
:106B300004231A46C2E700BF2DE9F04186B0804623
:106B400003912FF035F90DF11703054601930DF16F
:106B50001603009303990DF1150305AA00F092F8AE
:106B60006B6893B100249DF817709DF816609DF82E
:106B700015309DF814202146CDE90067284600F025
:106B80007BF96B680134A342EDD895F8283013B92E
:106B900006B0BDE8F081404600F00CFA06B0BDE852
:106BA000F08100BF08B52FF003F990F8280008BD68
:106BB00008B52FF0FDF8007B08BD00BF08B52FF029
:106BC000F7F890ED060A08BD08B52FF0F1F8406916
:106BD00008BD00BF08B52FF0EBF8406808BD00BF46
:106BE000B0B500AF0D462FF0E3F8D0E90813027BF3
:106BF000002B08BF0B4605FB0233417B9200073296
:106C000013F801C002F4FF62ADEB020D69464FEAD2
:106C10004C0242F001020A60827B9A5C520042F010
:106C200001024A60C27B9A5C520042F001028A6013
:106C3000027B032A17D9047C827C1B5DC2B103F05E
:106C40001F0307EE903AF8EEE77AB3EE0F7AC7EE3D
:106C5000877A17EE903A23F0030343F00203A3F17F
:106C6000FF43CB60027B104628F06AF9BD46B0BDF9
:106C70005B0043F00103CB60027B104628F060F913
:106C8000BD46B0BD2DE9F04383B00C460B9E0A9F74
:106C9000984691462FF08CF8837C5B423370E30773
:106CA000054611D5204626F09FFC031489F80030D4
:106CB000031288F800303870AB7C13B92A7B042AA1
:106CC00036D003B0BDE8F08314F0030304D1304B99
:106CD00022689A4202D1E5E7022B3CD020466A4660
:106CE00001A926F04DFB0422032140F2AB230198B9
:106CF0001FF090FF009B1868F6F7DAF9009B89F8FF
:106D000000005868F6F7D4F9009B88F800009868EE
:106D1000F6F7CEF9019B3870032BCDD9009BD868CC
:106D200000F00303022B22D026F05EFC3070C8E78F
:106D30006A7C002AC5D099F8001098F800208A4291
:106D4000BFD139789142BCD1317089F8003088F8D0
:106D500000303B70B5E70F4B2340062BBED02046DA
:106D600026F0A4FBFDEEC07A17EE900A9DE7094BD2
:106D70000340062BD8D026F099FBDFED077A20EEF2
:106D8000270AFCEEC07A17EE903A337099E700BFFD
:106D90003C4E0900070080FF00007F4310B50C4601
:106DA0002FF006F880F8284010BD00BF70B52DED1B
:106DB000028B0546B0EE408A2EF0FAFFDFED217A15
:106DC000428980ED068A68EE277AFCEEE77A17EEB4
:106DD000903A9BB29A421ED0068942684381B3F52D
:106DE000807F044602FB06F61FD0416A09B37EB1DC
:106DF0000023A17C09B19A0707D0626A6089D15C3F
:106E0000226A00FB01F10912D15401339E42F0D1F4
:106E100094F8283013B9BDEC028B70BDBDEC028B29
:106E20002846BDE8704000F0C5B8436A002BDED1AB
:106E3000F1E730461EF0DCFB216A606232461EF04C
:106E400083FFD4E70000804330B583B0CDE9002153
:106E500005462EF0ADFF0446DDE90021F6F75AF9AC
:106E600094F828300BB903B030BD284603B0BDE814
:106E7000304000F09FB800BF2DE9F0411D469DF85D
:106E800018709DF81C800C4616462EF091FF038961
:106E9000042B36D004FB03FC446A002C3DD004EBE9
:106EA0000C01046A6444042B04BF037C01F80380D2
:106EB000437BCE54837BCD54C37BCF54A4B1038991
:106EC000042B13D04289437B02FB06F63612E654AC
:106ED0004389827B03FB05F52D12A5544389C27BB0
:106EE00007FB03F31B12A354BDE8F081837C23B995
:106EF000438908FB03F8C8F30728037C04F80380E0
:106F0000E0E7827C002AC5D004FB03FC446A4FEA18
:106F1000D80848F0E008002CC1D1016A6144C2E7FA
:106F20002DE9F04784B00E460D9D904681462EF027
:106F30003FFF694604460C9823F06EFD0E2D1CBFE2
:106F400023896B6007464FF0000A384623F0A4FF00
:106F5000E8B10E2D21D02289BAFBF2F302FB13A374
:106F600002330AF1010A45F823002289BAFBF2F341
:106F700002FB13A3002BE8D1314620462A46F6F740
:106F8000C9F83846464423F087FF0028E1D194F839
:106F900028304BB904B0BDE8F087314602462046A0
:106FA000F6F7B8F84644D0E7484600F003F804B0D6
:106FB000BDE8F08730B585B005462EF0F9FE0446F1
:106FC00001AA284640F2322124F002FDE36903932E
:106FD00001AA0021012021F0A7FA05B030BD00BFB1
:106FE00010B4019C80F80C41029CC0F810415DF87F
:106FF000044B00F025B800BF90F80C31022B04D0F0
:10700000062B08D0012B03D070470430F0F79ABF4D
:107010000430F1F74DB80430F1F70CB890F80C31AA
:10702000022B04D0062B08D0012B03D0704704306C
:10703000F0F7C6BF0430F1F741B80430F0F7FABFFB
:107040002DE9F041041D17461D460E464FF484728B
:10705000002120461EF028FF3DB12B463A4631461E
:107060002046BDE8F041F1F7CBB83A46314620461C
:10707000BDE8F041F1F728B880F80C11704700BF67
:1070800000B583B0F7F78AFEF8F75AF9F8F7BAF8BF
:10709000044640F2FF30019149F06CF801994FF439
:1070A00080630022204648F0F1FC40F0B1FA00BFB6
:1070B00008B542F007FABDE8084019F0E3BB00BF8D
:1070C00030B50A4683B004460D4601460020F6F767
:1070D00011FEF8F797F800231A4648F0D7FC23F082
:1070E0001DFD30B10E200190F7F76EFF019803B03F
:1070F00030BDF5F709FC0138C0B20228F2D8F5F727
:1071000003FC01280CD0022808D129462046F8F7B4
:1071100061F8019042F0E2F90198E4E70E20F8E707
:1071200029462046F7F7DCFDF3E700BF08B59DF8D8
:1071300008C03BB90B792F2B07D84160027280F849
:1071400009C008BD02482AF0F7FD3FF091F800BFE2
:10715000DC8F090040687047007A704708B5F7F780
:107160001DFEF8F7EDF8F8F74DF80023012248F07E
:107170008DFCBDE80840F7F727BF00BF08B5F5F75D
:10718000C3FB022805D003280BD0012805D00E2010
:1071900008BDBDE80840F8F7D5B8BDE80840F7F7E6
:1071A00009BEBDE80840F8F713B900BF22B90A4686
:1071B00001460120F6F79EBD08B502484FF48961EB
:1071C0002AF04EFD108E090001EB030CBCF5807F08
:1071D00000D9704710B4044C104621441A465DF89B
:1071E000044B1EF0B1BD00BF205E01204FF4807043
:1071F000704700BF01EB030CBCF5807F01D9002074
:10720000704710B5044C0846204411461A461EF03B
:107210009BFD012010BD00BF205E012080ED010A12
:10722000704700BF90ED010A704700BF08B500200D
:107230002AF00EFD08B5F5F767FB0138C0B2022849
:107240008CBF0020012008BD38B54B79A3B10B7964
:107250001F2B88BF03F01F030C4603F5E0738CBFA0
:1072600006494FF0A0410546022241F8232020465E
:10727000FFF7E2F86C6038BD3EF0FAFF0003005003
:107280004368ABB110B51B791F2B86BF03F01F03FA
:1072900008494FF0A04103F5E073022241F8232092
:1072A00043680446187940F06FFA0023636010BD0C
:1072B000704700BF000300504068B0FA80F04009FA
:1072C000704700BF9FED010A704700BF3333534042
:1072D00010B485B0314B4FF6FF74ADF80240002179
:1072E00003220124C3F8F025C3F8F4150A46C3F8B5
:1072F0000045130103F1804303F5E0430132082AFE
:10730000C3F81415C3F81015F3D1244B4FF4905261
:10731000C3F81825416801224979C3F814150DF105
:107320000200C3F81015C3F82C06C3F830261A6003
:10733000D3F80021002AFBD00022C3F80021D3F8A3
:10734000002101921549019801225A60D1F80431B7
:10735000002BFBD00023C1F80431D1F80431029393
:107360000E4A029801238B60D2F81431002BFBD017
:107370000020C2F81401D2F814310393039BC2F821
:107380000005BDF90230834203DB181340EA830095
:1073900080B205B05DF8044B704700BF007000403C
:1073A0004EF054BB08B502484FF481712AF058FCE6
:1073B000108E0900704700BF01207047704700BF62
:1073C0002DE9F8431D461D4B9DF82090D3F8008011
:1073D000B8F1000F2FD116460446186008460F4634
:1073E000FFF72AF83046FFF727F82846FFF724F87A
:1073F00013493B7984F82130C1F86435337984F836
:107400002230C1F868352A7984F823200123C1F895
:107410007025C1F80485C1F80885C1F80C35C1F89C
:107420001035C1F81C35C1F82085C1F82495BDE898
:10743000F84346F09BBF03482AF056FCF44F012066
:1074400000500240F86A090090F82330FF2B20D04A
:1074500070B5104B0122002604465A60C3F800653F
:10746000FF2590F8210040F08FF994F8220084F86D
:10747000215040F089F994F8230084F8225040F01C
:1074800083F9054B84F823501E60BDE8704046F038
:1074900025BF704700500240F44F012090F82300B0
:1074A000A0F1FF00B0FA80F04009704790F8260084
:1074B000C0F3C000704700BF084BD3F8082142B1A9
:1074C00090F8262000216FF3410280F82620C3F8AF
:1074D000081190F82600C0F34000704700500240A9
:1074E00090F8263043F0080380F82630704700BF3C
:1074F0002DE9F04F2DED028B7A4BD3F8086185B062
:1075000005460C4646B190F826106FF3410180F80D
:1075100026100021C3F8081195F826309B070BD5DB
:10752000704901234B6095F8263043F0040385F839
:1075300026302023C1F8083395F826306C6062F3BA
:10754000041385F826302046FAF700FD034620464E
:1075500008EE103AFAF79AFC05F12403C00803AAD2
:1075600085F825000121CDE9002320460DF10B030C
:107570000DF10A02FAF7BEFC9DF80B309DF80A00E7
:1075800095F8261095F82520DFF858A1564C574E4F
:107590005B0143EA8013013A03F0600321F06001CC
:1075A00043EA010318BF012285F82630CAF81C25DA
:1075B00095F82430A3F10103B3FA83F300275B09A4
:1075C000CAF82835B7EE006AB846B946BC460AE0A4
:1075D00004EBCC034FEACC0E9B7953B90CF1010CB0
:1075E000BCF1090F32D0DAF81C35012BF0D04FEA8C
:1075F000CC0E3F4AF8EE486A02F15800A6445168A2
:10760000BEF9043096FBF3F393FBF1F307EE903AE7
:10761000F8EEE77AD2F800B054F83C1076EEE77A4C
:107620000832F0EEE77A87EEA67AB4EEC67AF1EE8B
:1076300010FA04D5B0EE476A1F46D84689469042F4
:10764000DDD10CF1010CBCF1090FCCD1254CC4F8F3
:107650001895C4F8148595F8243095F825006F83A3
:1076600010FB03F018EE103A03FB00F0214B000171
:10767000A3FB00308009033020F0030080B200211A
:1076800028831DF0B5FF0346AB60288B00211DF059
:10769000AFFF00221146E8606868FAF745FC95F8EC
:1076A000263023F00E03002243F00203C5E9042232
:1076B00085F8202085F8263028461AF00FF92B8B04
:1076C00001229B082021C4F85035C4F80413C4F8E3
:1076D000002522601AF0DEF805B0BDEC028BBDE893
:1076E000F08F00BF00500240A80301200048E801CD
:1076F000B0020120D34D621090F826306FF3C3031F
:1077000080F82630704700BF064A0123536090F886
:107710002630202143F0040380F82630C2F80813F5
:10772000704700BF005002402DE9F843044615465B
:1077300008461F460E469DF824909DF82080FEF7CF
:107740007BFE2846FEF778FE84F806903179217199
:107750002B796371B7F57A5F20D1B8F1100F20D182
:10776000114B1B68C3F840156579C3F844554FF0B9
:107770000464C3F80445012228200C490024C3F8FE
:107780002045C3F81805C3F81C05C3F80025C3F845
:107790006015C3F864251A60BDE8F88304482AF030
:1077A000CBFA04482AF0C8FA64030120144D0120E2
:1077B000A48609009486090038B5084B1B6800228E
:1077C0000446C3F800250079FF253FF0DDFF60790E
:1077D00025713FF0D9FF657138BD00BF64030120FA
:1077E0000079A0F1FF00B0FA80F04009704700BFB7
:1077F000102070474FF47A50704700BFF8B51D4F06
:107800003B6815460122C3F80825C3F86015C3F884
:107810006455194B064643F001034FF448500C469B
:1078200098473B68154A0021C3F80811C3F8602542
:107830000122C3F86425D3F8083133B947F074F94D
:107840003B68D3F80831002BF8D055B104EB450262
:10785000A11E023A31F8023FA3F500438A420B8091
:10786000F8D1B37913B125F00100F8BD25F003007C
:10787000F8BD00BF6403012030AD0900144D0120A4
:10788000DB009DF800C003738260029B9DF804201A
:1078900080F80DC04160827303617047002343602C
:1078A000704700BF4068B0FA80F04009704700BFE1
:1078B000007B7047807B70470069704701617047AB
:1078C00070B504468EB00163164601F1080000222F
:1078D0001D46002354F00EFB206B01AB0830102234
:1078E00005A954F080FE002840F08780019B102BF2
:1078F00003D1059A474B9A4203D040F239301FF02A
:107900009BF8079AA3F57003A3F2FB739A42F4D194
:1079100003F15B43089A03F5F11303F60F439A4210
:10792000EBD1206B01AB0830042202A954F05BFEBE
:10793000002862D1019B042B65D1029A142A62D8D7
:10794000206B01AB083009A954F04DFE002854D13A
:10795000BDF824300299012B52D1BDF82620022A0D
:107960004ED8BDF83230102B4AD8122903D1BDF8B9
:107970003410002944D1206BA3760A9B84F824207C
:10798000A362083001AB042203A954F02CFE0028A6
:1079900033D1019A042A03D103991F4B994202D093
:1079A0001E482AF0C9F9206B01AB083004A954F035
:1079B0001AFE10BB019B042B9FD1049A236B6261BA
:1079C0001B6C238335B16D087319E5626660E36053
:1079D0000EB070BD4FF48070E06229461DF008FEC5
:1079E000606098B1E06A29461DF002FEE060002860
:1079F000EED1E06A65601DF00BFE05202AF03CF92F
:107A000007482AF099F907482AF096F9E06AE560F4
:107A10001DF0FEFD5249464664617461A06A09008A
:107A2000BC760900E86D090000234360C36070471D
:107A30004068B0FA80F04009704700BF807E704710
:107A400090F82400704700BF806A704781627047D9
:107A50002DE9F0410446D0088000E0600D46002189
:107A60009DF818809DF81C701E461DF0C1FD6060D9
:107A700080B1E06800211DF0BBFD0246A06070B13E
:107A8000089B267484F81280E774636184F824509C
:107A9000BDE8F0810246A260E0681DF0B9FDE06833
:107AA00062601DF0B5FD00BF0023C0E901337047DF
:107AB0004068B0FA80F04009704700BF007C704712
:107AC000C07C704738B590F824308BB1002405464F
:107AD000234603E095F824209A4209D905EB830355
:107AE0000134D86A00F014F8E3B20028F2D038BDAF
:107AF000002038BD4069704700224FF40043826087
:107B000003837047038B00EE103ABBEEE80A704720
:107B10008068003818BF0120704700BF70B5044668
:107B200084B008460D461646FAF710FA63685B699A
:107B300098423CD12846FAF7B7F96368DB7C834268
:107B40003ED12846FAF7A2F963681B7C834234D100
:107B50000DF10B0203ABCDE9003200210DF10A0358
:107B60000DF109022846FAF7C5F962689DF80A3056
:107B7000927C9A421ED1002211462846A5602673A7
:107B8000FAF7D2F9002204F114030093114604F12C
:107B900010032846FAF796F96369A0F10100B0FADC
:107BA00080F040099B086361607304B070BD0648B3
:107BB0002AF0C2F805482AF0BFF805482AF0BCF8B8
:107BC00004482AF0B9F800BFE4730900FC73090007
:107BD000B4730900CC730900DFED047A20EE270AA4
:107BE000BCEEC00A10EE103A038370470000004755
:107BF0004160704700238360704700BFF8B50446BA
:107C00004FF40060C4E907000F46002115461E46E8
:107C10001DF0EEFCA06190B3F1F72CFA606038B370
:107C2000EB0744BF06F1FF360135B6F5105F09D307
:107C300005F59053C4E9095339462046BDE8F8409C
:107C400000F084B800214FF490501DF0D1FC606228
:107C500038B100214FF490501DF0CAFCA0620028FA
:107C6000EAD1204600F016F84FF490501DF0D0FCF9
:107C7000204600F00FF8054905482AF09FF82046F5
:107C800000F008F8E0691DF0C3FC00BF686A090055
:107C9000C448090010B504464068F1F797F900237D
:107CA000C4E909336360A361A363636410BD00BFCB
:107CB000406AB0FA80F04009704700BF102070475A
:107CC00090F83D00704700BF90F83C30026B00EB2D
:107CD000830351085B6A1DD003EB41029FED180A34
:107CE000023B023A33F902CF07EE90CAF8EEE77A88
:107CF0009A42A7EEA70AF5D1B5EE400AF1EE10FAC6
:107D00000BD4F1EEC07A07EE101AB8EEC70A87EE70
:107D1000800A70479FED0A0AF3E700B583B001902F
:107D200043F0BCFA0198016B490807EE101AF0EE17
:107D3000407AB8EEC70A87EE800A03B05DF804FB0C
:107D400000000000406B7047406C704730B504463F
:107D50000D4689B0FAF7CEF900220023A56305F19C
:107D6000080054F0C7F8E26922624FF47F43E387CA
:107D700020461EF02DFE20461EF07EFD606A4FF468
:107D8000905200211EF090F8A06A4FF4905200210A
:107D90001EF08AF808E0236A0133236220461EF0B1
:107DA0006BFD94F83E30C3B9A269236A60681A4437
:107DB00001A9F1F745F905460028ECD1FAF79CF93D
:107DC000DDE90221059B84F83D205A009B00C4E9AF
:107DD0000B326163656409B030BDFAF78DF9024971
:107DE000024829F0EBFF00BF286C09006C4909002C
:107DF000416370472DE9F04182B0002504461C30F4
:107E0000019000950F461646984601222B462946BA
:107E10004FF480703DF012FEA06000B3C0F80C5526
:107E2000A3680122C3F81025A3683D79257638465A
:107E3000C3F86055FEF700FB3EB1A2683379637664
:107E40003046C2F86835FEF7F7FAA2684FEA182301
:107E50000121A382C2F8001502B0BDE8F0810148FB
:107E600029F042FF908B090038B58368E3B10446DE
:107E70000FF012FFA3680022C3F80025207EB8B9D6
:107E8000607E90B9A06800213DF024FE002502210B
:107E9000A0683DF01FFEE068A5601DF0A7FB20690B
:107EA000E5601DF0A3FB256138BD3FF06DFCE9E7FF
:107EB0003FF06AFC607E0028E4D0F6E78068B0FA04
:107EC00080F04009704700BFC07F7047C37F33B95F
:107ED0008268D2F8041111B14377C2F80431407FAF
:107EE000704700BF836801210222C177C3F80022D6
:107EF000704700BF70B5C37F84B004460D46164678
:107F00002BB98268D2F80411002940F09A80637F6F
:107F1000002B40F09D80656084F820602846FAF7C9
:107F200015F806462846F9F7B1FF0DF10B03C00816
:107F300003AAE076002128460193009204F1210370
:107F400004F12202F9F7D6FF2846F9F7ADFF4FF406
:107F500022724FF6FF71A07603981EF043FEBDF823
:107F60000C50AD00002128461DF042FB94F8221071
:107F7000E060002970D006F574452335B5FBF6F5B1
:107F800006FB05F35D0805F5740505F51055B5FB11
:107F9000F3F56A08A16802F5740303F51053B3FB07
:107FA000F5F202EB5602B2FBF6F3013BC1F848359D
:107FB000A168C1F82835A3686A1EE282C3F8085593
:107FC000A3680122C3F81425002260681146F9F75E
:107FD000ABFF26480023024652F8041B002940D07C
:107FE0000133042BF8D1A36800250422A577294684
:107FF000C3F80022204616F025FEA368D3F82025FA
:10800000C3F84025A368D3F82425C3F84425A26803
:10801000C2F80851A268C2F80C51A268C2F8105107
:10802000A268C2F81451A268C2F80451A2680C21D7
:10803000C2F80413A268012393606377E57704B064
:1080400070BD4377C2F80431637F002B3FF463AF08
:10805000204600F01DF85EE728461DF0C9FA2061B1
:1080600089E740F8234046F081F9BCE798470120B2
:10807000836804210022C277C3F800128368D3F812
:10808000041121B1C3F80421836801229A6070476A
:1080900038B504460FF000FEA36801225A6000259F
:1080A000E068E5831DF0A2FA2069E5601DF09EFA04
:1080B000256138BD2DE9F04F2DED028B89B0CDE95A
:1080C00002219946F0EE408A43680693002605A9EE
:1080D000B0EE608A05460596079611F0F9FAF0EEC3
:1080E000687AFEEECC7AB9F1090F17EE90EAF0EE5D
:1080F000487AFEEECC7A17EE904A00F09080E9883C
:1081000009F0FB09002900F08580AB88019641F653
:10811000F07A039E019AB789B5F80C8002FB07F04C
:10812000029FB7F80CC0B76802FB08F802FB0CFC12
:10813000AA6802EB8808029A926807EB800702EBB4
:108140008C0C0026002B41D15EE013F5F84348BFAC
:10815000FF331B1223EAE37303F478431BB202F4E8
:10816000FC6B01F4FC6004FB0BFB0EFB00BB5248F4
:10817000834545DC1BF57C7048BF0BF2EF400012D5
:1081800020EAE07000F4FC6002F01F0201F01F0121
:1081900004FB02F20EFB012151452FDC11F10F0B04
:1081A00048BF01F5877B4FEA2B2222EAE27212B226
:1081B00003431343B9F1030F9BB201D15BBA9BB2E6
:1081C00028F8023BAB880136B3421CDDB9F1030F3E
:1081D00037F8021B3CF8022B03D149BA52BA89B2D4
:1081E00092B202F4784301F4784004FB03F30EFBEF
:1081F000003332488342A8DB314BB0E71F22D7E778
:108200004FF4FC60C0E7E988019A01329142019283
:108210003FF77FAF09B0BDEC028BBDE8F08FE98876
:108220000029F7D0DDE9028CAB884FF67F708B46D2
:10823000AF89AA68B8F80C90D8F8081006FB07F7C1
:1082400002EB8707BCF80C2006FB02FADCF80820DA
:1082500006FB09F901EB890902EB8A02002183B9C7
:1082600022E013F1800A48BF03F27F1A4FEA2A2363
:1082700023EAE373DBB207F8013BAB8801318B42A1
:1082800010DD19F8013B12F801AB04FB03F30EFB00
:108290000A338342E5DDFF2307F8013BAB88013158
:1082A0008B42EEDCB5F806B00136B345C0DC09B050
:1082B000BDEC028BBDE8F08F0FDD07000085F700F5
:1082C00000F8FFFF2DE9F04F89B015460393139F87
:1082D0009DF854B082460E4603F0AAFE0123149A7C
:1082E00003FA00F0129B934232DA129B029300F1E0
:1082F000FF39039BBB4225DA039CBDF90880019638
:1083000012E013F801CB019321B20CEA0903013406
:1083100042465046BBF1000F02D0169EB44501D034
:1083200011F0FAF9A7420CD0022D019B05D0042DC3
:10833000E7D153F804CB0193E6E733F802CB01937E
:10834000E2E7019E029B149A01339A420293D0D134
:10835000039B129AADF81430ADF816200023149A3E
:10836000ADF81870504605A9ADF81A20079311F022
:10837000AFF909B0BDE8F08F2DE9F04F8DB0DDF811
:108380005880434500F0EF800F460021054608461F
:108390009946164626F080FC0446384626F0EAFB4D
:1083A0000790304626F0E6FB07A90890022026F049
:1083B000C7FD0146204626F0EDF86FF000439845D2
:1083C00000F0E8804FF0000A03AA04A92046CDF887
:1083D00010A026F01FF9049BCDF814A0CDE900678A
:1083E0000DF1240B93B9ABE0069B586825F02CFEE9
:1083F000EB8801309842C0F2B98003AA04A9204654
:1084000026F008F9049B002B00F09A8003AA04A927
:10841000204626F0FFF80021204626F045F906AA5E
:1084200005A928F045F9069B186825F095F8069BE4
:108430008246586825F090F80FFA8AF102B2284671
:1084400003F01AFE8045D8D1069B186825F0FCFD84
:10845000069A8246506825F0F7FD019B5745C8BF34
:108460000FFA8AF75345BCBF0FFA8AF30193009BBA
:108470008642C8BF06B28342BCBF03B20093069BCC
:10848000186825F069F8069B8246586825F064F85C
:108490004B4602B20FFA8AF1284611F03DF9069BCD
:1084A000586825F0D1FD002812DD069B1A68099254
:1084B000586825F0C9FD431E5B0043F0010359468F
:1084C00002200A9326F03CFD0146204626F062F881
:1084D000069B186825F0B8FD002813DD069B186878
:1084E00025F0B2FD431E5B0043F001030993069B98
:1084F00059465B680A93022026F022FD0146204679
:1085000026F048F8069B186825F09EFDAB880130E0
:108510009842BFF669AF069B186825F095FD431C8D
:108520005B0043F001030993069B59465B680A937D
:10853000022026F005FD0146204626F02BF853E7E1
:10854000019BADF8247003F1010A009BADF8266091
:108550000133002259462846ADF828A0ADF82A304C
:108560000B9211F0B5F80DB0BDE8F08F069B1A68BC
:108570000992586825F068FD431C5B0043F0010335
:10858000594602200A9326F0DBFC0146204626F0DD
:1085900001F832E7079824F0DFFF8046089824F0BE
:1085A000DBFF0FFA88F102B2284603F065FD804632
:1085B00008E700BF2DE9F04F95B002AFC4887C6199
:1085C000B961446881883C60032A07EE100AF961AA
:1085D00000F06A8102F0FD01A2F10702B2FA82F214
:1085E0005209052906EE902A03D142F0020206EE56
:1085F000902AAF4A52F82340FB6962784FF0020894
:108600000321184611FB023118FB023303EB43032D
:108610005B0007336D46DB08A5EBC3039D4602EB09
:10862000820300F11F065B0003EB8003761102A8B2
:108630006D46C318A5EB461500EB410600EB420161
:10864000B8697B62AD46BB63C388BE6202ADC7E951
:108650000B1107EE905A7E63F3B1009200230A4695
:1086600016EE901A16F072FBC2886378B861012A80
:1086700012D900933246012316EE901A16F066FBCB
:10868000BA696378D288424506D900937A6A16EEB1
:10869000901A434616F05AFB7B69002B00F0F580D8
:1086A000FA69531EFB605B007B6017EE903A4FF057
:1086B00000085200C3F101053A61C7F82080BD608F
:1086C000FB69002B47D017EE903AFA6AD7F808B04A
:1086D00003F1FF3E3B69914603EB020A39F9026B55
:1086E00046447F2ECCBF012300230BEB0E0C0EF86B
:1086F000013FB6B2C8BFFF3E2378C8BFB6B236B29C
:10870000FBB12246002092F9045092F9031092F92D
:10871000053007F1480808EB8505614455F8185CF9
:1087200013FB06F3002B35F81180B8BFFF3308EBBD
:10873000232325F8113023780130834202F103020C
:10874000E1DCA37803FB06F6002EB8BFFF36CA456E
:1087500046F30F28C2D13D6A17EE902A294617EE3C
:10876000100A4EF049FEBA6A3A637A6A7A637A6905
:10877000FE6ABE632B460135AA4200F08680B869C6
:10878000C28803339A4206DD6278009216EE901A90
:10879000324616F0DBFAFB69D7F80C90002B4DD06F
:1087A000BB6A7A6803EB020B17EE903AFA69C4468B
:1087B00003EB020A3BF9023963440FFA83FCBCF174
:1087C0007F0FCCBF012200229BB20AF8012DC4BF4B
:1087D000FF3B0FFA83FC237803B32246002092F973
:1087E000046092F9031092F9053007F1480E0EEB80
:1087F0008606A9EB010156F8186C13FB0CF3002B4D
:1088000036F811E0B8BFFF330EEB232326F8113002
:1088100023780130834202F10302E0DCA3780CFBF1
:1088200003FCBCF1000F09F1FF39B8BF0CF1FF0CDC
:10883000B9F1FF3F4CF30F2CBCD1E04617EE902A64
:1088400017EE100A29464EF0D7FD7B6AB8693B63E4
:10885000FB6A7B633B6AC288B96AB96304339A4294
:1088600006DD627800920A4616EE901A16F06EFA4D
:10887000D7E909313A6A79627969023291423A62FA
:1088800003DDFA6AC7E90A231AE73A68002307F109
:108890003C0117EE100AC7E91023FB6310F018FF24
:1088A0004C37BD46BDE8F08F012206EE902AA0E6C7
:1088B000780001202DE9F04F2DED048B87B099420F
:1088C000BDF95080DDF854900C461F46064615460B
:1088D00080F289805A1C454512B2084680F2898090
:1088E00008F101031BB22946ADF806300023CDE99B
:1088F0000233ADF80000ADF80210ADF80420059386
:108900006A467368049303A9684610F057FC6946E9
:10891000304610F0DDFEBC427FD045456DD0A8EB5F
:10892000050AA7EB040BBAF1000FB8BFCAF1000AA1
:10893000BBF1000FB8BFCBF1000BDA4543462A4626
:108940003846214605DD3B46224647462C468046B2
:108950000D46BC4208DD9C46284621461346454646
:108960003C46624680460F469B1A002BB8BF5B42CE
:108970001AB23B1B19B2C3F3C0330B445B1007EEB2
:10898000903A4545B4BF4FF001084FF0FF38BC4264
:1089900009EE101AB8EEE78A20DC07EE902AF8EE0E
:1089A000E78ADA4522464B4629463046DFBF214654
:1089B0002A464B46304610F0AFFE38EE688A013446
:1089C000B5EEC08AF1EE10FA24B205D5F8EEC97AF8
:1089D000454438EE278A2DB2A742E2DA07B0BDEC53
:1089E000048BBDE8F08F4A1C454512B21846FFF6CD
:1089F00077AF6B1C1BB2414676E7BC4202DD2346D3
:108A00003C461F46214601344B462A46304624B296
:108A100010F082FEA742F5DAE0E7454502DD2B467D
:108A2000454698462A4601354B46214630462DB2EA
:108A300010F072FEA845F5DAD0E700BFF0B587B0B8
:108A400006460024ADF804306846BDF93030ADF874
:108A50000010ADF80220ADF806300D9F029410F022
:108A60009BFB736805946A4603A96846CDE90343F6
:108A700010F0A4FB6946304610F02AFEBDF9005004
:108A8000BDF90430AB4217DDBDF90620BDF9024047
:108A9000A2420DDD22463B462946304610F03CFE00
:108AA0000134BDF9062024B2A242F3DCBDF9043042
:108AB00001352DB2AB42E9DC07B0F0BD2DE9F04F36
:108AC0002DED028B93B000AF904697F878407C6311
:108AD00097F87C407C6297F880407A6106461D4694
:108AE0008A46BB6108EE901A3C6203F0A1FA0121AC
:108AF00001FA00F000F1FF39504621F06FFF002429
:108B00007368B86207F13C0130463B64FC637C64E7
